:020000040000FA
:100000000002040000000000EEA20000EEA20000CA
:10001000EEA20000EEA20000EEA20000EEA20000A0
:10002000EEA20000EEA20000EEA20000EEA2000090
:10003000EEA20000EEA20000EEA20000EEA2000080
:10004000EEA20000EEA20000EEA20000EEA2000070
:10005000EEA200000079000026790000EEA2000068
:10006000EEA20000EEA20000EEA20000EEA2000050
:10007000EEA20000EEA20000EEA20000EEA2000040
:10008000EEA20000EEA20000EEA20000EEA2000030
:10009000EEA20000EEA20000EEA20000EEA2000020
:1000A000EEA20000EEA20000EEA20000EEA2000010
:1000B000EEA20000EEA20000EEA20000EEA2000000
:1000C000EEA20000EEA20000EEA20000EEA20000F0
:1000D000EEA20000EEA20000EEA20000EEA20000E0
:1000E000EEA20000EEA20000EEA20000EEA20000D0
:1000F000EEA20000EEA20000EEA20000EEA20000C0
:10010000EEA20000EEA20000EEA20000EEA20000AF
:10011000EEA20000EEA20000EEA20000EEA200009F
:10012000EEA20000EEA20000EEA20000EEA200008F
:10013000EEA20000EEA20000EEA20000EEA200007F
:10014000EEA20000EEA20000EEA20000EEA200006F
:10015000EEA20000EEA20000EEA20000EEA200005F
:10016000EEA20000EEA20000EEA20000EEA200004F
:10017000EEA20000EEA20000EEA20000EEA200003F
:10018000EEA20000EEA20000EEA20000EEA200002F
:10019000EEA20000EEA20000EEA20000EEA200001F
:1001A000EEA20000EEA20000EEA20000EEA200000F
:1001B000EEA20000EEA20000EEA20000EEA20000FF
:1001C000EEA20000EEA20000EEA20000EEA20000EF
:1001D000EEA20000EEA20000EEA20000EEA20000DF
:1001E000EEA20000EEA20000EEA20000EEA20000CF
:1001F000EEA20000EEA20000EEA20000EEA20000BF
:10020000FFFFFF00FFFFFF00EEA20000EEA20000D4
:10021000EEA20000EEA20000EEA20000EEA200009E
:10022000EEA20000EEA20000EEA20000EEA200008E
:10023000EEA20000EEA20000EEA20000EEA200007E
:10024000EEA20000EEA20000EEA20000EEA200006E
:10025000EEA200000079000026790000EEA2000066
:10026000EEA20000EEA20000EEA20000EEA200004E
:10027000EEA20000EEA20000EEA20000EEA200003E
:10028000EEA20000EEA20000EEA20000EEA200002E
:10029000EEA20000EEA20000EEA20000EEA200001E
:1002A000EEA20000EEA20000EEA20000EEA200000E
:1002B000EEA20000EEA20000EEA20000EEA20000FE
:1002C000EEA20000EEA20000EEA20000EEA20000EE
:1002D000EEA20000EEA20000EEA20000EEA20000DE
:1002E000EEA20000EEA20000EEA20000EEA20000CE
:1002F000EEA20000EEA20000EEA20000EEA20000BE
:10030000EEA20000EEA20000EEA20000EEA20000AD
:10031000EEA20000EEA20000EEA20000EEA200009D
:10032000EEA20000EEA20000EEA20000EEA200008D
:10033000EEA20000EEA20000EEA20000EEA200007D
:10034000EEA20000EEA20000EEA20000EEA200006D
:10035000EEA20000EEA20000EEA20000EEA200005D
:10036000EEA20000EEA20000EEA20000EEA200004D
:10037000EEA20000EEA20000EEA20000EEA200003D
:10038000EEA20000EEA20000EEA20000EEA200002D
:10039000EEA20000EEA20000EEA20000EEA200001D
:1003A000EEA20000EEA20000EEA20000EEA200000D
:1003B000EEA20000EEA20000EEA20000EEA20000FD
:1003C000EEA20000EEA20000EEA20000EEA20000ED
:1003D000EEA20000EEA20000EEA20000EEA20000DD
:1003E000EEA20000EEA20000EEA20000EEA20000CD
:1003F000EEA20000EEA20000EEA20000EEA20000BD
:100400006F242200007F220000018800000000000D
:100410000C000700C06F2900010020001100070038
:10042000000020000000E000020032000000020096
:100430000000000036A20200000000000040DA00C8
:100440000000FE004440A900403120000000E00010
:100450000300320000002000A00188004440A800F2
:100460000000060091018800800078000000EB0089
:1004700015003700E280400032A0B4009101BA00BC
:10048000E280400032A0B4009102BA00E280400055
:1004900032A0B4000002EB00472BDE00F507B200EB
:1004A000602CE10004003A000059EB008301E900F0
:1004B000FDFF3E00040037006128E100010032002A
:1004C0000082EB00040007001101BA000200E00006
:1004D000E8FF3A00000006003159BA008301E90044
:1004E0000C0032002159BA008301E90008003200F3
:1004F0000400E00003003A00E280400032A0B400B3
:10050000F5FF370011D9BA008301E900FAFF3A007C
:100510008100E800E180400032A0B4000000060045
:1005200000000000000000000000000000000000CB
:1005300000000000000000000000000000000000BB
:1005400000000000000000000000000000000000AB
:10055000000000000000000000000000000000009B
:1007E0000000000000000000889FBE008A9FBE003D
:1007F000010578000100E0000400350008003C001D
:100800000000E0002000320005003700600010000A
:10081000E080180002003B0001F02C001A003700B5
:100820000004BE006011B8006B0920000982CF00EF
:10083000020039000882CF000441B0006942520032
:100840000E00320008003B008281710061016400EB
:100850008904D1000884D3008B05E8000442E80035
:10086000F9FF3A00050037000804440089844C0071
:100870008B05E9000442E900FBFF3A002C01070068
:100880000AF0A70001F0A0004F05BE004F04BE0013
:1008900000000600F4FF2F004B0137001400200079
:1008A00049013700889FBE008A9FBE008C1F7800D8
:1008B000600107006701330003866C006450E100AB
:1008C0002E0032006420E100330032006150E1006C
:1008D0002F0032006120E100310032008585550093
:1008E000EB07B000090020000804200005003700D5
:1008F0000804440089844C000A00310006034300C8
:1009000087834B000001530081815B00F8FF3300B7
:100910000203BE000800A0000804440089844C00C3
:10092000F6FF3900C639DD00830173000100320093
:10093000130020008904D1000884D3000998A30083
:10094000050032000800A7000300A0008904D100C0
:100950000884D3008B05E8008904D1000884D30003
:100960000001EB000281D200F100070001F0A100BC
:100970000CF0A70001F0A0003F0137006420E10067
:10098000410132000801BE000200BE00F7FF37003F
:100990006120E1003C0132006000B800F3FF370045
:1009A0000000200001F82700F0FF370003F0A2004C
:1009B000889FBE008A9FBE008C1F78001D01070023
:1009C000240133006450E1004F0032006420E10054
:1009D0005200320003826C0007003B000905D00082
:1009E0000306D000820F54000C065D00020039009F
:1009F00002003200890178000306780085825500E4
:100A000004003D000003FD008103FD008502EA00B3
:100A10008B854200840F720002003B0060001000D2
:100A2000E08018006011B8000005EB007A28E100B2
:100A30000A00390006007800C75DDD00F707B20044
:100A4000878075002D003700828171000A017800CF
:100A5000610560008180D1000080D3008502E9003B
:100A6000F9FF3B00060440008784480002003B0079
:100A700060041400E0841C000988A3000700320011
:100A80008A81710082817100610164008904D10052
:100A90000884D3008B05E800170037000978A3000D
:100AA00013003A000B00E000130034008B05E9004E
:100AB0000804440089844C000A4474000978A300A7
:100AC0000D003A000B00E000070034008B05E90040
:100AD0000804440089844C0001003A000B00200007
:100AE0000978A300F7FF32000001EB000200370095
:100AF000828171000A0178008D0007000CF0A700C8
:100B000001F0A000DC0037006420E10002003A00A0
:100B1000838F6C00DC0033000801BE000200BE00C1
:100B2000D5003700889FBE008A9FBE008C1F7800CA
:100B3000C0000700C700330003866C006450E1006A
:100B4000240032006420E100270032006150E100FF
:100B5000220032006120E100210032008B8542003A
:100B6000EB07B1000134B800003AB80008044200B5
:100B700089844A00013AB8000030B80088804000FB
:100B800009014A0004003300000040008180480051
:100B9000020149008B05E900C909DD0083017000ED
:100BA0000100320013002000C814DE004814DD00EC
:100BB0004709DE001200B200C808DE000884700099
:100BC0005B00070001F0A1000CF0A70001F0A000FD
:100BD000A90037006120E100AB0032000801BE002F
:100BE0000200BE00F7FF37006150E100FCFF3A0051
:100BF000A50037000001BE00A60007000470A70092
:100C000003F0A10003F8A30013003A006509B10046
:100C100010003200090035006928E10002003500AB
:100C2000010028000000050000004000818048000D
:100C30008502E900FCFF3A0000000600F88F420040
:100C4000050035008100D1000080D3008502E80056
:100C5000FCFF3A00000006008000EB0000000500E9
:100C60006022B800060220000000D0008180D2007F
:100C70000482D2008582D2000000A000020252004D
:100C800083825A00030031000202420083824A003C
:100C90000000A1000603E900F3FF3A00000006008F
:100CA000EFFF07000400BE00000006000001BE00C8
:100CB000780007000470A70003F0A1006509B100E7
:100CC000160032000D0035006828E10006003500EE
:100CD000F0FF2F00F1FF27000300E00013003B00AE
:100CE000010028000000050000004000818048004D
:100CF0008502E900FCFF3A0008003700F88F420047
:100D000002003C008000EB00000005008100D100E3
:100D10000080D3008502E800FCFF3A000300E000F9
:100D200002003B0060001000E08018000000060098
:100D300081002000618055000B003D000B00200069
:100D400061FE2F000100E1001D003400828171006E
:100D5000610164008904D1000884D3000000E80028
:100D6000FAFF3A0071002000610064000300700087
:100D7000020060000900320061044400E0844C007D
:100D80000988A500050032008B05E8006808E1002D
:100D900002003A008904D1000884D300F20F200039
:100DA0000258E10005003D00C75DDD00F907B20013
:100DB0008980750008007800000006000BF8270005
:100DC0008B00780000000500889FBE008A9FBE004F
:100DD000841F7800170007004F00780011003300CF
:100DE000F0FF2F00838F6C0006003B0004056500B8
:100DF0000A00A7000800370009F0A6001000200034
:100E000008003700820F5400838F5C000300390014
:100E10001000200001003E000000200009F0A700A3
:100E20000000EA004F05BE004F04BE000000E000D5
:100E3000000006000004BE00160007000003BE000C
:100E40000405BE000200BE0012000700844F7500BA
:100E5000000006000200BE006450E10005003600FC
:100E60006420E100020036000968A30001003A0096
:100E70000800BE000160A0004F0678004F05BE00CC
:100E80004F04BE0000000600F0FF2F00F1FF270016
:100E9000F9FF3700C70ADE00F107B200F50FB20014
:100EA00008003200E1CF4200020032000170A000D1
:100EB00024000500810F70000100320004080500C5
:100EC00044000500810F700002003A001400050084
:100ED0008502E9000000400081C04800FCFF3B00A3
:100EE0000170A00024000500005E0000BCE20000CC
:100EF000613F0000DD830000C29C00007E200000F6
:100F0000A3FD00001F4100009DC30000217F0000E1
:100F1000FCA20000401E00005F010000E3BD0000D5
:100F20003E60000082DC0000237D00009FC10000C5
:100F3000421C0000FEA00000E1BF00005D030000B5
:100F400080DE00003C620000BEE00000025C0000A9
:100F5000DF810000633D00007C220000C09E000095
:100F60001D430000A1FF000046180000FAA4000085
:100F7000277900009BC5000084DA00003866000075
:100F8000E5BB000059070000DB8500006739000061
:100F9000BAE400000658000019470000A5FB000055
:100FA00078260000C49A0000653B0000D987000045
:100FB000045A0000B8E60000A7F900001B45000035
:100FC000C69800007A240000F8A60000441A000029
:100FD00099C70000257B00003A64000086D8000015
:100FE0005B050000E7B900008CD20000306E000005
:100FF000EDB30000510F00004E100000F2AC0000F5
:101000002F71000093CD0000114F0000ADF30000E0
:10101000702E0000CC920000D38D00006F310000D4
:10102000B2EC00000E500000AFF10000134D0000C4
:10103000CE900000722C00006D330000D18F0000B4
:101040000C520000B0EE0000326C00008ED00000A8
:10105000530D0000EFB10000F0AE00004C12000094
:1010600091CF00002D730000CA9400007628000084
:10107000ABF500001749000008560000B4EA000074
:1010800069370000D58B000057090000EBB5000060
:10109000366800008AD4000095CB00002977000054
:1010A000F4AA000048160000E9B70000550B000044
:1010B00088D60000346A00002B75000097C9000034
:1010C0004A140000F6A80000742A0000C896000028
:1010D000154B0000A9F70000B6E800000A54000014
:1010E000D78900006B3500004C450000540000001B
:1010F0004946000000540000484500004E00000032
:10110000454C000053450000004700004F540000CC
:101110004F000000474F0000535500004200000000
:101120005245000054550000524E0000005200008D
:10113000454D000000500000524900004E54000090
:10114000004900004E5000005554000000460000C9
:101150004F520000005400004F0000004E450000B8
:1011600058540000005200004541000044000000B7
:10117000444100005441000000530000544100006D
:10118000525400005200000053540000415200002D
:1011900054000000535400004F5000005200000063
:1011A000535400004F50000000530000454E000013
:1011B000440000005245000043450000495600002D
:1011C00045000000434C00004B000000444100007B
:1011D0005400000042490000545200004541000004
:1011E000440000004144000043000000415500005D
:1011F00058500000494E00000050000053550000B8
:1012000000500000554C00004C55000050000000FC
:10121000444500004C4100005900000041550000C9
:1012200058000000465200004551000000440000F4
:1012300055540000590000004D4100004352000089
:101240004F000000454E0000440000000052000026
:10125000554E0000004C00004953000054000000AF
:101260004558000049540000004400004542000079
:1012700055470000004E00004557000000000000E8
:101280003E00000008200000080000001B5B00007A
:10129000440000001B5B000000440000001B000035
:1012A0005B430000001B00005B3200004B0D0000A0
:1012B00000430000000000001B5B000032440000FF
:1012C000002000003D2000000056000052450000B4
:1012D00047200000746F00006F2000006C6F00005A
:1012E000772C000020690000732000007468000063
:1012F0006572000065200000612000007368000036
:101300006F720000743F0000002E0000203C0000BF
:10131000002E0000200000000D0A00002800000040
:10132000293E0000004200007573000020500000BC
:1013300069720000617400006520000076310000D1
:101340006100000046690000726D000077610000D6
:101350007265000020760000352E0000313000005C
:1013600020280000723500003539000029200000D7
:101370000020000028320000344600004A360000F9
:1013800034470000413000003032000020000000EF
:1013900041330000004200003400000042350000EC
:1013A0000042000038000000554E00004B000000D5
:1013B0002900000049090000004F0000090000005A
:1013C00048090000004C000009000000456E0000C4
:1013D0007465000072200000726100007720000038
:1013E000766100006C75000065200000666F0000EB
:1013F00072200000425200004700000030620000EE
:1014000000300000303000002C00000030300000C0
:101410000030000031320000333400003536000067
:1014200037380000394100004243000044450000C5
:101430004630000078000000436F0000756C00002B
:10144000646E000027740000206B000065650000DA
:101450007020000075700000000000005350000074
:1014600049310000000000000029000000200000B9
:1014700057000000205200000049000032430000E5
:10148000310000003A200000000000002E000000A3
:1014900031570000303100000000000031410000F1
:1014A0004C53000000420000507600003300000062
:1014B0000808000008080000080000000000000004
:1014C000204800007A0000000000000000410000F9
:1014D000525400003100000042420000494F000019
:1014E00031000000524100005731000000000000B0
:1014F0004F430000443100000000000000000000E5
:1015000000000000290000000000000000000000B2
:101510002800FA000000EB00600F98000000EB00CC
:10152000E06788000000EB00D0678800D06780008B
:10153000200798000000EB00100798000000EB0067
:10154000000F78000000EB00A04088000000EB00D6
:10155000500798000000EB00F06788000000EB00E7
:10156000400798000000EB00000F980014003700BF
:101570000000EB00600798000B0037000E08900099
:10158000EE0090004500DD008100400000D020000A
:10159000808040000040EB00804878006E009000A2
:1015A0000000E800600798006E009000FF0F5000F8
:1015B000F2FF34000E0890000000E800000F9800D1
:1015C0000E089000E40F5000E9FF34000000EB002B
:1015D000006D8800A1408000E00220000088B90072
:1015E0006102200080804000E093200000804000E5
:1015F0004C74020000000000D14080000020200058
:10160000008060000000E000040032007100200053
:10161000C0592000489E02000000000000942800ED
:101620004C7402000000000032043700006D80009E
:101630000000E00063003200006D80000000E9005F
:10164000006D88000000EB00600798001E00370066
:10165000D2678000006D8000EE0090004500DD0044
:101660008100400000D020000080400090407800C1
:10167000A0BF20000000410001487800006D8000FC
:10168000EE0090004500DD008100400000D0200009
:101690000080400010407800A878020000000000A0
:1016A000D06780000000E800D06788006E009000DE
:1016B0000000E80060079800D1678000F00F20006C
:1016C00000806000D0678800006D8000EE00900010
:1016D0004500DD008100400000D020000080400077
:1016E000104078000004E000D9FF3A000000EB0051
:1016F000006D880033003700C0B52000104078002E
:10170000644060000004E0002E003200A140800030
:10171000E00220000088B900FA004000E0932000B9
:101720000080400010007800000001000000E00090
:1017300024003200A1408000E00220000088B900AF
:101740006102200080804000E09320000080400083
:101750004C74020000000000009428004C74020049
:1017600000000000E1678000D0678000808F50009B
:1017700014003200E0678000600798000D00370019
:10178000EE009000A0BF20000080400010407800D4
:10179000A878020000000000EE009000F00F20008A
:1017A00000806000600798006E0090000000E80074
:1017B00060079800EE009000D0678000808F500096
:1017C000EFFF3A008A780200000000000004E00009
:1017D000C9FF320022C2BF00624060000004E00086
:1017E0000500320010118000D1FF2F0001006000C1
:1017F00010118800BF033700967802000000000037
:10180000604F98006E4890000080FB006101B900B5
:101810000217980013179800F0072000010020001D
:101820000E1190009E119000800F5100818F590081
:101830003C033E000E1090009E10900000600100DE
:101840002D033700E20237003E0137003503370031
:10185000D8003700F9023700530137003103370051
:10186000770037002F0337000F0337002D033700B1
:101870002C0337000C033700FE0137002903370023
:101880005A013700270337002603370025033700A6
:1018900024033700230337002203370021033700D6
:1018A000200337001F0337001E03370002013700F3
:1018B0001C0337001B0337001A03370019033700D6
:1018C00018033700170337001603370015033700D6
:1018D00014033700130337001203370011033700D6
:1018E000100337000F0337000E0337000D033700D6
:1018F0000C0337000B0337000A03370009033700D6
:1019000008033700070337000603370005033700D5
:1019100004033700030337000203370001033700D5
:1019200000033700FF023700FE023700FD023700D8
:10193000FC023700FB023700FA023700F9023700D9
:10194000F8023700F7023700F6023700F5023700D9
:10195000F4023700F3023700F2023700F1023700D9
:10196000F0023700EF023700EE023700ED023700D9
:10197000EC023700EB023700EA023700E9023700D9
:10198000E8023700E7023700E6023700E5023700D9
:10199000E4023700E3023700E2023700E1023700D9
:1019A000E0023700DF023700DE023700DD023700D9
:1019B000DC023700DB023700DA023700D9023700D9
:1019C000D8023700D7023700D6023700D5023700D9
:1019D000D4023700D3023700D2023700D1023700D9
:1019E000D0023700CF023700CE023700CD023700D9
:1019F000CC023700CB023700CA023700C9023700D9
:101A0000C8023700C7023700C6023700C5023700D8
:101A1000C4023700C3023700C2023700C1023700D8
:101A2000C0023700BF023700BE023700BD023700D8
:101A3000BC023700BB023700BA0237005D00370036
:101A4000E16780002E009000810F500055003200A9
:101A5000D16780002E009000810F500010003A00E6
:101A6000D06780008000E900F00F20000080600057
:101A7000D0678800D1678000A0BF20008080400030
:101A80000040EB0080487800D16780002107980073
:101A9000209428004C740200000000001503370059
:101AA0000000EB00000F98002E0090008000E9007D
:101AB000F00F20000080600020079800609428004C
:101AC0004C740200000000002E0190006207980094
:101AD000210037006E0190006E0090008000E80049
:101AE000A0BF20000080400090407800A0BF2000F0
:101AF0000000410001487800EE009000A0BF2000E7
:101B000000804000104078000004E0000700320030
:101B1000EE009000A0BF2000008040001040780040
:101B2000A8780200000000000300370000C2B300E4
:101B3000A8780200000000000E0890000000E800F5
:101B4000000F98006E0090008000E800F00F200069
:101B50000080600060079800EE009000D067800071
:101B6000808F5000DBFF3A00D06780008000E900E2
:101B7000F00F200000806000D0678800A09428004B
:101B80004C740200000000000E089000E476020091
:101B900000000000D09428004C74020000000000F7
:101BA000D402370070C0B300A87802000000000023
:101BB000D0023700D16780002E009000810F5000C6
:101BC000390032000000EB00000F9800AE019000D9
:101BD00063079800210037006E0190006E009000AE
:101BE0008000E800A0BF2000008040009040780006
:101BF000A0BF20000000410001487800EE009000E6
:101C0000A0BF200000804000104078000004E000E9
:101C100007003200EE009000A0BF200000804000CE
:101C200010407800A8780200000000000300370090
:101C300000C2B300A8780200000000000E08900067
:101C40000000E800000F98006E0090008000E8009F
:101C5000F00F20000080600060079800EE00900008
:101C6000D0678000808F5000DBFF3A00D067800093
:101C70008000E900F00F200000806000D06788003D
:101C8000A09428004C740200000000000E08900090
:101C9000E476020000000000D09428004C7402009A
:101CA000000000009302370070C0B300A878020063
:101CB000000000008F02370096780200000000004C
:101CC000604F9800EE489000B0C5B30080CF500040
:101CD00088023A009678020000000000604F9800E9
:101CE0006E4890000080FB00700F980020042000D8
:101CF000FE089000808F5000DE003200200420009B
:101D00007E099000800F510005003C001004200067
:101D1000FE099000808F51003400320075023700B8
:101D200030042000FE089000808F50001E0032001A
:101D3000400420007E099000800F51000100320015
:101D40006C0237004E009000E40F50000500340094
:101D5000A88A0200000000000000EB004007980085
:101D600064023700E16780002E009000810F500070
:101D7000090032002E0090008000E900F00F2000E2
:101D80000080600020079800609428004C740200D6
:101D9000000000005702370070C0B300A8780200AE
:101DA0000000000053023700D16780002E00900031
:101DB000810F5000090032002E0090008000E800E2
:101DC000F00F20000080600020079800F0942800A9
:101DD0004C740200000000004602370070C0B300DF
:101DE000A878020000000000420237000000EB006B
:101DF000000F7800E06780000000E90080007800B4
:101E0000F00F200000806000600798008D00370010
:101E1000EE009000A0BF200000804000104078003D
:101E20000004E00082003A006E0090008000E900AB
:101E3000F00F200080806000A0BF200000804000E4
:101E4000104078000004E000790032001E0FE80026
:101E50001E0090009E0F1000750036001E009000BE
:101E60000000E80010079800E1678000D06780005C
:101E7000808F5000140032000A003700D1678000C4
:101E8000A0BF2000808040000040EB008048780028
:101E9000D06780008000E900F00F20000080600023
:101EA000D0678800D1678000E0678000808F500095
:101EB000F2FF3A00D1678000A0BF20008080400080
:101EC0000040EB00804878006E0090008000E90040
:101ED000F00F200000806000000F98001100370014
:101EE0008E089000A0BF20000080400010407800C5
:101EF0000004E00006003A000E0890008000E800B0
:101F0000F00F2000008060005007980009003700A3
:101F10000E0890008000E900F00F200000806000B3
:101F2000000F98008E089000D0678000808F5000CE
:101F3000EBFF3A00309528004C74020000000000CE
:101F4000A1408000E00220000088B900610220006A
:101F500080804000E0932000008040004C7402002C
:101F600000000000D14080000020200000806000C0
:101F70000000E0000400320071002000C059200081
:101F8000489E020000000000009428004C740200EB
:101F900000000000DE019000030F980018003700D9
:101FA0008E089000A0BF2000008040001040780004
:101FB000A878020000000000D26780008E08900020
:101FC000A0BF20000080400090407800A0BF20000B
:101FD0000000410001487800D06780008000E800E0
:101FE000F00F200000806000D06788000E0890008D
:101FF0008000E800F00F200000806000000F9800D3
:102000008E0890006E009000808F5000E4FF3A0030
:10201000D1678000A0BF2000808040000040EB001E
:1020200080487800D06780002007980009003700BA
:102030006E0090008000E900F00F2000008060003A
:1020400060079800EE009000D0678000808F5000FD
:102050006FFF3A00EE009000D0678000808F500044
:10206000A4013A0070C0B300A8780200000000008C
:10207000A00137000000EB00000F7800E06780004F
:102080000000E90080007800F00F20000080600070
:10209000600798008E003700EE009000A0BF20007F
:1020A00000804000104078000004E00083003A0007
:1020B0006E0090008000E900F00F2000808060003A
:1020C000A0BF200000804000104078000004E00025
:1020D0007A0032001E0FE8001E0090000000E900A8
:1020E0009E0F500075003A001E0090000000E900AD
:1020F00010079800E1678000D0678000808F500053
:10210000140032000A003700D1678000A0BF200011
:10211000808040000040EB0080487800D06780005D
:102120008000E900F00F200000806000D067880088
:10213000D1678000E0678000808F5000F2FF3A0096
:10214000D1678000A0BF2000808040000040EB00ED
:10215000804878006E0090008000E900F00F2000B9
:1021600000806000000F9800110037008E0890007A
:10217000A0BF200000804000104078000004E00074
:1021800006003A000E0890008000E800F00F2000E2
:102190000080600050079800090037000E0890008A
:1021A0008000E900F00F200000806000000F980020
:1021B0008E089000D0678000808F5000EBFF3A00BF
:1021C000309528004C74020000000000A1408000FF
:1021D000E00220000088B9006102200080804000F9
:1021E000E0932000008040004C74020000000000DA
:1021F000D140800000202000008060000000E0004E
:102200000400320071002000C0592000489E0200E6
:1022100000000000009428004C7402000000000040
:10222000DE009000010F9800180037008E08900023
:10223000A0BF20000080400010407800A878020075
:1022400000000000D26780008E089000A0BF200030
:102250000080400090407800A0BF200000004100B6
:1022600001487800D06780008000E800F00F20006F
:1022700000806000D06788000E0890008000E800B1
:10228000F00F200000806000000F98008E08900082
:102290006E009000808F5000E4FF3A00D16780000C
:1022A000A0BF2000808040000040EB008048780004
:1022B000D267800022079800090037006E00900066
:1022C0008000E900F00F20000080600060079800A7
:1022D000EE009000D0678000808F50006EFF3A00C3
:1022E000EE009000D0678000808F500001013A001E
:1022F0001E009000E10F500031003A003095280098
:102300004C74020000000000A1408000E0022000A8
:102310000088B9006102200080804000E093200026
:10232000008040004C74020000000000D14080009A
:1023300000202000008060000000E0000400320067
:1023400071002000C0592000489E020000000000DB
:10235000009428004C740200000000000A003700BE
:10236000D1678000A0BF2000808040000040EB00CB
:1023700080487800D06780008000E900F00F2000DE
:1023800000806000D0678800D1678000E06780002F
:10239000808F5000F2FF3A00D1678000A0BF20007C
:1023A000808040000040EB0080487800D3678000C8
:1023B000230798000000EB0010079800CD003700BD
:1023C00070C0B300A878020000000000C900370008
:1023D000E16780002E009000810F50001300320052
:1023E000E16780002E00900001005000800078001E
:1023F000F00F200000806000000F9800A0942800DB
:102400004C740200000000000E089000E476020008
:1024100000000000D09428004C740200000000006E
:10242000E067800020079800B200370070C0B3005A
:10243000A878020000000000AE003700D1678000DD
:102440002E009000810F500013003200D1678000F1
:102450002E0090000080500080007800F00F2000D7
:1024600000806000000F9800A09428004C740200C7
:10247000000000000E089000E4760200000000005A
:10248000909528004C74020000000000D167800085
:10249000210798009700370070C0B300A8780200A9
:1024A000000000009300370010002000600F98002B
:1024B0000000EB0010079800D1678000A0BF20004B
:1024C000808040000040EB0080487800D0678000AA
:1024D0008000E800F00F200000806000D0678800D6
:1024E000D267800022079800B09528007874020017
:1024F000000000007F0037004E0090000000E80060
:10250000400798004E009000F40F500079003A0008
:10251000087F0200000000000000EB004007980068
:1025200074003700D06780008000E800F00F2000C2
:1025300080806000E0678000808F50006A00320079
:102540006E489000FF4F500067003600EE48900044
:10255000E0C7B30080CF500063003E00D167800029
:102560002E009000808F500015003A006E489000B9
:10257000A878020000000000D16780006E4990003A
:10258000A0BF20000080400002487800D067800093
:102590008000E800F00F200000806000D067880015
:1025A000D1678000A0BF2000808040000040EB0089
:1025B00080487800D3678000230798004D003700DB
:1025C000D16780002E0090000080500080007800CD
:1025D000F00F200000806000000F9800A0942800F9
:1025E0004C740200000000000E089000E476020027
:1025F00000000000909528004C74020000000000CC
:10260000D0678000600798001D0037006E009000C2
:102610000001E800EE009000A0BF20000080400014
:1026200090407800A0BF20000000410001487800E1
:10263000EE009000A0BF2000008040001040780015
:102640000004E00009003200EE009000A0BF20006E
:102650000080400010407800A878020000000000D0
:10266000C09528004C740200000000006E0090002D
:102670008000E900F00F20000080600060079800F3
:102680006E0190002E0090008000E900F00F200005
:1026900000806000800F5100DCFF3A006E4890001F
:1026A000A878020000000000AE0090006E49900083
:1026B000A0BF200000804000024878002E0090005B
:1026C0008000E800F00F20000080600020079800E4
:1026D000D06780008000E800F00F200000806000DC
:1026E000D06788000300370070C0B300A8780200EC
:1026F000000000006E0890000000E000CBFB3200FC
:10270000D0678000400F9800E0678000300F98008D
:102710000000EB00600F98000000EB00500F9800E5
:102720000000EB00F0678800D1408000002020000E
:10273000008060000000E000D00432000A36020091
:102740000000000051002000305A2000D29E0200FC
:102750000000000010002000500F9800C704370050
:10276000E1678000A0BF200000804000104078009A
:10277000604F98006E4890000080FB006101B90036
:102780002217980033179800D0072000010020007E
:102790002E119000BE119000800F5100818F5900C2
:1027A0008A043E002E109000BE10900000600100D0
:1027B0008804370085043700840437008304370019
:1027C0008204370081043700800437007F0437001B
:1027D0007E0437007D0437007E0437007B04370019
:1027E0007A0437007B043700780437007704370019
:1027F000760437007504370074043700730437001B
:102800007204370071043700700437006F0437001A
:102810006E0437006D0437006C0437006B0437001A
:102820006A0437006904370068043700670437001A
:10283000680437004504370085023700E40037009C
:10284000ED0037009C0137008A0137005F04370034
:102850005E0237005D0437005C0437005D0437001A
:102860005C043700F10337000A043700D503370052
:10287000FE023700FD023700FC023700FB02370082
:10288000FA023700F9023700F8023700F702370082
:10289000F6023700F50237004C0437004B043700CE
:1028A000A50137008F003700480437003E0037008D
:1028B000FF003700F10037004404370064003700A0
:1028C0006901370041043700400437003F043700F6
:1028D0003E0437003D0437003C0437003B0437001A
:1028E00066003700390437003804370037043700F2
:1028F00036043700350437003404370083013700CD
:10290000320437003104370030043700FE0037004E
:102910002E0437002D0437002C043700AF02370097
:10292000B5033700BF023700E9033700CC03370097
:1029300026043700C400370026003700390037006E
:102940003B01370021043700280037002A003700F8
:102950001E043700170037001C0437001B04370023
:102960005300370019003700180437001B003700E8
:102970001604370015043700380337005F013700AD
:102980001204370011043700160037001401370015
:102990000E0437000D0437000C043700980237008E
:1029A0006B003700A8023700E89E0200000000001C
:1029B0000804370077070700A04080000000E0000F
:1029C00004043200D5070700020437002C06070074
:1029D00000043700F9080700FE033700D30807009A
:1029E000FC03370047080700FA033700607C020049
:1029F00000000000F7033700A04080000000E00066
:102A000005003A00D1012000305D2000D29E020076
:102A100000000000EF033700C87A02000000000049
:102A2000EC033700C0B52000104078000000A10082
:102A30000010A100C1B5200080487800610120008D
:102A4000805A2000D29E020000000000E1033700FF
:102A5000C0B52000104078000000A0000010A100C8
:102A6000C1B520008048780051012000E05B2000C3
:102A7000D29E020000000000D6033700C0B520003F
:102A8000104078000030A000C1B5200080487800D8
:102A9000C1012000B07E2000489E0200000000001E
:102AA000B09528007874020000000000C9033700C8
:102AB000C0B52000104078000030A100C1B5200052
:102AC00080487800B1012000007D2000489E02006F
:102AD00000000000B095280078740200000000009B
:102AE000BC033700E06780008000E800F00F2000A2
:102AF00000806000E0678800D1050700E903070057
:102B0000600798006E009000467702000000000009
:102B1000109628004C740200000000006E00900027
:102B2000E476020000000000109628004C740200B9
:102B3000000000006E009000AC7402000000000075
:102B4000B09528007874020000000000A10337004F
:102B5000E06780008000E800F00F20000080600047
:102B6000E0678800B6050700CE03070060079800FD
:102B70006E0090000080FB000C9C02000000000032
:102B8000600798006E009000467702000000000089
:102B9000109628004C740200000000006E009000A7
:102BA000E476020000000000109628004C74020039
:102BB000000000006E009000AC74020000000000F5
:102BC000B0952800787402000000000081033700EF
:102BD0005100200030632000D29E0200000000005F
:102BE00023C2BF00614060000004E000FCFF32002F
:102BF0000000FE0077033700789F0200000000000D
:102C00000000E00073033200A10020008063200078
:102C1000D29E02000000000040062000AA9B020095
:102C200000000000FC9902000000000023C2BF0069
:102C3000614060000004E000FCFF320081BF2A0018
:102C400001400100630337003B0507000000E80076
:102C5000000F9800020037009E7D02000000000077
:102C60000E0890000000E900000F98000E08900088
:102C70000000E000F8FF3A00560337002E05070079
:102C80000000E800000F9800020037007C7D020081
:102C9000000000000E0890000000E900000F9800FE
:102CA0000E0890000000E000F8FF3A0049033700EA
:102CB000210507000000E800000F98000B00370016
:102CC0006101200020642000489E020000000000F6
:102CD000C07D020000000000367402000000000009
:102CE000B095280078740200000000000E089000E3
:102CF0000000E900000F98000E0890000000E000BE
:102D0000EFFF3A0033033700A04080000000E000EE
:102D100005003A00D1012000305D2000D29E020063
:102D2000000000002B033700C082A900C282A80067
:102D3000C8A2A900CAA2A80021E3A8002000200080
:102D4000AA9B020000000000A0C0B3004C9A020041
:102D50000000000080007800001B2000808F5000E1
:102D60000F00360090C0B3004C9A02000000000033
:102D700080007800702B2000808F50000800360003
:102D80001101200080652000489E02000000000024
:102D9000B095280078740200000000000E00370093
:102DA000C082A900C282A900C8A2A900CAA2A90023
:102DB00050962800787402000000000021012000D5
:102DC00090662000489E020000000000B095280098
:102DD000787402000000000021E3A900FD02370022
:102DE000A04080000000E00005003A00D101200072
:102DF000305D2000D29E020000000000F502370086
:102E0000C082A900C282A900C8A2A900CAA2A900C2
:102E10002101200090662000489E02000000000072
:102E2000B09528007874020000000000E902370025
:102E3000F1002000A0392000489E020000000000A0
:102E4000669A02000000000011002000903A200065
:102E5000489E020000000000B0952800787402002F
:102E600000000000DB023700789A0200000000003A
:102E7000D8023700B0040700000F9800610020005E
:102E800070682000489E0200000000000E089000BC
:102E9000867602000000000021002000D06820009B
:102EA000D29E0200000000000E089000D69B020097
:102EB00000000000C70237009F040700000F9800C1
:102EC0006100200070682000489E020000000000A1
:102ED0000E0890008676020000000000210020000D
:102EE00090EC2000D29E0200000000000E0890002E
:102EF000AA9B020000000000B6023700D04080000C
:102F00000090A000D0408800B2023700A0408000AE
:102F10000000E00005003A00D1012000305D2000F3
:102F2000D29E020000000000AA023700F47D0200D9
:102F300000000000A702370010002000F0678800A2
:102F4000100020006007980010003700E167800043
:102F50006E00900080804000F00F200080806000B4
:102F6000A0BF20000080400090407800E0C3B30084
:102F700080CF500002003A000000EB00F0678800AC
:102F80006E0090000000E80060079800E167800094
:102F90006E00900080804000F00F20008080600074
:102FA000A0BF200000804000104078000004E00036
:102FB000E6FF3A00EE00900020022000808F5000D3
:102FC0000200340010002000F0678800F0678000E5
:102FD0000000E0007F023A00E06780008000E80027
:102FE000F00F200000806000E0678800AD0207005D
:102FF00060079800E1678000F00F2000808060008B
:10300000A0BF20000080400090407800D0C3B300F3
:1030100080CF500040003A006E0090000000E000B9
:103020003A0034006E009000E50F500037003C007D
:10303000E06780008000E800F00F20000080600062
:10304000E06788006E0090000000E90060079800CB
:103050000000EB00000F98000B0037006E0090009E
:103060008E0890004500DD008100400000D0200067
:10307000808040000040EB00804878000E089000FF
:103080000000E800000F98000E089000FF0F5000AD
:10309000F2FF34000000EB00000F9800130037002F
:1030A000EE0190000E0A9000E1678000A0BF2000B2
:1030B00000804000104178004518DD008400400089
:1030C00000D0200000804000024878000E089000E8
:1030D0000000E800000F9800E06780008000E80032
:1030E000F00F200000806000E0678800E16780004A
:1030F000A0BF20000080400090407800E0C3B300F3
:1031000080CF5000E6FF3A00320237001000200066
:10311000F06788002F0237006E0090000000E0008A
:103120001B003A000000EB00000F9800140037006D
:103130000E0890000040E800E47602000000000065
:10314000509828004C740200000000000E08900007
:103150004500DD008000780000D0200000804000A5
:103160004C740200000000000094280078740200F3
:10317000000000000E0890000000E800000F98001A
:103180000E089000E40F5000E9FF340011023700F0
:103190006E0090000000E000090034006E00900016
:1031A000E50F500006003C00B0952800787402003E
:1031B00000000000EE009000016D8800050237005D
:1031C00010002000F067880002023700E0678000EE
:1031D0008000E800F00F200000806000E0678800B9
:1031E00030020700200F980015040700E1678000F7
:1031F000F00F200080806000A0BF20000080400011
:103200009040780090C2B30080CF50000D003A008B
:10321000A1408000E00220000088B900FC004000CE
:10322000E093200000804000900078002E0890007D
:1032300001000100B0952800787402000000000031
:10324000E401370010002000F0678800E10137003A
:1032500010002000F0678800100020006007980030
:1032600010003700E16780006E0090008080400011
:10327000F00F200080806000A0BF20000080400090
:103280009040780020C2B30080CF500002003A0086
:103290000000EB00F06788006E0090000000E8007E
:1032A00060079800E16780006E0090008080400019
:1032B000F00F200080806000A0BF20000080400050
:1032C000104078000004E000E6FF3A00F06780005C
:1032D0000000E000BF013A0071002000F06820000B
:1032E000489E02000000000020C2B300A87802003F
:1032F0000000000022003700E1678000F00F20008E
:1033000000806000E0678800E1678000A0BF2000C7
:103310000080400010407800A87802000000000003
:10332000E1678000A0BF20000080400010407800CE
:103330000000FB00200F9800C0B52000104078006E
:10334000684060000004E000040032002E08900095
:103350000C9C020000000000200F9800A14080009B
:10336000E00220000088B900E8004000E09320005F
:1033700000804000900078002E08900001000100BD
:10338000E06780000000E800E0678800E1678000F7
:10339000F00F200080806000A0BF2000008040006F
:1033A0009040780020C2B30080CF5000D2FF3A0096
:1033B000E0678000F10F200001006000E0678800F6
:1033C00020C2B300A878020000000000B0952800D9
:1033D00078740200000000007E013700A1408000E8
:1033E000E00220000088B90080007800E09320000F
:1033F00000804000100078000000010075013700D7
:10340000A1408000E00220000088B9008080E80030
:10341000E0932000008040001000780000000100D0
:103420006C013700A1408000E00220000088B90054
:10343000E4004000E093200000804000100078008D
:103440000000010063013700A1408000E00220007D
:103450000088B900E6004000E093200000804000B2
:1034600010007800000001005A01370071002000B0
:10347000F0682000489E020000000000890107005B
:10348000200F9800E06780000000E900E0678800F6
:10349000E1678000F00F200000806000E067880096
:1034A000250307000000E800000F9800450307000F
:1034B000300798003E0090000000E0005D00320000
:1034C0003E00900080407800B0B4200001487800B1
:1034D0003E009000E80F500006003400C0B5200008
:1034E000104078000050A000C1B52000804878004E
:1034F00050003700C0B52000104078000050A100F7
:10350000C1B52000804878004A0037002E0890009E
:10351000049B020000000000C0B5200010407800AD
:103520000042B2000004E00004003A00B0B4200001
:1035300010407800E84F500009003A00C0B5200064
:10354000104078000042B2000004E0000B0032009E
:10355000B0B4200010407800F04F50000700320057
:10356000B0C3B300A878020000000000B0B420008F
:1035700010407800E476020000000000C0B5200092
:1035800010407800684060000004E0000400320051
:103590002E0890000C9C020000000000200F9800F4
:1035A000A1408000E00220000088B900E80040004F
:1035B000E093200000804000900078002E089000EA
:1035C00001000100100F980000C2B300A8780200AB
:1035D00000000000C0B52000104078000044B20098
:1035E0000004E00013003200610020006069200048
:1035F000489E020000000000C0B520001040780086
:10360000684060000004E000040032001E089000E2
:103610000C9C020000000000100F98001E08900093
:10362000049B02000000000000C2B300A878020062
:10363000000000000E0890000000E900000F980054
:103640000E0890000000E000B0FF3A00B09528009E
:103650007874020000000000DE00370061002000E6
:1036600060692000489E020000000000B2020700CE
:103670000000E800000F9800D20207003007980011
:103680003E0090000000E000440032003E00900048
:1036900080407800B0B42000014878003E009000DF
:1036A000E80F500006003400C0B52000104078003C
:1036B0000050A000C1B520008048780037003700D6
:1036C000C0B52000104078000050A100C1B5200016
:1036D0008048780031003700A1408000E0022000DF
:1036E0000088B900EA004000E0932000008040001C
:1036F0001000780000000100100F9800C0B52000F5
:1037000010407800684060000004E00004003200CF
:103710001E0890000C9C020000000000100F980092
:103720001E089000049B020000000000C0B52000AD
:10373000104078000042B2000004E00004003A00AB
:10374000B0B4200010407800E84F500009003A0063
:10375000C0B52000104078000042B2000004E00034
:103760000B003200B0B4200010407800F04F500041
:1037700007003200B0C3B300A878020000000000C8
:10378000B0B4200010407800E47602000000000091
:1037900000C2B300A8780200000000000E089000EC
:1037A0000000E900000F98000E0890000000E00003
:1037B000C9FF3A00B09528007874020000000000AC
:1037C0008400370081002000C0692000D29E0200E2
:1037D00000000000A1408000E00220000088B90045
:1037E000EC004000E09320000080400010007800D2
:1037F000000001007700370081002000406A2000AF
:10380000D29E020000000000A1408000E0022000E3
:103810000088B900EE004000E093200000804000E6
:1038200010007800000001006A003700E10020006D
:10383000C06A2000D29E020000000000A14080006B
:10384000E00220000088B900F0004000E093200072
:103850000080400010007800000001005D0037008B
:10386000E1002000A06B2000D29E020000000000BA
:10387000A1408000E00220000088B900F200400072
:10388000E09320000080400010007800000001005C
:1038900050003700C1002000B0672000489E0200A1
:1038A00000000000A1408000E00220000088B90074
:1038B000F4004000E09320000080400010007800F9
:1038C00000000100367402000000000041003700D3
:1038D00019020700000F9800D1002000806D200021
:1038E000489E0200000000000E089000049B0200A9
:1038F000000000000E0890000000E800000F980093
:1039000008003700A1408000E00220000088B900D4
:10391000F6004000E0932000008040001000780096
:10392000000001000E0890000000E900000F980060
:103930000E0890000000E000F2FF3A00B095280069
:10394000787402000000000022003700FA0107002E
:103950000000E800000F9800A1002000506E200039
:10396000489E0200000000000D003700A1408000CA
:10397000E00220000088B900F8004000E093200039
:103980000080400010007800000001003674020042
:103990000000000000C2B300A87802000000000090
:1039A0000E0890000000E900000F98000E0890003B
:1039B0000000E000EDFF3A0001012000806C2000D3
:1039C000D29E02000000000002003700100020001C
:1039D000F0678800E06780008000E800F00F2000BA
:1039E00000806000E0678800F06780000000E00071
:1039F0001C00320051012000F06E2000489E0200A1
:103A000000000000BE089000E0678000808F50003A
:103A100007003100E0678000804078003E08900099
:103A200000C05000E47602000000000006003700ED
:103A3000E0678000804078003E08900000C05000A1
:103A4000E4760200000000000000EB00F067880050
:103A500010002000500F9800B095280078740200E4
:103A600000000000E1678000D0678000808F500078
:103A700002003A0010002000500F98005E089000ED
:103A80000000E00036FB32004E089000E06788003E
:103A90004E089000D06788000000EB00600F98008F
:103AA000CCF637000600FA000000EB001007980083
:103AB0000000EB00000F7800E16780001E0090001E
:103AC00080804000F00F200080806000A0BF2000B8
:103AD000008040009040780000C3B30080CF5000C9
:103AE00043003400E16780001E00900080804000A9
:103AF000F00F200080806000A0BF20000080400008
:103B00009040780090C3B30080CF500038003C0054
:103B1000E16780001E00900080804000F00F2000D0
:103B200080806000A0BF200000804000104078002E
:103B30008000FB0000FD2F00008F40001E00900061
:103B40000000E80010079800120037001E007800FF
:103B50006A00B900000F7800E16780001E00900045
:103B600080804000F00F200080806000A0BF200017
:103B700000804000104078000000FB009E004000E4
:103B800000FD2F00008F40001E0090000000E800A4
:103B900010079800E16780001E00900080804000C0
:103BA000F00F200080806000A0BF20000080400057
:103BB00090407800F0C2B30080CF50005101340033
:103BC000E16780001E00900080804000F00F200020
:103BD00080806000A0BF20000080400090407800FE
:103BE00090C3B30080CF5000D8FF340045013700A8
:103BF000E16780001E00900080804000F00F2000F0
:103C000080806000A0BF20000080400090407800CD
:103C100000C3B30080CF500035013A001E00900071
:103C20000000E80010079800E16780001E00900087
:103C300080804000F00F200080806000A0BF200046
:103C4000008040009040780020C6B30080CF500034
:103C50000B003200E16780001E0090008080400071
:103C6000F00F200080806000A0BF20000080400096
:103C70009040780020C4B30080CF50002D003A005F
:103C80001E0090000000E8001007980012003700A6
:103C90001E00780000004000000F7800E1678000FF
:103CA0001E00900080804000F00F200080806000A7
:103CB000A0BF200000804000104078000000FB0002
:103CC0009E00400000FD2F00008F40001E0090006D
:103CD0000000E80010079800E16780001E009000D7
:103CE00080804000F00F200080806000A0BF200096
:103CF000008040009040780010C3B30080CF500097
:103D0000E3FF3200E16780001E00900080804000E9
:103D1000F00F200080806000A0BF200000804000E5
:103D20009040780000C3B30080CF5000D8FF32002D
:103D3000F4003700E16780001E00900080804000A2
:103D4000F00F200080806000A0BF200000804000B5
:103D50009040780080C7B30080CF50000B00320045
:103D6000E16780001E00900080804000F00F20007E
:103D700080806000A0BF200000804000904078005C
:103D800080C5B30080CF50008E003A001E00900026
:103D90000000E80010079800470037001E00780078
:103DA0004400DD00000F7800E16780001E009000F5
:103DB00080804000F00F200080806000A0BF2000C5
:103DC0000080400090407800F0C2B30080CF5000E7
:103DD00018003400E16780001E00900080804000E1
:103DE000F00F200080806000A0BF20000080400015
:103DF0009040780090C3B30080CF50000D003C008D
:103E0000E16780001E00900080804000F00F2000DD
:103E100080806000A0BF200000804000104078003B
:103E20000000FB009E00400000FD2F00008F4000BE
:103E30001E003700E16780001E0090008080400077
:103E4000F00F200000816000E16780001E009000FC
:103E500080804000F00F200080806000A0BF200024
:103E6000008040009040780000C2B30080C0700025
:103E7000A0BF20000000410001487800E1678000F9
:103E80001E00900080804000F00F200080806000C5
:103E9000A0BF200000804000104078000000FB0020
:103EA0009E00400090FA2F00008F40001E009000FE
:103EB0000000E80010079800E16780001E009000F5
:103EC00080804000F00F200080806000A0BF2000B4
:103ED0000080400090407800F0C2B30080CF5000D6
:103EE0000B003400E16780001E00900080804000DD
:103EF000F00F200080806000A0BF20000080400004
:103F00009040780090C3B30080CF5000A3FF3400EE
:103F1000E16780001E00900080804000F00F2000CC
:103F200080806000A0BF20000080400090407800AA
:103F300000C4B30080CF50000B003400E167800064
:103F40001E00900080804000F00F20008080600004
:103F5000A0BF2000008040009040780060C4B30003
:103F600080CF50008DFF3400E16780001E0090007C
:103F700080804000F00F200080806000A0BF200003
:103F8000008040009040780000C6B30080CF500011
:103F90005C003400E16780001E00900080804000DB
:103FA000F00F200080806000A0BF20000080400053
:103FB0009040780060C6B30080CF500077FF340097
:103FC00050003700E16780001E00900080804000B4
:103FD000F00F200080806000A0BF20000080400023
:103FE00090407800F0C2B30080CF5000450034000C
:103FF000E16780001E00900080804000F00F2000EC
:1040000080806000A0BF20000080400090407800C9
:1040100090C3B30080CF50003A003C00E1678000BD
:104020001E00900080804000F00F20008080600023
:10403000A0BF200000804000104078008000FB00FE
:1040400000FD2F00008F4000120037001E00780096
:104050006A00B900000F7800E16780001E00900040
:1040600080804000F00F200080806000A0BF200012
:1040700000804000104078000000FB009E004000DF
:1040800000FD2F00008F40001E0090000000E8009F
:1040900010079800E16780001E00900080804000BB
:1040A000F00F200080806000A0BF20000080400052
:1040B00090407800F0C2B30080CF5000110034006F
:1040C000E16780001E00900080804000F00F20001B
:1040D00080806000A0BF20000080400090407800F9
:1040E00090C3B30080CF5000D8FF340005003700E4
:1040F00010002000F06788000000EB002007980007
:104100000A003700E16780001E0090000080400038
:10411000E0678800E1678000F00F20000080600009
:10412000E06788001E007800200798002E009000AD
:104130000080FA00000006000400FA00E06780003A
:104140008000E800F00F200080806000A0BF200009
:104150000080400090407800A0C3B30080CF5000A2
:1041600013003A00E06780000080E800E067880004
:10417000E1678000F00F200000806000E0678800A9
:1041800048FE0700000F7800E06780000000E900AB
:10419000E0678800E1678000F00F20000080600089
:1041A000E06788001E0078001007980002003700C2
:1041B00010002000100798001E0090000080FA00F8
:1041C000000006000400FA00E06780008000E800BC
:1041D000F00F200080806000A0BF20000080400021
:1041E00090407800B0C3B30080CF50000F003A0079
:1041F000E06780008080E800F00F20000080600011
:10420000E067880027FE0700000F7800E067800065
:104210008000E900F00F200000806000E067880067
:104220001E00780010079800020037000000EB0025
:10423000100798001E0090000080FA0000000600A1
:104240000000FA0005003700E06780008000E80009
:10425000F00F200000806000E0678800E1678000C8
:10426000A0BF2000008040009040780000C2B30052
:1042700080CF5000F4FF32000080FA0000000600FA
:104280000400FA000000EB00000F7800E0678000F7
:104290008000E800F00F200000806000E0678800E8
:1042A000E7FF0700FFFD0700000F78001E00E00099
:1042B0004D003A000000EB00100798001300370093
:1042C0001E0090000040E800E476020000000000BC
:1042D000909828004C740200000000009E0090009E
:1042E000E00220000088B9006102200080804000C8
:1042F000E09320000080400078740200000000007D
:104300001E0090000000E800100798001E009000BA
:10431000E80F5000EAFF34007101200040702000D7
:10432000D29E0200000000000000EB00F067880051
:104330001300200092002000110020001000200037
:1043400055000700000FE900E0FF2F009E0F10004E
:10435000030032000080EB009E0F100005003A00C1
:10436000E1002000B0712000D29E02000000000099
:1043700042003700A1408000E00220000088B90020
:104380000102200080804000E09320000080400077
:104390001000780000000100FC99020000000000FD
:1043A0001E007800A0408800A1408000E0022000AC
:1043B0000088B900FE004000E0932000008040002B
:1043C00010007800000001001E00E0000100320033
:1043D000CA82A80051002000305A2000D29E02005C
:1043E00000000000250037001E0FE90080002000BB
:1043F0009E0F10001D003C00A1408000E002200044
:104400000088B9000102200080804000E093200075
:10441000008040001000780000000100FC990200BC
:10442000000000001E007800A0408800A14080002D
:10443000E00220000088B900FE004000E093200068
:104440000080400010007800000001001E00E00025
:1044500001003200CA82A80051002000305A20001A
:10446000D29E02000000000004003700510120002D
:1044700090722000D29E020000000000D0678000F1
:104480008000E900F00F200000806000E0678800F5
:104490000080FA00000006001E00FA00100F9800CD
:1044A000210F9800320F9800430F98000000EB0096
:1044B000400798000000EB00200798000000EB0088
:1044C000100798000000EB00000F7800C09828004B
:1044D0004C740200000000001E089000E476020008
:1044E00000000000009928004C7402000000000049
:1044F000670037009678020000000000204F980007
:104500002E4890000000FB00600F98006E0890009D
:10451000ED0F500029003200EE089000ED8F5000A2
:1045200007003C006E099000E80F51000D003200BA
:104530006E089000EA0F500020003200350037006E
:10454000D0022000EE089000808F50001E00320044
:10455000800720006E099000800F51002700320074
:104560002C0037004E0090000000E00007003200F1
:104570004E0090000000E9004007980020942800B9
:104580004C74020000000000410037001E00E000F3
:10459000060032000000EB00000F78002094280095
:1045A0004C740200000000003900370070C0B300F6
:1045B000A87802000000000035003700100020003D
:1045C00020079800320037004E0090000000E00005
:1045D00006003A00D0C2B300A87802000000000034
:1045E00010002000000F78002900370070C0B300D1
:1045F000A878020000000000250037004E08900057
:104600000000E000030032000080EB00500F980033
:104610005D003700AE489000F0C2B30080CF50007C
:1046200018003400AE48900090C3B30080CF500013
:1046300014003C004E009000E30F500006003400D0
:1046400070C0B300A8780200000000004000200005
:10465000400798000E0037002E489000A87802000E
:1046600000000000CE0090006B0047002E49900033
:10467000827078004E0090000000E800400798002B
:104680000300370070C0B300A878020000000000EB
:104690002E0090000000E00096FF3200B095280048
:1046A00078740200000000004E0090000000E0005E
:1046B00003003A001E089000500F980032003700A7
:1046C0000000EB00100798004E0090000000E90089
:1046D00040079800CE009000310798001100370085
:1046E0001E0090006A00B90010079800BE009000FC
:1046F0004E009000808050006B00470061407800C1
:104700008000FB001E0090008080400000FD2F0014
:1047100000804000100798004E0090000000E90063
:10472000400798004E0090000000E000ECFF3D00C4
:104730009E0090002E089000808F50000D003500E4
:104740009E0090003E089000808F500009003C00C1
:104750001E00E000040032001E0090000000EA008D
:10476000500F9800080037001E019000520F98006B
:1047700005003700B1012000E0EA2000D29E0200CF
:104780000000000049FF37005E0890000080FA003A
:10479000000006000400FA00309928007874020036
:1047A00000000000209A28004C7402000000000065
:1047B000D100200070802000489E02000000000010
:1047C000A1BF2A000000EB00027A020000000000F6
:1047D000000F78001E0078004800DE00E47602003A
:1047E00000000000E0C2B300A87802000000000052
:1047F0001E007800E476020000000000B09528005A
:1048000078740200000000006100200000762000A3
:10481000489E020000000000B04080009E77020029
:10482000000000007100200070EA2000489E020095
:1048300000000000C04080009E77020000000000E1
:10484000909B28004C74020000000000C0408000D3
:1048500010079800200423009E009000808F5000D5
:1048600016003200200423009E009000808F50002C
:1048700005003E00300023009E009000808F500015
:104880000A00320019003700300423009E00900017
:10489000808F50000D003200600423009E009000C5
:1048A000808F50000D00320010003700809C2800DF
:1048B0004C740200000000000F003700B09C28007C
:1048C0004C740200000000000B003700E09C280040
:1048D0004C7402000000000007003700109D280003
:1048E0004C7402000000000003003700409D2800C7
:1048F0004C74020000000000809D280078740200C3
:1049000000000000E101200060762000D29E02003D
:10491000000000000080FA00000006000000FA001D
:104920005100200020922000489E0200000000005C
:10493000C1BF2A000000EB00027A02000000000064
:104940009E770200000000006100200070922000AD
:10495000489E020000000000E1BF2A000000EB00BA
:10496000027A0200000000009E77020000000000B2
:10497000B09528007874020000000000C1002000FB
:1049800040782000D29E0200000000005D00070079
:10499000CAC2BF000042B2000004E00005003200BD
:1049A0001101200080652000489E020000000000E8
:1049B000040037002101200090662000489E02007C
:1049C00000000000C0C2B300A87802000000000090
:1049D00000C2B300A878020000000000C0B52000AB
:1049E00010407800704060000004E00005003200D4
:1049F0002102200000792000D29E02000000000069
:104A000004003700E1012000207B2000D29E02003C
:104A100000000000C0B52000104078006840600031
:104A20000004E00005003A00B1012000007D2000F4
:104A3000489E02000000000004003700C101200071
:104A4000B07E2000489E020000000000C0C2B300FB
:104A5000A87802000000000000C2B300A87802009D
:104A600000000000B101200010192100489E020042
:104A700000000000B0B4200010407800E47602008E
:104A800000000000B09528007874020000000000CB
:104A9000C0B520001040780063406000E14F500036
:104AA00005003A0051012000E05B2000D29E020088
:104AB000000000000400370061012000805A20003F
:104AC000D29E020000000000A1408000E002200011
:104AD0000088B9004102200080804000E09320005F
:104AE000008040001000780000000100C10020009C
:104AF00040782000D29E0200000000000080FA00F2
:104B0000000006000000FA00A1002000A00521001E
:104B1000D29E02000000000061042000200B210052
:104B2000D29E020000000000A101200040062100EA
:104B3000489E020000000000A1408000E00220002A
:104B40000088B9002102200080804000E09320000E
:104B5000008040001000780000000100A10020004B
:104B6000E0072100489E02000000000000402000F5
:104B700050000700001020004E0007000020200019
:104B80004C000700000420004A0007000008200035
:104B900048000700B095280078740200000000006B
:104BA00041002000800F2100489E0200000000000C
:104BB00021E3A800A0C0B3004C9A0200000000004E
:104BC000E87702000000000011002000903A200069
:104BD000489E02000000000090C0B300A8780200C8
:104BE0000000000090C0B3004C9A020000000000DA
:104BF000E87702000000000011002000903A200039
:104C0000489E02000000000090C0B300A878020097
:104C100000000000C0C0B3004C9A02000000000079
:104C2000E87702000000000011002000903A200008
:104C3000489E02000000000090C0B300A878020067
:104C400000000000B0C0B3004C9A02000000000059
:104C5000E87702000000000011002000903A2000D8
:104C6000489E02000000000090C0B300A878020037
:104C70000000000021E3A900004020001C00070004
:104C8000001020001A000700002020001800070074
:104C90000004200016000700000820001400070090
:104CA000B095280078740200000000000080FA002F
:104CB000000006000200FA00000F78004016800095
:104CC0001E0060000000E00004003200A09D2800EB
:104CD0004C7402000000000003003700D09D280043
:104CE0004C740200000000000080FA000000060082
:104CF0000200FA00000F7800501680001E006000CD
:104D00000000E00004003200009E28004C74020005
:104D10000000000003003700309E28004C740200A1
:104D2000000000000080FA00000006000200FA0007
:104D3000E06780008000E800F00F20000080600045
:104D4000E06788003EFD070056FB0700000F780073
:104D50001E00E00006003400400020009E0F1000FE
:104D600003003C001E00E900904088000D00370061
:104D70000000EB00F0678800210220004081200045
:104D8000D29E0200000000008001EB0042002000E3
:104D90001100200010002000BFFD07000000E90006
:104DA000904088002101200060832000D29E0200F4
:104DB000000000000080FA00000006000200FA0077
:104DC0000040EB00004F7800E06780008000E800C2
:104DD000F00F200000806000E067880018FD0700E9
:104DE00030FB0700104798001E4090000004E000D0
:104DF000090032001E409000EA4F500006003E00BD
:104E00001E4090000040E9008040780000812000B2
:104E1000014878000F0037000000EB00F0678800C1
:104E2000D108200030872000D29E02000000000040
:104E30008001EB00A2002000110020009000200063
:104E400095FD07000040E9008040780000812000C7
:104E5000014878000081200010407800E94F5000A0
:104E600010003A00F6FC07000EFB0700004F780028
:104E70001E04E0000B003A000000EB00F067880021
:104E8000609E280078740200000000008001EB00A2
:104E9000F2FF27008000EB00200220007EFD0700CB
:104EA000004F78004101200000902000D29E0200B7
:104EB000000000001101200000182100D29E020015
:104EC0000000000023C2BF00614060000004E00059
:104ED000FCFF32000081200010407800E94F5000B4
:104EE00003003A001E407800C6780200000000006F
:104EF000D69A020000000000000037008A78020005
:104F0000000000000004E000FCFF32009678020080
:104F1000000000008040780000C2B30080CF500045
:104F200001003200F5FF37000080FA0000000600A3
:104F30000000FA00D171800020E4200000804000D1
:104F40009040780030C8B30080CF50000E003A0087
:104F5000D07180000000E800D071880003003700A5
:104F6000D07180000000E800D0718800D17180000D
:104F700020E42000008040009040780000CEB30084
:104F800080CF5000F6FF36000080FA0000000600D7
:104F90000A00FA00300798000000EB002007980094
:104FA000AE00900020E42000008040009040780097
:104FB00000CEB30080CF500003003E000080EB0025
:104FC0004007980023003700AE00900020E4200046
:104FD00000804000104078008080FB0000F22F002D
:104FE00000804000100798002E0090008000E8002C
:104FF00020E4200000804000104078000080FB008A
:105000004801DD002E0090008080E80020E42000B0
:1050100000804000104078000080FB00000F41003D
:105020009E0078003E009000808F500003003A0000
:105030002E00900040079800060037009E00900068
:105040002E00900000804000630040002007980080
:10505000D3FF37004E0090000080FA0000000600E9
:105060000600FA00881F78000000EB00000F7800AF
:10507000D171800020E42000008040009040780042
:1050800080C2B30080CF500010003A00D071800081
:105090000000E800D07188001F010700000F7800B1
:1050A000D171800020E42000008040009040780012
:1050B00090C2B30080CF5000AC003A00D0718000A5
:1050C0000000E800D0718800A8003700D17180008E
:1050D00020E42000008040009040780000C4B3002D
:1050E00080CF500016003600D171800020E42000EF
:1050F0000080400090407800A0C5B30080CF5000F1
:105100000F003E00D271800020E42000000041002A
:10511000104078008080FB00F0FB2F0000804000F2
:1051200080004000A0DD20000080400010007800DA
:10513000200798000200E800D07188008D00370039
:10514000D171800020E42000008040009040780071
:1051500000C8B30080CF500076003600D1718000C7
:1051600020E4200000804000104078000080FB0018
:10517000100798000100E800D07188007009200035
:105180009E009000808F5000410032007009200086
:105190009E009000808F50000D003C0040092000D0
:1051A0009E009000808F50001600320060092000A1
:1051B0009E009000808F50002B00320030092000AC
:1051C0009E009000808F5000180032004800370089
:1051D000A00920009E009000808F50003600320011
:1051E000D00920009E009000808F50001A003200ED
:1051F000800920009E009000808F50003500320012
:105200003B003700A1408000E00220000088B90088
:10521000EA004000E0932000008040001000780089
:1052200000000100000F780050003700A14080000E
:10523000E00220000088B900E8004000E093200070
:10524000008040001004780084000700080001007E
:10525000000F780045003700C07D0200000000000C
:10526000000F780041003700A1408000E0022000DC
:105270000088B900F4004000E09320000080400066
:105280001000780000000100000F780037003700A0
:10529000A1408000E00220000088B900F800400032
:1052A000E093200000804000100078000000010022
:1052B000000F78002D003700CAC2BF000080FB003D
:1052C0004500DE00614060000080FB00000F7800B8
:1052D0002600370021E3A800C0C0B3004C9A0200AA
:1052E00000000000000F780021E3A9001F00370034
:1052F0000000EB00000F78001C0037001E00780053
:105300006A00B900000F7800D171800020E420000D
:1053100000804000104078000080FB009E004000AC
:1053200000FD2F00008F4000D07180000000E800D9
:10533000D0718800D171800020E4200000804000FE
:1053400090407800F0C2B30080CF500007003600D4
:10535000D171800020E4200000804000904078005F
:1053600090C3B30080CF5000E4FF36001E007800E9
:10537000200798002E0090004F0478000080FA006B
:10538000000006000600FA0035FF0700000F780055
:1053900000003700D171800020E420000080400030
:1053A00090407800A0C2B30080CF50000A003200C5
:1053B000D171800020E420000080400090407800FF
:1053C000F0C2B30080CF5000030032001E0078000E
:1053D000200798001E003700D171800020E42000D3
:1053E00000804000104078000080FB00100798000B
:1053F0000100E800D0718800A00220009E0090000B
:10540000808F500005003200F00220009E009000C6
:10541000808F500007003200DEFF370010FF0700CA
:10542000800078001E0078000180B900000F78002D
:10543000D8FF37000AFF0700000178001E0078003F
:10544000110009000200D800000F7800D1FF3700DA
:105450002E0090000080FA00000006000600FA000E
:10546000C8FF0700000F780000003700D1718000EE
:1054700020E420000080400090407800D0C2B300BB
:1054800080CF50000A003200D171800020E420005B
:105490000080400090407800B0C2B30080CF500040
:1054A000030032001E007800200798001700370024
:1054B000D171800020E4200000804000104078007E
:1054C0000080FB00100798000100E800D071880000
:1054D000B00220009E009000808F50000800320033
:1054E000D00220009E009000808F5000010032000A
:1054F000DEFF3700A3FF07001E0F1000DBFF3700A1
:10550000A0FF07001E0F4000D8FF37002E009000BC
:105510000080FA00000006000C00FA00D271800042
:1055200020E4200000004100104078008080FB0053
:10553000F0FB2F000080400080004000A0DD200034
:105540000080400090007800210798000200E800E9
:10555000D07188000000EB00000F78000B003700CE
:105560009E017800D271800020E4200000004100FC
:105570001040780080407800660047008171780014
:105580000200E800D07188001E0FE800D171800091
:1055900020E42000008040009040780000C4B30068
:1055A00080CF500007003600D171800020E4200039
:1055B0000080400090407800A0C5B30080CF50002C
:1055C0000E003600D171800020E4200000804000F1
:1055D00090407800F0C2B30080CF5000E0FF36006A
:1055E000D171800020E420000080400090407800CD
:1055F00090C3B30080CF5000D9FF3E0097FF070053
:105600001007980066004700104078000000FB007B
:1056100050079800C0032000DE009000808F5000EB
:1056200032003200C0032000DE009000808F500066
:1056300005003C0010022000DE009000808F50002A
:10564000410032004E003700D0032000DE00900001
:10565000808F500005003200E0032000DE00900043
:10566000808F50000A003200450037000000EB0038
:1056700040079800AE0090001E009000808F500000
:1056800041003A0011002000410798003E00370019
:105690006600470090409000D0C3B30080CF500018
:1056A00009003A000000EB0040079800AE009000AF
:1056B0001E009000808F5000330035001100200044
:1056C00041079800300037000000EB0040079800C9
:1056D000AE0090001E009000808F50002A00340021
:1056E000110020004107980027003700660047009E
:1056F00090409000D0C3B30080CF500009003A0022
:105700000000EB0040079800AE0090001E009000E3
:10571000808F50001C003C001100200041079800C1
:10572000190037000000EB0040079800AE00900021
:105730001E009000808F500013003D0011002000DB
:105740004107980010003700660047009040900025
:10575000D0C3B30080CF500009003A000000EB0036
:1057600040079800AE0090001E009000808F50000F
:1057700005003200110020004107980002003700A8
:105780000000EB00400798004E0090000080FA00F7
:10579000000006001C00FA00881F78000000EB00E3
:1057A000D07188000000EB00300798000000EB008B
:1057B000200798000000EB00100798000000EB00A5
:1057C000E07188000000EB00F07188000000EB0041
:1057D000007288000000EB0050079800D040800065
:1057E0000080A000D04088000000EB004007980037
:1057F000090037004E00900080004000A0DD20002E
:10580000808040000000EB00800878004E0090008F
:105810000000E800400798004E009000F90F50008B
:10582000F4FF3400350437001E0090000000E00053
:1058300021003A00D171800020E420000080400067
:1058400090407800F0CDB30080CF500003003E00C0
:1058500020002000300798002B043700D171800011
:1058600020E4200000804000104078008080FB0091
:1058700000F22F000080400060079800D071800087
:105880008000E80020E42000008040001040780004
:105890000080FB004801DD00D07180008080E800BE
:1058A00020E4200000804000104078000080FB00D1
:1058B00000007100500798000000EB0010079800EE
:1058C000D0718000E300400020E420000080400010
:1058D000104078000080FB006101B90000F82F0043
:1058E000F1FF2F000201400083814800420F980021
:1058F000530F980010022000010020004E09900074
:10590000DE099000800F5100818F5900EF033E00A7
:105910004E089000DE089000006001002100370072
:1059200035003700E9033700E8033700710037001E
:1059300081003700A3003700B7003700BE003700F2
:105940003B01370088013700E0033700EE013700E4
:105950003502370099023700AF0237009F02370047
:10596000CB023700BB023700D8023700D70337001D
:105970007C03370060033700D4033700D3033700BC
:1059800004033700F0023700A3033700AE033700EB
:10599000DE0237001603370036033700B603370040
:1059A000C70337001000200020079800D071800046
:1059B00066004000D0718800D07180008080E900CE
:1059C00020E4200000804000104078008080FB0030
:1059D000F0FB2F0000844000A0FE070000017800CB
:1059E00088004400A0DD200000804000020878000C
:1059F0004FFD0700B7033700100020002007980074
:105A0000D071800064004000D0718800C2FE0700A1
:105A10000000E0001C003200D1718000310F9800BE
:105A200020E420003E0990000000410090407800F2
:105A30008041EB004357980020C8B30080CF50004E
:105A400002003A0010C0B30040579800BE08900012
:105A50000100E800D07188004E5190000204E0007F
:105A60009C0332001000200010079800D0718000C5
:105A700063005000D071880096033700D071800019
:105A80000000E800D0718800D171800020E420007F
:105A9000008040009040780030C8B30080CF5000B4
:105AA00007003200D171800020E420000080400017
:105AB0009040780000CEB30080CF5000EFFF36005A
:105AC000D171800020E420000080400090407800E8
:105AD00030C8B30080CF50007E033A001000200091
:105AE00010079800D07180000080E900D071880014
:105AF000780337001000200020079800D071800044
:105B000064004000D071880054FE070020FD0700AB
:105B1000000F78008081EB009E8F1100030032009F
:105B20001E007800D07188006A03370060002000F2
:105B30003007980067033700100020002007980006
:105B4000D071800064004000D0718800F071800046
:105B5000E90F500018003C00F2718000D171800004
:105B60006E009000008040008001E900820041004A
:105B7000E0E020000080400003087800F071800021
:105B80000000E800F071880034FE070000FD070007
:105B9000000F78008080EB009E8F10000300320021
:105BA0001E017800D27188004A033700600020008F
:105BB0003007980047033700700020003007980036
:105BC00044033700008928004C74020000000000E4
:105BD0001000200020079800F07180000000E00015
:105BE0000A003200F07180000000E900F0718800C6
:105BF000F071800080004000E0E020000080400064
:105C000010007800D0718800320337008000200037
:105C1000300798002F03370010002000200798005D
:105C2000D17180006E009000008040006300400051
:105C3000D07188002703370010002000200798004B
:105C4000D071800064004000D07188005700370098
:105C5000D171800020E42000008040009040780056
:105C600020C2B30080CF50001F003A00D0718000E6
:105C70000000E800D071880010003700D04080009C
:105C80000080A100D0408800D171800020E4200075
:105C90000080400010407800004178000100E800DA
:105CA000D071880002407800A8780200000000004F
:105CB000D04080000080A000D0408800D1718000DA
:105CC00020E42000008040009040780020C2B30013
:105CD00080CF5000E9FF3A00D07180000000E8005A
:105CE000D071880031003700D171800020E420009D
:105CF000008040009040780000C4B30080CF500086
:105D000007003600D171800020E4200000804000B0
:105D100090407800A0C5B30080CF50000D00360041
:105D2000D171800020E42000008040001040780005
:105D30000004E00013003D00D171800020E4200049
:105D40000080400090407800F0CDB30080CF50003C
:105D50000C003E00C1FD0700000F7800D04080001D
:105D60000080A100D04088001E00780086760200E6
:105D700000000000D04080000080A000D0408800DB
:105D80000A003700D171800020E42000008040002C
:105D900090407800B0C3B30080CF500003003A00B9
:105DA000D07180000000E800D0718800D1718000BF
:105DB00020E420000080400090407800F0CDB30047
:105DC00080CF500007003E00D171800020E4200009
:105DD000008040009040780030C8B30080CF500071
:105DE0009BFF3A00D07180008000E90020E4200091
:105DF0000080400090407800B0C3B30080CF5000D6
:105E000009003200D04080000080A100D04088000E
:105E1000609228007874020000000000D0408000EA
:105E20000080A000D040880041FC0700A902370094
:105E30001000200020079800D04080000080A100C2
:105E4000D0408800D071800064004000D07188008C
:105E5000D171800020E42000008040009040780054
:105E600020C2B30080CF500018003A00D0718000EB
:105E70000000E800D07188000A003700D17180006E
:105E800020E42000008040001040780000417800AD
:105E90000100E800D071880002407800A878020074
:105EA00000000000D171800020E42000008040004C
:105EB0009040780020C2B30080CF5000EFFF3A003E
:105EC000D07180000000E800D0718800D17180009E
:105ED00020E420000080400090407800C0C2B30061
:105EE00080CF500004003A00D07180000000E8002C
:105EF000D071880002003700300020003007980081
:105F0000D171800020E42000008040001040780023
:105F10008080FB00F0FB2F00008440008001EB003C
:105F2000F2FF27008000EB000000EB004C22020093
:105F3000000000000001780088004400A0DD20007F
:105F40000080400002087800D07180000000E80066
:105F5000D0718800F6FB0700D04080000080A000D0
:105F6000D04088005B023700100020002007980016
:105F7000D071800064004000D0718800E071800022
:105F8000E30F500004003C00E07180000000E800D6
:105F9000E0718800020037004000200030079800C0
:105FA000E2718000D371800020E420000080410075
:105FB000104078008080FB0000FC2F000082400031
:105FC0006610B9008080E80020E2200000804000D8
:105FD000040878000300E800D0718800D1718000C7
:105FE00020E420000080400090407800D0C3B3003F
:105FF00080CF500011003A00D07180000000E8000E
:10600000D0718800E07180006600B9008080E800EF
:1060100020E2200000804000100078000004E90029
:106020000EFD07000001780088004400A0DD20007C
:106030000080400002087800020037003000200095
:1060400030079800D3718000130F980020E42000DF
:106050009E08900000804000904078000041EB00D6
:1060600002579800B0C8B30080CF500002003A0039
:1060700013C0B300035798009E0890000100E80089
:10608000D07188000E5190000204E0000900320037
:10609000E8718000F1FC0700000178006640B9005B
:1060A000E400400020E22000008040000208780068
:1060B000020037003000200030079800D1718000C6
:1060C00020E420000080400090407800F0CDB30034
:1060D00080CF500008003600E0718000D27180004F
:1060E0006600B9008000780020E2200000804000B7
:1060F00002087800020037003000200030079800C6
:106100008BFB0700F30137001000200020079800E8
:10611000D071800064004000D0718800D27180008E
:1061200020E4200000004100104078008080FB0047
:1061300000FC2F00008F40000200E800D0718800B2
:1061400050002000300798000000EB004007980046
:106150002F0037004E0090006600B9008080E800F4
:1061600020E2200000804000100078009E0F5000C8
:1061700024003A001E00E90080004000A0DD20005D
:1061800000804000100178004E0090006600B900C9
:10619000E400400020E22000008040001000780071
:1061A000800F510012003D009E00E9000181400077
:1061B000A0DD200000004100100078000001E80090
:1061C00081804000A0DD20000080400002087800AF
:1061D0004E0090006600B9008000780020E22000A8
:1061E0000080400010007800D07188000300370064
:1061F000E07180000000E900E07188000000EB0021
:10620000300798004E0090000000E800400798001A
:10621000E17180004E009000810F5000CDFF3400EE
:1062200043FB0700AB013700100020002007980057
:10623000D071800064004000D0718800007280003E
:106240000000E00027003A000000EB004007980043
:106250000A003700CE00900020E4200000804000BB
:10626000104078008080FB004E009000808040004D
:1062700030F22F0000804000400798004E00900050
:10628000E300400020E420000080400090407800BF
:10629000E0C8B30080CF500006003200CE0090006E
:1062A00020E4200000804000104078000004E0005E
:1062B000E8FF3A00CE00900020E42000008040007B
:1062C000104078000004E000040032004E0090000E
:1062D0006400400000728800020037009000200037
:1062E00030079800D3718000030F7800007280009F
:1062F000D07188009E00780020E4200000804000DB
:10630000104078008080FB00F0FB2F0000844000EC
:1063100053FB07000001780088004400A0DD200046
:106320000080400002087800D07180000072880070
:106330001E00E800D07188000172800020E4200077
:106340000080400090407800C0C2B30080CF500071
:1063500003003A00007280000000E800007288002C
:106360000172800020E4200000804000904078000E
:1063700000CEB30080CF50000E00360000728000C7
:10638000E300400020E420000080400090407800BE
:10639000E0C8B30080CF5000030032000000EB00E3
:1063A0000072880003003700007280006400400023
:1063B00000728800DEFA0700460137001000200056
:1063C00020079800D17180006E009000008040008E
:1063D00063004000D07188003E01370010002000AB
:1063E00020079800D071800064004000D0718800C0
:1063F000A1408000E00220000088B9008000780001
:10640000E0932000008040001000780000000100B0
:10641000C7FA07002F01370010002000200798005E
:10642000D071800064004000D0718800A1408000DD
:10643000E00220000088B9008080E800E09320009E
:10644000008040001000780000000100B8FA07004A
:10645000200137001000200020079800D071800034
:1064600064004000D0718800A1408000E00220005C
:106470000088B900E4004000E09320000080400064
:106480001000780000000100A9FA07001101370090
:106490001000200020079800D071800064004000A8
:1064A000D0718800A1408000E00220000088B9007F
:1064B000E6004000E09320000080400010007800DB
:1064C000000001009AFA07000201370010002000C6
:1064D00020079800D071800064004000D0718800CF
:1064E000A1408000E00220000088B900E8004000E0
:1064F000E09320000080400010047800D7FB0700E4
:10650000080001008AFA0700F2003700100020009E
:1065100020079800D071800064004000D07188008E
:10652000CEFB07000000E000030032007C7D02008B
:1065300000000000020037009E7D02000000000005
:106540007BFA0700E30037001000200020079800C6
:10655000D071800064004000D0718800BFFB07004C
:106560000000E00005003200C082A900C282A8003D
:10657000C8A2A900CAA2A80004003700C082A900CE
:10658000C282A900C8A2A900CAA2A90068FA07008D
:10659000D00037001000200020079800D071800044
:1065A00064004000D0718800ACFB07000000E000F0
:1065B00007003200C0B52000104078000000A000A5
:1065C0000010A100C1B52000804878000600370007
:1065D000C0B52000104078000000A0000010A1000D
:1065E000C1B520008048780051FA0700B900370093
:1065F0001000200020079800D07180006400400047
:10660000D071880095FB0700B05F8800B05F800004
:106610000000E00002003D000000EB00B05F8800D9
:10662000B15F800000FA2000808F5000020034002B
:1066300000FA2000B05F8800C05F8000E10F5000CA
:1066400002003C0020002000C05F8800C15F800085
:1066500030062000808F50000200340030062000F9
:10666000C05F8800267A02000000000030FA0700B0
:10667000980037001000200020079800D07180009B
:1066800064004000D071880074FB0700C05F880080
:10669000B05F80000000E00002003D000000EB0061
:1066A000B05F8800B15F800000FA2000808F50004A
:1066B0000200340000FA2000B05F8800C05F800054
:1066C000E10F500002003C0020002000C05F880065
:1066D000C15F800030062000808F5000020034002F
:1066E00030062000C05F8800267A0200000000000B
:1066F0000FFA0700770037001000200020079800ED
:10670000D071800064004000D071880053FB070006
:106710000000E00009003200A1408000E0022000FB
:106720000088B900F0004000E093200000804000A5
:10673000100078000000010008003700A140800030
:10674000E00220000088B900F2004000E093200041
:10675000008040001000780000000100F4F90700FC
:106760005C0037001000200020079800D0718000E6
:1067700064004000D071880038FB07007007980063
:106780007E009000E10F500010003200FE009000EB
:10679000E28F5000160032007E0190000200E000FF
:1067A000010032001A003700A1408000E002200002
:1067B0000088B900EE004000E09320000080400017
:1067C000100078000000010011003700A140800097
:1067D000E00220000088B900EC004000E0932000B7
:1067E0000080400010007800000001000800370021
:1067F000A1408000E00220000088B900F6004000BF
:10680000E0932000008040001000780000000100AC
:10681000C7F907002F00370010002000200798005C
:10682000D071800064004000D0718800D171800078
:106830006E009000008040000000E900D0718800E8
:10684000BBF9070023003700100020002007980044
:10685000D071800064004000D0718800FFFA07000A
:10686000000F78001E007800AA9B020000000000C4
:10687000AFF907001700370010002000200798002C
:10688000D071800064004000D0718800F3FA0700E6
:10689000000F7800A1408000E00220000088B900CD
:1068A000FC004000E0932000008040009000780051
:1068B0001E007800010001009DF907000500370067
:1068C0001000200030079800020037003000200040
:1068D000300798002E0090000000E00005003A000C
:1068E000D17180006E009000008040006300400085
:1068F000D07188000000EB00200798003E00900057
:106900000000E000C8FB3200D04080000080A10001
:10691000D04088003E009000E10F50001800320087
:1069200061002000A03A2000489E02000000000004
:106930003E009000867602000000000081002000EA
:10694000003B2000489E0200000000005E00900016
:106950008676020000000000B1002000803B20008D
:10696000489E020000000000D07180008676020080
:10697000000000006092280078740200000000000F
:106980004F0478000080FA00000006000200FA00C0
:10699000000F780000C2B300A878020000000000D9
:1069A0001E0078004C7402000000000000C2B3001A
:1069B000A8780200000000000080FA000000060035
:1069C0000400FA000000EB00D07188003F0037009F
:1069D000D171800020E420000080400090407800C9
:1069E000214798002E4090000004E000040035008C
:1069F0002E409000A8780200000000003000370010
:106A0000AE40900000CEB30080CF50001C00360096
:106A1000609228007874020000000000D0718000AD
:106A20008000E80020E42000008040001040780052
:106A30000080FB004801DD00D07180008080E8000C
:106A400020E4200000804000104078000080FB001F
:106A500000004100000F7800D07180000080E80045
:106A6000D07188001E0078008676020000000000C9
:106A700000C2B300A8780200000000001000370038
:106A800000C2B300A8780200000000002E40900071
:106A90008080FB0000F82F00008040008000400054
:106AA00040B0200000804000100078004C740200CC
:106AB0000000000000C2B300A8780200000000003F
:106AC000D07180000000E800D0718800D171800092
:106AD00020E4200000804000104078000004E00026
:106AE000BBFF3A00609228007874020000000000AA
:106AF000D07180000000E9008676020000000000EE
:106B000071002000303C2000D29E020000000000F6
:106B10000080FA00000006000600FA001007980046
:106B2000E0678000000F7800150037001E0090001D
:106B300010417800E1678000A0BF20000080400085
:106B400010407800804F5100050032001E00780090
:106B5000E06788000000EB00200798000E00370077
:106B6000E06780008000E800F00F200000806000F7
:106B7000E06788001E0090000000E8001007980001
:106B80001E009000104078000004E000E7FF3A008B
:106B900010002000200798002E0090000080FA00CE
:106BA000000006000400FA000000EB00000F78006F
:106BB000100037001E0078008000400040B0200028
:106BC0000080400010007800D3FF07000000E000C4
:106BD000070032001E0078008040780000C8B30033
:106BE00000C040000080FB0010079800060037003E
:106BF0001E0FE800100220009E0F1000EDFF340071
:106C00000000EB00100798001E0090000080FA00C2
:106C1000000006003600FA00E0678000000F9800D0
:106C20001F0037008E089000A0BF200000804000A9
:106C30009040780000C6B30080CF500011003400AF
:106C40008E089000A0BF2000008040009040780097
:106C5000A0C7B30080CF50000A003C000E0990008E
:106C60008E089000A0BF2000008040009040780077
:106C7000F0CDB30080C06000A0BF20000000410044
:106C8000014878000E0890000000E800000F98000E
:106C90008E089000F00F200000806000000F980028
:106CA0008E089000D0678000808F5000DDFF3A0092
:106CB0000000EB00000F9800E1678000A0BF2000FB
:106CC0000080400090407800F0C2B30080CF5000B8
:106CD0002D013400E1678000A0BF2000008040004B
:106CE0009040780090C3B30080CF500026013C0054
:106CF0000000EB00000F9800070037000E0990001D
:106D0000F20047000040EB0000F178000E08900010
:106D10000000E800000F98008E089000200220007C
:106D2000808F5000F5FF3400521D0200000000006B
:106D3000600798006E0090004880DE008040780078
:106D400072004700114098006E009000804078006B
:106D500000C0EB0080C06000720047002140980036
:106D60006E0090008AF80700500798005E009000BF
:106D7000E10F40002B003200DE00900020E42000F4
:106D800000804000104078008080FB0030F22F002F
:106D900000804000300798005E009000000F9800CF
:106DA0000D0037000E0990008E0890003E00900004
:106DB0008080400020E42000008040009040780067
:106DC00020E4200000004100014878000E089000F7
:106DD0000000E800000F9800014020003E009000F5
:106DE000808050000E089000808F5000EDFF3C0026
:106DF000080037008E08900020E4200080804000CA
:106E00000040EB00804878000E0890000000E80089
:106E1000000F98008E089000F03F2000808F5000F7
:106E2000F4FF340030002000000F98000000EB0059
:106E300020079800202102000000000043003700D6
:106E40002E0090000000E00002003A002021020025
:106E5000000000002E0090000000E00004003A0056
:106E600050FF07000080FB00600798000200370019
:106E70000000EB00600798006E009000467702006B
:106E8000000000006E0090000000E0000C003200E6
:106E90000E0990006E00900080407800720047005C
:106EA00001717800EE00900070082000808F500083
:106EB0001A003A0010002000200798001700370041
:106EC000E1678000A0BF2000008040009040780073
:106ED00020C2B30080CF500003003A002E00900083
:106EE0000000A200200798000E099000E1678000D2
:106EF000A0BF200000804000104078008040780053
:106F00007200470001717800E06780008000E800AF
:106F1000F00F200000806000E06788000E089000FD
:106F20000000E800000F98008E089000300220005A
:106F3000808F50000500340091002000A03C20000C
:106F4000D29E020000000000D4003700E1678000FC
:106F5000D0678000808F5000B9FF3A000E08900083
:106F6000E30F5000CD0032000E089000E40F5000F7
:106F7000CA0032000E08900080407800C0CDB300F7
:106F800000C040008040780072004700014878004F
:106F90000000EB00000F98000000EB004007980095
:106FA0000000EB0050079800460037008E08900064
:106FB00020E42000008040009040780000CEB30024
:106FC00080CF50002E0036008E08900020E4200074
:106FD00000804000104078008080FB0000F22F000D
:106FE00000804000300798000E0890008000E80004
:106FF00020E4200000804000104078000080FB006A
:107000004801DD000E0890008080E80020E42000A8
:1070100000804000104078000080FB00000041002C
:107020001007980072004700104090000080FB009D
:10703000C800DD0072004700204090000080FB0087
:1070400000804000000F78001E0090009E0F50004E
:10705000050031008E0890003E0090000080400046
:107060006300400050079800BE0090000E0890009A
:107070000080400063004000000F980002003700CD
:107080000E089000400798000E0890008000E8006D
:1070900020E4200000804000104078000080FB00C9
:1070A0004801DD000E0890008080E80020E4200008
:1070B00000804000104078000080FB00000041008C
:1070C000600798004E0090000000E000B7FF32001B
:1070D00072004700104078008080FB0030F22F00E3
:1070E00000804000600798004E009000000F98005C
:1070F0000D0037008E0890006E0090000081400067
:107100008E08900020E4200000804000904078002D
:1071100020E4200000004100014878000E089000A3
:107120000000E900000F98008E0890005E009000BB
:10713000808F5000EFFF3D000000EB00000F980033
:107140000C003700DE0090000E0890000081400027
:107150008E08900072004700E140780020E4200093
:1071600000004100014878000E0890000000E8008F
:10717000000F98008E0890006E009000808F5000E5
:10718000F0FF3500450037007092280062FE0700CE
:107190000000E000050032007EF907006092280040
:1071A00078740200000000003C003700B092280014
:1071B00059FE07000000E0000200320000FE070058
:1071C000360037000093280053FE07000000E0005F
:1071D00004003200D04080000090A100D040880020
:1071E0002E003700509328004BFE07000000E000FF
:1071F000200032000000EB00000F9800180037005C
:107200000000EB00700798000F0037008E08900018
:107210007E0090008080400020E42000008040003C
:10722000104078000080FB0046770200000000005C
:1072300000C2B300A8780200000000007E009000A9
:107240000000E800700798007E009000EF0F5000EB
:10725000EEFF34000E08900070004000000F980010
:107260008E089000F03F2000808F5000E4FF340033
:107270000A003700B093280027FE07000000E00056
:10728000020032000700070004003700C1002000A0
:10729000303D2000D29E0200000000000080FA0075
:1072A000000006000200FA000000EB00000F78006A
:1072B000060037009E00780020E420008080400017
:1072C0000040EB00804878001E0FE800F03F2000EF
:1072D0009E0F1000F7FF340011CEB30020E4200011
:1072E0000148780080C0EB0030E4200001487800BD
:1072F00080C0EB0040E420000148780011CAB300D0
:1073000050E42000014878000080FA0000000600E8
:107310005752490054452000424954003A20200069
:107320002A6E650078742000636C6F00636B200028
:10733000285E2900207769006C6C20007573650059
:10734000207468006973200076616C0075653100F7
:1073500057495200452072006F757400696E6500D0
:1073600073202800432920003230300030204D00A7
:107370006963680061656C0020506500617263009C
:10738000652047004E55200047504C004E6F2000AE
:1073900064657600696365002C20740072792000B2
:1073A00028414C0041524D002920530045415200D4
:1073B000434820006D616300726F200066697200AF
:1073C000737441004444520045535300204D410022
:1073D00043524F00202030002E4D610063726F0039
:1073E000206D65006E754D00616372006F20200096
:1073F000202020003157490052452000616464007C
:1074000072657300730D0A00202020002A31570096
:107410004952450020524F004D2043004F4D4D0032
:10742000414E4400204D410043524F00733A0D003D
:107430000A203500312E52004541440020524F00B1
:107440004D20280030783300332920002A666F0051
:1074500072207300696E67006C65200064657600B9
:107460006963650020627500730D0A0020383500DD
:107470002E4D41005443480020524F004D2028001B
:1074800030783500352920002A666F006C6C6F005B
:1074900077656400206279002036340062697400E8
:1074A000206164006472650073730D000A2032006D
:1074B00030342E00534B4900502052004F4D2000D5
:1074C0002830780043432900202A66006F6C6C0046
:1074D0006F77650064206200792063006F6D6D0036
:1074E000616E64000D0A2000323336002E414C00DC
:1074F00041524D002053450041524300482028008E
:107500003078450043290D000A20320034302E0027
:10751000534541005243480020524F004D2028005F
:1075200030784600302941004C4152004D20530034
:107530004541520043482000283078004543290047
:10754000534541005243480020283000784630001F
:107550002944650076696300652049004473200072
:10756000617265002061760061696C0061626C0087
:107570006520620079204D00414352004F2C2000CD
:107580007365650020283000292E520045414400D3
:1075900020524F004D2028003078330033293A0024
:1075A000204D41005443480020524F004D202800F8
:1075B00030783500352953004B49500020524F0098
:1075C0004D20280030784300432955006E6B6E0033
:1075D0006F776E00206D610063726F002C20740065
:1075E000727920003F206F0072202800302920008F
:1075F000666F7200206865006C7042005553200071
:107600005245530045542000576172006E696E0068
:10761000673A20002A5368006F727400206F72006E
:10762000206E6F00207075006C6C2D00757020004E
:107630002A4E6F002064650076696300652064004F
:10764000657465006374650064204400533138003C
:10765000533230002048690067682000507265008E
:10766000732044006967200054686500726D44000F
:107670005331380042323000205072006F672000D2
:1076800052657300204469006720540068657200E9
:107690006D4453003138320032204500636F6E0074
:1076A0002044690067205400686572006D445300EF
:1076B0003234300034204500636F6E0072616D001B
:1076C000207469006D6520004368690070445300B0
:1076D00032343300312031004B20450045505200F8
:1076E0004F4D55006E6B6E006F776E002064650025
:1076F00076696300655057004D206400697361002E
:10770000626C650064314B00487A2D00342C3000E7
:1077100030304B00487A200050574D0046726500CB
:10772000717565006E63790020696E00204B48001A
:107730007A2050007265730063616C00653A5000F6
:1077400052323A00447574007920630079636C000A
:10775000652069006E202500205057004D206100F3
:10776000637469007665450052524F00523A20001A
:1077700050574D002061630074697600652C20002D
:10778000672074006F20640069736100626C65009B
:10779000415558002046720065717500656E6300A2
:1077A000793A20004155580020494E005055540068
:1077B0002F4849002D5A410055582000484947009C
:1077C0004841550058204C004F5756004F4C54002C
:1077D0004D455400455220004D4F440045564F0042
:1077E0004C5441004745200050524F0042453A005A
:1077F0002056450072726F007228290020406C00EC
:10780000696E65003A20400070676D00737061001A
:1078100063653A0020627900746573002E546F002E
:107820006F206C006F6E6700215379006E746100E9
:107830007820650072726F00724E6F00204545001F
:1078400050524F004D457200617369006E676400CD
:107850006F6E650053617600696E670020746F007B
:1078600020736C006F742000496E7600616C6900B3
:10787000642073006C6F74004C6F610064696E006B
:1078800067206600726F6D0020736C006F742000BB
:10789000455252004F523A0020636F006D6D6100F7
:1078A0006E64200068617300206E6F0020656600C2
:1078B00066656300742068006572650041434B0093
:1078C0004E4143004B493200432053005441520083
:1078D00054204200495449003243200053544F0081
:1078E0005020420049544900324320006D6F64002B
:1078F000653A0D000A2031002E2053006F66740097
:1079000077617200650D0A0020322E002048610068
:1079100072647700617265005365740020737000B3
:10792000656564003A0D0A0020312E00207E350086
:107930004B487A000D0A2000322E20007E353000A0
:107940004B487A000D0A2000332E20007E31300093
:10795000304B48007A0D0A0020342E00207E34007F
:1079600030304B00487A570041524E00494E470094
:107970003A204800415244005741520045204900F6
:10798000324320006973200062726F006B656E00E5
:10799000206F6E0020746800697320005049430016
:1079A000212028005245560020413300295365000C
:1079B0007420730070656500643A0D000A20310080
:1079C0002E20310030304B00487A0D000A20320062
:1079D0002E20340030304B00487A0D000A2033004E
:1079E0002E2031004D487A004932430020286D0096
:1079F0006F64200073706400293D2800202030004F
:107A00002E4D610063726F00206D65006E750D0074
:107A10000A2031002E37620069742000616464001E
:107A200072657300732073006561720063680D00F6
:107A30000A2032002E493200432073006E6966002E
:107A4000666572005365610072636800696E670065
:107A50002049320043206100646472006573730042
:107A600020737000616365002E2046006F756E0004
:107A700064206400657669006365730020617400AA
:107A80003A536E00696666006572280042415300F1
:107A90004943290052656100647961002F412F003C
:107AA000402063006F6E7400726F6C0073204100A1
:107AB0005558200070696E00612F41002F40200052
:107AC000636F6E0074726F006C732000435320006C
:107AD00070696E00436F6D006D616E0064206E0012
:107AE0006F74200075736500642069006E20740057
:107AF00068697300206D6F0064655000756C6C00E0
:107B00002D7570002072650073697300746F7200C8
:107B100073204F0046465000756C6C002D75700048
:107B20002072650073697300746F720073204F00D8
:107B30004E5365006C662D007465730074206900F7
:107B40006E204800695A20006D6F640065206F0048
:107B50006E6C790052455300455442004F4F54001B
:107B60004C4F4100444552004155580020494E00B9
:107B7000505554002F4849002D5A2C0020524500E2
:107B800041443A0020506F00776572002073750001
:107B900070706C0069657300204F4E00506F770065
:107BA0006572200073757000706C69006573200049
:107BB0004F46460044415400412053005441540074
:107BC000453A200044454C00415920007573570048
:107BD00052495400453A200052454100443A2000A1
:107BE000434C4F00434B2C00203143004C4F43008B
:107BF0004B2C200030444100544120004F5554008C
:107C0000505554002C2031004441540041204F0075
:107C10005554500055542C00203020002A70690023
:107C20006E20690073206E006F77200048695A004B
:107C3000434C4F00434B2000544943004B533A0000
:107C40002052450041442000424954003A2053004C
:107C5000796E740061782000657272006F72200086
:107C60006174200063686100722078002E20650036
:107C7000786974002877690074686F007574200053
:107C8000636861006E676500296E6F00206D6F008C
:107C900064652000636861006E6765004E6F6E006A
:107CA00065786900737465006E74200070726F00EF
:107CB000746F63006F6C2100782E20006578690076
:107CC000740D0A00496E7600616C690064206300DF
:107CD000686F690063652C00207472007920610070
:107CE000676169006E444500564944003A68740073
:107CF00074703A002F2F6400616E670065726F0028
:107D000075737000726F74006F7479007065730022
:107D10002E636F006D2A2D002D2D2D002D2D2D0091
:107D20002D2D2D002A4F7000656E200064726100B9
:107D3000696E20006F7574007075740073202800E0
:107D4000483D4800692D5A002C204C003D474E000C
:107D500044294E006F726D00616C20006F757400D5
:107D60007075740073202800483D33002E33760070
:107D70002C204C003D474E0044294D00534220002A
:107D8000736574003A204D004F535400207369000E
:107D900067206200697420006669720073744C0089
:107DA00053422000736574003A204C004541530053
:107DB00054207300696720006269740020666900BE
:107DC0007273740020426F006F746C006F61640006
:107DD00065722000762031002E20480045580D00A5
:107DE0000A2032002E20440045430D000A203300B3
:107DF0002E204200494E0D000A2034002E20520051
:107E000041574400697370006C61790020666F000F
:107E1000726D610074207300657456006F6C74009D
:107E200061676500206D6F006E6974006F7273008A
:107E30003A203500563A2000207C2000332E3300B3
:107E4000563A2000207C2000565055004C4C5500DE
:107E5000503A200053657400207365007269610018
:107E60006C2070006F727400207370006565640090
:107E70003A20280062707300290D0A0020312E007C
:107E800020333000300D0A0020322E002031320025
:107E900030300D000A2033002E2032003430300004
:107EA0000D0A2000342E200034383000300D0A0036
:107EB00020352E002039360030300D000A203600E3
:107EC0002E20310039323000300D0A0020372E00CC
:107ED00020333800343030000D0A2000382E2000C6
:107EE0003537360030300D000A2039002E203100A1
:107EF0003135320030300D000A3130002E20420082
:107F00005247200072617700207661006C75650031
:107F100041646A007573740020796F0075722000E7
:107F2000746572006D696E00616C410072652000BD
:107F3000796F75002073750072653F00204346001D
:107F400047313A002043460047323A00285C2D0072
:107F50002F5F5C002D2928005C5F2F002D29530026
:107F6000656C6500637420006F7574007075740033
:107F70002074790070653A000D0A2000312E20002F
:107F80004F7065006E206400726169006E202800E9
:107F9000483D4800692D5A002C204C003D474E00BA
:107FA00044290D000A2032002E204E006F726D0011
:107FB000616C200028483D00332E3300562C2000F1
:107FC0004C3D47004E442900523257002028730090
:107FD0007064200068697A00293D28002020300064
:107FE0002E4D610063726F00206D65006E750D008F
:107FF0000A2031002E4953004F37380031362D000A
:108000003320410054520D000A2032002E49530003
:108010004F37380031362D00332070006172730005
:1080200065206F006E6C790049534F00203738008F
:1080300031362D0033204100545220002852450093
:1080400053455400206F6E0020435300290D0A0051
:10805000524553004554200048494700482C200011
:10806000434C4F00434B2000544943004B2C20000D
:1080700052455300455420004C4F570049534F0080
:108080002037380031362D003320720065706C00C7
:108090007920280075736500732063007572720083
:1080A000656E7400204C53004220730065747400A8
:1080B000696E6700293A200050726F00746F630088
:1080C0006F6C3A0020736500726961006C332000A8
:1080D0007769720065322000776972006552460048
:1080E00055756E006B6E6F00776E520065616400AF
:1080F0002074790070653A0020746F0020656E006E
:108100006476610072696100626C6500206C6500D4
:108110006E6774006844610074612000756E6900C8
:1081200074733A00206E6F0020696E00646963000A
:10813000617469006F6E44006174610020756E00A7
:10814000697420006C656E00677468002028620006
:1081500069747300293A200043532000454E4100C2
:10816000424C4500444353002044490053414200DF
:108170004C4544005233570020287300706420009F
:1081800063736C00206869007A293D00282029006B
:108190000D0A4400697363006F6E6E0065637400BE
:1081A00020616E0079206400657669006365730064
:1081B0000D0A43006F6E6E00656374002028560040
:1081C00070752000746F20002B3556002920610047
:1081D0006E64200028414400432074006F202B006F
:1081E000332E33005629430074726C0041555800F9
:1081F0004D4F440045204C0045445000554C4C0028
:1082000055502000485055004C4C550050204C0013
:108210005652450047414400432061006E642000EF
:1082200073757000706C79003556560050553300E8
:108230002E335600414443004275730020686900A4
:10824000676842007573200048692D005A2030008D
:1082500042757300204869002D5A2000314D4F00AF
:1082600044452000616E64002056520045472000BE
:108270004C45440073207300686F75006C642000E7
:10828000626520006F6E2100466F75006E642000ED
:1082900020657200726F7200732E4D004F534900BB
:1082A000434C4B004D4953004F435300204F4B006C
:1082B00020464100494C53006574200073706500EE
:1082C00065643A000D0A2000312E200033304B0047
:1082D000487A0D000A2032002E20310032354B0042
:1082E000487A0D000A2033002E20320035304B0032
:1082F000487A0D000A2034002E2031004D487A00C3
:10830000436C6F00636B2000706F6C0061726900DA
:1083100074793A000D0A2000312E200049646C0067
:1083200065206C006F7720002A6465006661750027
:108330006C740D000A2032002E204900646C650028
:108340002068690067684F007574700075742000BC
:10835000636C6F00636B200065646700653A0D0015
:108360000A2031002E204900646C650020746F00E3
:108370002061630074697600650D0A0020322E00CA
:108380002041630074697600652074006F206900E5
:10839000646C6500202A640065666100756C740079
:1083A000496E70007574200073616D00706C65001B
:1083B00020706800617365003A0D0A0020312E00BC
:1083C000204D690064646C0065202A0064656600C5
:1083D00061756C00740D0A0020322E0020456E007D
:1083E00064535000492028007370640020636B00C0
:1083F000702073006B652000736D70002063730044
:108400006C206800697A29003D28200020302E0069
:108410004D616300726F20006D656E00750D0A007E
:1084200020312E00536E6900666620004353200001
:108430006C6F77000D0A2000322E53006E696600C3
:10844000662061006C6C20007472610066666900D1
:10845000632D7000202D6600202A4200797465008B
:1084600073206400726F7000706564002A464100DA
:10847000494C4500442C20004E4F200044415400FC
:1084800041446100746120006269740073206100DE
:108490006E64200070617200697479003A0D0A0000
:1084A00020312E0020382C00204E4F004E45200059
:1084B0002A646500666175006C7420000D0A200056
:1084C000322E2000382C2000455645004E200D004D
:1084D0000A2033002E2038002C204F004444200076
:1084E0000D0A2000342E2000392C20004E4F4E0063
:1084F000455374006F70200062697400733A0D0078
:108500000A2031002E203100202A640065666100B7
:10851000756C74000D0A2000322E20003252650066
:108520006365690076652000706F6C006172690098
:1085300074793A000D0A2000312E200049646C0045
:1085400065203100202A640065666100756C740046
:108550000D0A2000322E200049646C006520300096
:10856000554152005420280073706400206272004C
:1085700067206400627020007362200072787000CF
:10858000206869007A293D0028202000302E4D0007
:10859000616372006F206D00656E75000D0A20002A
:1085A000312E540072616E007370610072656E004E
:1085B000742062007269640067650D000A20320051
:1085C0002E204C0069766500206D6F006E69740086
:1085D0006F720D000A2033002E427200696467003A
:1085E000652077006974680020666C006F77200052
:1085F000636F6E0074726F006C554100525420001E
:1086000062726900646765005265730065742000DA
:10861000746F2000657869007452610077205500FE
:108620004152540020696E0070757400554152002B
:1086300054204C00495645002044490053504C00FA
:1086400041592C00207D2000544F200053544F00EE
:10865000504C49005645200044495300504C4100BD
:1086600059205300544F5000504544005741520088
:108670004E494E00473A200070696E0073206E002C
:108680006F7420006F7065006E2064007261690075
:108690006E20280048695A0029205200455649009A
:1086A000443A0D000A496E0076616C00696420004E
:1086B00063686F00696365002C2074007279200084
:1086C00061676100696E6D0073525300204C4F006A
:1086D000572C2000434F4D004D414E0044204D008B
:1086E0004F4445005253200048494700482C200081
:1086F0004441540041204D004F4445004164640012
:108700007265730073206F00662050004346380086
:10871000353734003F546800697320006D6F640082
:1087200065207200657175006972650073206100D3
:108730006E20610064617000746572004C434400F7
:108740002074790070653A000D0A2000312E200057
:1087500048443400343738003020280075736900ED
:108760006E672000504346003835370034204900FA
:108770004F206500787061006E64650072294C00BE
:108780004344200028747900702061006464720002
:1087900029203D002028200020302E004D6163005C
:1087A000726F20006D656E00750D0A0020312E007D
:1087B0004C43440020526500736574000D0A20008C
:1087C000322E49006E697400204C4300440D0A00AB
:1087D00020332E00436C6500617220004C4344003E
:1087E0000D0A2000342E4300757273006F72200052
:1087F000706F7300697469006F6E200065783A00CD
:108800002834290020300D000A2036002E5772002F
:108810006974650020746500737420006E756D00C6
:108820006265720073206500783A280036292000BE
:1088300038300D000A2037002E5772006974650029
:1088400020746500737420006368610072616300C6
:108850007465720073206500783A2800372920007B
:1088600038304400697370006C617900206C6900D5
:108870006E6573003A0D0A0020312E002031200071
:108880000D0A2000322E20004D756C0074697000B6
:108890006C6549004E495400434C45004152430029
:1088A000555253004F522000534554004E6F200044
:1088B00041434B002C206300686563006B2061001E
:1088C0006461700074657200434C4B00094D4F00A9
:1088D00053490900435309004D4953004F50690063
:1088E0006E73740061746500733A47004E4409006A
:1088F000332E3300560935002E305600094144000E
:1089000043095600505509004155580009500900C7
:10891000500950000949090049092D00094F570025
:1089200044092D00092D2D000954780044092D001B
:1089300009527800445343004C0953004441090054
:108940002D092D00504743000950470044092D00D0
:10895000092D31002E28420052290900322E28000C
:108960005244290009332E00284F520029093400AF
:108970002E28590057290900352E2800474E290076
:1089800009362E0028424C00290937002E285000B5
:1089900055290900382E28004752290009392E0090
:1089A00028575400290930002E2842006C6B2900FA
:1089B000474E440009474E00440941004443090022
:1089C000352E3000560933002E335600095650001C
:1089D00055094100555809006578650063757400B4
:1089E00065203A002020610075746F0072616E008E
:1089F000676520002B4D48007A292B006B487A00D0
:108A00002952610077207600616C75006520660050
:108A10006F7220004252470020284D00494449000F
:108A20003D3132003729570041524E00494E470030
:108A30003A2050006F73730069626C006520620019
:108A40007566660065726F0076657200666C6F0011
:108A500077416E0079206B0065792000746F2000EB
:108A600065786900745370006163650020746F005D
:108A700020636F006E7469006E7565004E756D0041
:108A800062657200206F66002062690074732000C6
:108A900072656100642F770072697400653A200086
:108AA00043533A000D0A2000312E200043530D009D
:108AB0000A2032002E202F00435320002A64650034
:108AC000666175006C7450006F73690074696F00A3
:108AD0006E2069006E206400656772006565730032
:108AE00053657200766F20006163740069766500DB
:108AF00047656E00657261006C090900090909008B
:108B000050726F00746F63006F6C2000696E7400A8
:108B100065726100637469006F6E2D002D2D2D004C
:108B20002D2D2D002D2D2D002D2D2D002D2D2D0029
:108B30002D2D2D002D2D2D002D2D2D002D2D2D0019
:108B40002D2D2D002D2D2D002D2D2D002D2D2D0009
:108B50002D2D2D002D2D2D002D2D2D002D2D2D00F9
:108B60002D2D2D002D2D2D002D2D2D002D2D2D00E9
:108B70002D2D2D002D2D2D002D2D2D002D2D3F00C7
:108B8000095468006973200068656C007009090069
:108B90000928300029094C006973740020637500AE
:108BA000727265006E7420006D616300726F7300F5
:108BB0003D582F007C580900436F6E0076657200A7
:108BC00074732000582F720065766500727365001B
:108BD000205809000928780029094D0061637200B6
:108BE0006F2078007E095300656C66007465730021
:108BF00074090900095B0900537461007274230051
:108C0000095265007365740009090900095D0900CE
:108C100053746F00702409004A756D007020740051
:108C20006F2062006F6F74006C6F6100646572008A
:108C300009097B0009537400617274002077690090
:108C4000746820007265610064262F0025094400C5
:108C5000656C610079203100207573002F6D730001
:108C6000090909007D095300746F7000612F4100EC
:108C70002F4009004155580050494E0020286C00F3
:108C80006F772F0048492F005245410044290900C1
:108C90000922610062632200095365006E642000AE
:108CA00073747200696E6700620953006574200076
:108CB0006261750064726100746509000909310020
:108CC000323363002F43090041555800206173007F
:108CD000736967006E6D65006E7420002861750011
:108CE000782F4300532909000930780031323300CE
:108CF000642F4400094D65006173750072652000A2
:108D00004144430020286F006E6365002F434F00ED
:108D10004E542E00290930006231310030095300D1
:108D2000656E6400207661006C75650066094D0013
:108D3000656173007572650020667200657175006B
:108D4000656E63007909090072095200656164006B
:108D5000672F5300094765006E65720061746500F6
:108D6000205057004D2F5300657276006F0909009F
:108D70002F0943004C4B20006869680009436F00CD
:108D80006D6D61006E646800697374006F727900C4
:108D9000090909005C0943004C4B20006C6F690015
:108DA00009566500727369006F6E69006E666F0028
:108DB0002F7374006174750073696E00666F09002B
:108DC000095E0900434C4B0020746900636B6C0022
:108DD0002F4C0900426974006F72640065722000B4
:108DE000286D7300622F4C005342290009092D00A1
:108DF0000944410054206800696D0900436861001E
:108E00006E676500206D6F006465090009095F00E9
:108E10000944410054206C006F6F090053657400D1
:108E2000206F75007470750074207400797065008F
:108E3000090909002E0944004154200072656100AF
:108E400064702F0050095000756C6C007570200024
:108E500072657300697374006F72730020286F006D
:108E600066662F004F4E29000921090042697400EF
:108E700020726500616473000953630072697000B9
:108E8000742065006E6769006E65090009093A0083
:108E90000952650070656100742065002E672E0020
:108EA00020723A0031307600095368006F77200055
:108EB000766F6C0074732F007374610074657300B7
:108EC00009092E000942690074732000746F2000A4
:108ED00072656100642F7700726974006520650017
:108EE0002E672E002030780035352E0032772F0087
:108EF0005709500053552000286F6600662F4F0019
:108F00004E290900093C78003E2F3C00783D2000A6
:108F10003E2F3C00303E090055736500726D6100C4
:108F200063726F0020782F006173730069676E00B1
:108F300020782F006C697300742061006C6C000055
:108F40000000FA00C0B52000104078000060A000CA
:108F5000C1B5200080487800A0B6200010407800FD
:108F6000684060000004E00002003200CAC2A900AC
:108F700001003700CAC2A800A0B620001040780047
:108F8000684060000004E00003003200F0C2B3005B
:108F9000A878020000000000A100200060AB2000C3
:108FA000D29E0200000000000080FA0000000600CF
:108FB0000000FA00C0B52000104078000060A10059
:108FC000C1B5200080487800A0B62000104078008D
:108FD000684060000004E00002003200CAC2A9003C
:108FE00001003700CAC2A800A0B6200010407800D7
:108FF000684060000004E00003003200F0C2B300EB
:10900000A878020000000000A100200060AB200052
:10901000D29E0200000000000080FA00000006005E
:109020000000FA00A0B62000104078006840600000
:109030000004E00002003200CAC2A80001003700AC
:10904000CAC2A900A0B620001040780068406000A5
:109050000004E00003003200F0C2B300A878020070
:1090600000000000B100200000AC2000D29E0200F1
:10907000000000000080FA00000006000000FA0076
:1090800000C0EB00820207000080FB000080FA00B5
:10909000000006000600FA00100798001E0090006D
:1090A0007B020700004F7800C0B520001040780018
:1090B0000044B2000004E000030032001E80FB0008
:1090C0002007980001003700010037002E009000B3
:1090D0000080FA00000006000000FA0001022000F3
:1090E000D0C92000489E020000000000A0B420006B
:1090F000104078000040E800E47602000000000024
:1091000000C2B300A878020000000000A0B6200052
:109110001040780061406000E4760200000000002A
:1091200000C2B300A878020000000000A0B6200032
:10913000104078000080FB000000D100614060001A
:10914000E47602000000000000C2B300A87802002C
:1091500000000000A0B62000104078000080FB0056
:109160004200DE0061406000E47602000000000082
:1091700000C2B300A878020000000000A0B62000E2
:10918000104078000080FB004300DE00614060007A
:10919000E47602000000000000C2B300A8780200DC
:1091A00000000000C0B52000104078000080FB00E7
:1091B0004400DE0061406000E47602000000000030
:1091C00000C2B300A87802000000000031002000B7
:1091D000F0AD2000489E0200000000000080FA0070
:1091E000000006000C00FA00202102000000000030
:1091F000521D0200000000005007980020210200CC
:1092000000000000521D020000000000400798000E
:109210002021020000000000521D0200000000009A
:10922000300798002021020000000000521D0200BB
:10923000000000002007980020210200000000002C
:10924000521D020000000000000F780020210200E3
:1092500000000000521D02000000000010079800EE
:109260005E0090000000E000090034005E00900005
:10927000E40F500006003C005E0090000040E90052
:1092800080407800A0B42000014878000200370038
:109290000000EB00500798004E0090000000E00036
:1092A0000F0034004E009000E20F50000C003C0014
:1092B0004E0090000040E900E1406000A0B62000B0
:1092C0001040780061C16000E1CFB3000140600050
:1092D00002407000A1B620008048780002003700EC
:1092E0000000EB00500798003E0090000000E000F6
:1092F000100034003E009000E20F50000D003C00D2
:109300003E0090000040E90061416000A0B62000EE
:10931000904078006140610000414000D0CFB30030
:1093200080C0600082C07000A0B6200001487800B4
:10933000020037000000EB00500798002E0090005C
:109340000000E000100034002E009000E20F5000FA
:109350000D003C002E0090000040E90061416000DB
:10936000A0B6200090407800614061004201DD001D
:10937000B0CFB30080C0600082C07000A0B62000F3
:1093800001487800020037000000EB005007980009
:109390001E00E00010003400200020009E0F10008E
:1093A0000D003C001E0078000040E90061416000B3
:1093B000A0B6200090407800614061004301DD00CC
:1093C00070CFB30080C0600082C07000A0B62000E3
:1093D00001487800020037000000EB0050079800B9
:1093E0001E0090000000E000100034001E009000FD
:1093F000E20F50000D003C001E0090000040EA000B
:1094000061416000C0B5200090407800614061007B
:109410004401DD00F0CEB30080C0600082C0700067
:10942000C0B5200001487800020037000000EB00C2
:10943000500798005E0090000000E00079003A00BC
:109440000000EB00F067880071032000D0BB200013
:10945000D29E0200000000008001EB0042002000CC
:1094600011002000100020004C220200000000002B
:109470000040E90080407800A0B420000148780056
:109480005103200040BF2000D29E020000000000D7
:109490008001EB00220020001100200010002000BD
:1094A0004C220200000000000040E900E1406000A2
:1094B000A0B620001040780061C16000E1CFB30089
:1094C0000140600002407000A1B620008048780092
:1094D0003104200090C22000D29E02000000000053
:1094E0008001EB002200200011002000200020005D
:1094F0004C220200000000000040E90061416000D1
:10950000A0B620009040780061406100004140001A
:10951000D0CFB30080C0600082C07000A0B6200031
:109520000148780011032000C0C62000D29E02002E
:10953000000000008001EB0022002000110020004C
:10954000100020004C220200000000000040E90052
:1095500061416000A0B62000904078006140610049
:109560004201DD00B0CFB30080C0600082C0700057
:10957000A0B6200001487800D1012000C01A2100C7
:10958000D29E0200000000008001EB0022002000BB
:1095900011002000200020004C22020000000000EA
:1095A0000040E90061416000A0B6200090407800D2
:1095B000614061004301DD0070CFB30080C06000F6
:1095C00082C07000A0B6200001487800F10420009D
:1095D000B0932000D29E0200000000008001EB004A
:1095E0002200200011002000100020004C22020068
:1095F000000000000040EA0061416000C0B52000AA
:1096000090407800614061004401DD00F0CEB3007D
:1096100080C0600082C07000C0B5200001487800A2
:1096200001003700ACFE0700C0B5200010407800F4
:109630000060A100C1B5200080487800A0B42000DF
:10964000104078008080FB00E08120000080400016
:1096500010407800A6000700A0B620001040780057
:109660000080FB004300DE0061406000614060005C
:109670004601DD00A12C200091407800F0CBB30022
:1096800000C0600002407000CAE2B7000080FA002B
:10969000000006000000FA00E90007000080FA0060
:1096A000000006000600FA00000F78001E00780097
:1096B0006101B8001207980023079800F00020000D
:1096C000010020001E019000AE019000800F5100AB
:1096D000818F590079003E001E009000AE0090007E
:1096E000006001000F003700130037001E00370034
:1096F0007600370071003700700037006F003700C8
:109700006E0037006D0037006C0037002200370014
:10971000270037002C0037003100370036003700B3
:109720003B00370041032000D0CB2000D29E020036
:109730000000000065003700710020005059200033
:10974000D29E020000000000F1002000101721004E
:10975000D29E02000000000011C0B3000040EB00E8
:10976000D90007005900370071002000505920002F
:10977000D29E020000000000F1002000101721001E
:10978000D29E02000000000011C0B30010C0B30060
:10979000CD0007004D003700A0B620001040780033
:1097A0000000A100A1B62000804878001D0037000D
:1097B000A0B62000104078000000A000A1B6200054
:1097C0008048780017003700A0B6200010407800CD
:1097D0000010A100A1B620008048780011003700D9
:1097E000A0B62000104078000010A000A1B6200014
:1097F000804878000B003700A0B6200010407800A9
:109800000020A100A1B620008048780005003700A4
:10981000A0B62000104078000020A000A1B62000D3
:1098200080487800A0B620001040780061406000B9
:10983000614060004601DD00212420009140780055
:10984000F0CBB30000C060000240700042E2B700FD
:10985000A0B62000104078000080FB000000D1007E
:109860006140600061416000312420009140780037
:10987000E0CFB30000C060000240700043E2B700D8
:10988000A0B62000104078000080FB004200DE00FF
:1098900061406000614060000041400031242000D0
:1098A00091407800D0CFB30000C06000024070004B
:1098B00043E2B70008FE0700040037004102200021
:1098C000C0202000D29E0200000000000080FA00AC
:1098D000000006000000FA0001012000A0042100A1
:1098E000D29E0200000000000080FA000000060086
:1098F0000200FA00004F780041E2A900C0B5200044
:1099000010407800704060000004E0000400320065
:10991000CEE2A800CF02A800CEC2A8000300370004
:10992000CEE2A900CF02A900CEC2A900816A200020
:109930009140780000CEB30000C060007040B300DA
:10994000A8E6B700916C20009140780000CEB300EB
:1099500000C060007040B300C9E6B700816C200011
:109960009140780000CEB30000C060000034A00039
:10997000C8E6B700CAC2A800C8C2A900C902A900A7
:10998000C8E2A800C922A9001E80FB0010128800AE
:1099900042A2A800A0B620001040780061406000FC
:1099A000614060004601DD002124200091407800E4
:1099B000F0CBB30000C060000240700042E2B7008C
:1099C000A0B62000104078000080FB000000D1000D
:1099D00061406000614160003124200091407800C6
:1099E000E0CFB30000C060000240700043E2B70067
:1099F000A0B62000104078000080FB004200DE008E
:109A0000614060006140600000414000312420005E
:109A100091407800D0CFB30000C0600002407000D9
:109A200043E2B7000000EB00201288000000EB00CA
:109A30000012880041E2A8000080FA000000060041
:109A40000000FA0041E2A900A8C6BF00F041B3003F
:109A5000A8E6B700916C20009140780000CEB300DA
:109A600000C06000C9E6B700816C2000914078001A
:109A700000CEB30000C06000C8E6B700CEE2A90087
:109A8000CF02A900CEC2A9000080FA0000000600A3
:109A90000200FA00004F78001E80FB004012880090
:109AA00085C0BF00644060000004E000FCFF32009D
:109AB00040128000004F78008540A9001E80FB0006
:109AC0000080FA00000006000400FA002047980019
:109AD0003147980010C0B300004F78005079020061
:109AE00000000000D6FF0700850007002E40900010
:109AF0000004E00002003A0042E2A80062E2A8008E
:109B00002E409000E14F500002003E0041E2A800CC
:109B100061E2A8001E04E00009003A00CAC2BF00CA
:109B20000044B2000004E00005003200D0C5B300DC
:109B3000647902000000000010C0B300004F7800FC
:109B400040C2BF000042B2000004E0002F003A0013
:109B500060C2BF000042B2000004E0002B003A00E7
:109B6000401280001047980010C0B3009E4F1000B4
:109B700005003A00B0C5B30064790200000000009F
:109B80000040EB00004F78003E4090000004E000F1
:109B9000050032001E4090000080FB00707702003C
:109BA0000000000006003700C0C5B3006479020061
:109BB000000000001E4090006479020000000000D8
:109BC00040138000104798003E4090000004E000E1
:109BD0000B00320080C2B300647902000000000074
:109BE0001E4090000080FB00707702000000000023
:109BF00090C2B30064790200000000000300370047
:109C00001E409000647902000000000040C2BF00C6
:109C10000044B2000004E00009003A0060C2BF0046
:109C20000044B2000004E00005003A00D04080008B
:109C300001402000010060000000E000140032003C
:109C4000D040800001402000010060000000E000E2
:109C500002003A00CC790200000000000000EB0096
:109C6000001288000000EB00001388003E409000C6
:109C70000004E00004003200C0A128007874020053
:109C80000000000093FF3700CA82A90012003700CD
:109C900023C2BF00624060000004E00002003A00FE
:109CA0009A7902000000000022C2BF0061406000FB
:109CB0000004E00097FF3200301180001047980048
:109CC0003E4090000004E00003003200D0A22800D3
:109CD000787402000000000088000700A0B4200093
:109CE000104078008080FB00E08120000080400070
:109CF00010407800FEFE07000080FA000000060019
:109D00000000FA00C8C2A800C902A800C8E2A80062
:109D1000C922A800A16A20009140780000CEB300BB
:109D200000C060006040B300AAE6B700E16A20000E
:109D30009140780000CEB30000C060006040B300E6
:109D4000AEE6B700816A20009140780000CEB300F3
:109D500000C060009040B300A8E6B700916A200000
:109D60009140780000CEB30000C060000034A00035
:109D7000A9E6B700C16A20009140780000CEB30088
:109D800000C060007040B300ACE6B700D16A2000AC
:109D90009140780000CEB30000C060000034A00005
:109DA000ADE6B700A0B42000104078008080FB0032
:109DB000E081200000804000104078000080FB001F
:109DC00010128800A0B620001040780061406000AA
:109DD000614060004601DD002124200091407800B0
:109DE000F0CBB30000C060000240700042E2B70058
:109DF000A0B62000104078000080FB000000D100D9
:109E00006140600061416000312420009140780091
:109E1000E0CFB30000C060000240700043E2B70032
:109E20000000EB00201288000000EB000012880008
:109E3000A0B42000104078008080FB00E08120006A
:109E400000804000104078000080FB001013880064
:109E5000A0B62000104078006140600061406000C2
:109E60004601DD002126200091407800F0CBB300B0
:109E700000C060000240700062E2B700A0B620009F
:109E8000104078000080FB000000D10061406000BD
:109E9000614160003126200091407800E0CFB3009E
:109EA00000C060000240700063E2B7000000EB00F9
:109EB000201388000000EB00001388000000EB0076
:109EC000401288000000EB00401388004322A900E4
:109ED0006322A9004362A80042A2A9006362A8000D
:109EE00062A2A90040C2A90060C2A9004402A80061
:109EF0006402A8000080FA00000006000000FA00DA
:109F000041E2A9004362A90061E2A9006362A900DD
:109F1000AAC6BF00F041B300AAE6B700AEC6BF00B4
:109F2000F041B300AEE6B700A8C6BF00F041B300F1
:109F3000A8E6B700A9C6BF00F041B300A9E6B70084
:109F4000ACC6BF00F041B300ACE6B700ADC6BF0081
:109F5000F041B300ADE6B7000080FA000000060053
:109F60000000FA00E0A228004C740200000000008B
:109F70000080FA00000006000A00FA00881F78003E
:109F800011C0B300A0B4200001487800A0B62000A2
:109F9000104078000000A100A1B6200080487800A1
:109FA000A0B62000104078000010A000A1B620004C
:109FB00080487800A0B62000104078000020A10062
:109FC000A1B6200080487800C0B52000104078007D
:109FD0000040A000C1B5200080487800A0B4200057
:109FE000104078008080FB0020822000008040002C
:109FF000104078003EFE0700D9FF07000000370040
:10A0000022C2BF00614060000004E000FCFF32009B
:10A01000301180008040780080B620000148780030
:10A0200080B62000104078000080FB004400DE0075
:10A030008040780070B620000148780070B620009B
:10A04000104078000080FB00400798004E00900010
:10A05000E40F5000FB0032004E009000E40F50006F
:10A0600007003C004E0090000000E0000B003200B2
:10A070004E009000E10F5000CC0032005D0137002F
:10A080004E009000E60F5000F60032004E009000A7
:10A09000E80F5000080132005601370080B620005A
:10A0A000104078000080FB00300798003E009000D0
:10A0B000E30F5000270032003E009000E30F5000F5
:10A0C0000A003C003E009000E10F500017003200F3
:10A0D0003E009000E10F500016003C003E00900052
:10A0E0000000E0000F003200AC0037003E0090009E
:10A0F000ED0F50001F0032003E009000ED0F5000A9
:10A1000004003C003E009000E50F5000A3003C001E
:10A11000260037003E009000EE0F50001C00320079
:10A120009E00370046FE0700360137008CFF07000F
:10A13000B3FF370060168000F1FB2F0001006000C4
:10A140006016880010C0B300A8780200000000006C
:10A15000ABFF370060168000010420000100700092
:10A160006016880010C0B300A8780200000000004C
:10A17000A3FF370010C0B300A87802000000000061
:10A180008040EB0010C0B3004FFE07009CFF37007B
:10A1900010C0B300A8780200000000008040EB006F
:10A1A0000040EB0048FE070095FF370022C2BF00C9
:10A1B000614060000004E000FCFF320030118000CC
:10A1C000100798001E0090004800DD00100798005E
:10A1D00022C2BF00614060000004E000FCFF3200CA
:10A1E000301180009E0090000080700010079800E1
:10A1F00022C2BF00614060000004E000FCFF3200AA
:10A2000030118000000F78001E0078004800DD004B
:10A21000000F780022C2BF00614060000004E0002F
:10A22000FCFF3200301180001E0F70009E00900075
:10A2300000002100808F500003003E00000021003C
:10A240009E0F1000040036000040EB00A8780200CA
:10A25000000000006AFF37000000EB0020079800B4
:10A260000C00370022C2BF00614060000004E00023
:10A27000FCFF3200714080002E0090008080400082
:10A2800030118000804878002E0090000000E80027
:10A2900020079800AE0090001E009000808F5000B4
:10A2A000F0FF390080B6200010407800E44F5000E5
:10A2B00001003A00CAC2A9000000EB002007980084
:10A2C00008003700714080002E00900000804000A0
:10A2D00010407800EEFD07002E0090000000E8001E
:10A2E00020079800AE0090001E009000808F500064
:10A2F000F4FF390010002000D69B0200000000008F
:10A300000000EB0020079800090037007140800032
:10A310002E0090000084400000C0EB00DCFD070030
:10A32000004C78002E0090000000E8002007980004
:10A330002E0090009E0F5000F4FF390080B62000E0
:10A3400010407800E44F500001003A00CAC2A80053
:10A3500010C0B300A8780200000000000000EB006D
:10A360002007980009003700714080002E009000FF
:10A370000080400010407800A87802000000000033
:10A380002E0090000000E800200798002E009000AA
:10A390009E0F5000F4FF390019FF37000040EB001A
:10A3A000A87802000000000015FF370080B62000EA
:10A3B00090407800F0C0B30080C0600080B62000FC
:10A3C0000148780080B62000104078008040E80006
:10A3D00080B620000148780010C0B300A8780200C1
:10A3E000000000008040EB0060B6200001487800CB
:10A3F0000D00370022C2BF00614060000004E00091
:10A40000FCFF320030118000A1FD0700A878020097
:10A410000000000060B62000104078008040E80096
:10A4200060B620000148780060B6200090407800B7
:10A4300080B620001040780080CF5000EDFF39003A
:10A44000EFFE370080B620001040780028A10200FF
:10A450000000000010C0B300A87802000000000057
:10A46000E7FE370080B620009040780070C0B3004F
:10A4700080C0600080B620000148780080B62000CF
:10A4800090407800A0B4200001487800A0B42000DB
:10A49000104078008080FB00208220000080400077
:10A4A0001040780012FD070010C0B300A878020029
:10A4B00000000000D2FE3700A0B620001040780057
:10A4C0000000A100A1B6200080487800A0B62000BE
:10A4D000104078000010A100A1B62000804878004C
:10A4E000A0B62000104078000020A100A1B62000F6
:10A4F00080487800C0B52000104078000040A100DE
:10A50000C1B520008048780080B620001040780057
:10A510000080FB004200DE00610060000004E000FB
:10A5200005003200A0B62000104078000000A00016
:10A53000A1B620008048780080B620001040780046
:10A540000080FB000000D100610060000004E0001A
:10A5500005003200A0B62000104078000010A000D6
:10A56000A1B620008048780080B620001040780016
:10A570000080FB00610060000004E0000500320084
:10A58000A0B62000104078000020A000A1B6200056
:10A590008048780080B62000104078000080FB00E2
:10A5A0004300DE000000A200610060000004E00043
:10A5B00005003200C0B52000104078000040A00027
:10A5C000C1B5200080487800A0B420001040780079
:10A5D0008080FB0020822000008040001040780036
:10A5E000C3FC070010C0B300A87802000000000000
:10A5F00083FE37000040EB00A87802000000000056
:10A600007FFE37004F0478000080FA00000006004B
:10A610000400FA0086A00200000000000004E00030
:10A620002200320032C2BF00684060000004E00037
:10A63000040032003100200010CF2000489E0200AC
:10A640000000000032C2BF00644060000004E0006F
:10A65000040032003100200040CF2000489E02005C
:10A660000000000076A0020000000000000F78004B
:10A6700032C2BF00624060000004E0000800320007
:10A68000F100200070CF2000489E02000000000072
:10A6900090118000D1FF2F00010060009011880010
:10A6A0001E0078001007980006003700F100200017
:10A6B00060D02000489E0200000000000000EB0077
:10A6C000100798001E0090000080FA0000000600AD
:10A6D0000200FA00000F78001E00780062A002005D
:10A6E000000000000000EB000080FA0000000600FF
:10A6F0000000FA0001022000C0DB2000489E02009A
:10A7000000000000A0B4200010407800E4760200B1
:10A710000000000000C2B300A878020000000000A2
:10A72000A0B4200010407800E94F500007003A0024
:10A73000C0118000867602000000000000C2B30055
:10A74000A8780200000000000C003700A0B4200030
:10A75000104078000080FB0080004000C0AD200069
:10A7600000804000100078008676020000000000A3
:10A7700000C2B300A878020000000000C0DA200088
:10A780001040780063406000E476020000000000A2
:10A7900000C2B300A878020000000000C0DA200068
:10A7A000104078000080FB004200DE006140600045
:10A7B000E47602000000000000C2B300A8780200A6
:10A7C00000000000C0DA2000104078000080FB008C
:10A7D0004300DE0061406000E476020000000000FB
:10A7E00000C2B300A878020000000000C0B520003D
:10A7F000104078000080FB004400DE0061406000F3
:10A80000E47602000000000000C2B300A878020055
:10A810000000000031002000F0AD2000489E020042
:10A82000000000000080FA00000006000C00FA00A2
:10A830000000EB00000F7800202102000000000063
:10A84000521D020000000000500798005E009000BA
:10A85000EA0F500005003A0020210200000000002D
:10A86000521D020000000000000F780020210200AD
:10A8700000000000521D0200000000004007980088
:10A880002021020000000000521D02000000000014
:10A89000300798002021020000000000521D020035
:10A8A00000000000200798002021020000000000A6
:10A8B000521D020000000000100798005E0090008A
:10A8C0000000E000090034005E009000EA0F500034
:10A8D00006003C005E0090000040E90080407800E7
:10A8E000A0B4200001487800020037000000EB000F
:10A8F000500798004E0090000000E0000F00340068
:10A900004E009000E40F50000C003C004E00900000
:10A910000040E900E3406000C0DA20001040780009
:10A9200063C16000C1CFB30001406000024070000D
:10A93000C1DA200080487800020037000000EB00F8
:10A94000500798003E0090000000E0001000340026
:10A950003E009000E20F50000D003C003E009000D1
:10A960000040E90061416000C0DA200090407800BA
:10A97000614061004201DD00B0CFB30080C06000E3
:10A9800082C07000C0DA2000014878000200370061
:10A990000000EB00500798002E0090000000E0003F
:10A9A000100034002E009000E20F50000D003C001B
:10A9B0002E0090000040E90061416000C0DA2000F4
:10A9C00090407800614061004301DD0070CFB3002A
:10A9D00080C0600082C07000C0DA200001487800AA
:10A9E000020037000000EB00500798001E009000A6
:10A9F0000000E000100034001E009000E20F500044
:10AA00000D003C001E0090000040EA006141600023
:10AA1000C0B5200090407800614061004401DD0035
:10AA2000F0CEB30080C0600082C07000C0B52000CE
:10AA300001487800020037000000EB005007980042
:10AA40005E0090000000E00073003A000000EB00A0
:10AA5000F0678800D108200030872000D29E0200D5
:10AA6000000000008001EB00A20020001100200087
:10AA7000100020004C220200000000000040E9000D
:10AA800080407800A0B4200001487800A0B42000E5
:10AA900010407800E94F50000B003A00C10120003F
:10AAA00050132100D29E0200000000008001EB0044
:10AAB000F2FF270011002000200220004C2202009B
:10AAC00000000000000F78004105200050D1200058
:10AAD000489E0200000000008001EB0042002000C0
:10AAE00011002000100020004C2202000000000095
:10AAF0000040E900E3406000C0DA20001040780028
:10AB000063C16000C1CFB30001406000024070002B
:10AB1000C1DA2000804878001102200090D6200081
:10AB2000489E0200000000008001EB00220020008F
:10AB300011002000100020004C2202000000000044
:10AB40000040E90061416000C0DA200090407800D8
:10AB5000614061004201DD00B0CFB30080C0600001
:10AB600082C07000C0DA2000014878002103200074
:10AB7000A0D82000489E0200000000008001EB00E9
:10AB80002200200011002000100020004C220200B2
:10AB9000000000000040E90061416000C0DA2000D0
:10ABA00090407800614061004301DD0070CFB30048
:10ABB00080C0600082C07000C0DA200001487800C8
:10ABC000F1042000B0932000D29E0200000000009B
:10ABD0008001EB0022002000110020001000200066
:10ABE0004C220200000000000040EA0061416000C9
:10ABF000C0B5200090407800614061004401DD0054
:10AC0000F0CEB30080C0600082C07000C0B52000EC
:10AC10000148780001003700B5FE0700A0B420000D
:10AC200010407800E94F50001C003A00C0DA2000C4
:10AC3000104078000080FB004200DE0061406000B0
:10AC400080417800C0DA2000104078006340600046
:10AC500080427800C0DA2000104078000080FB00BD
:10AC60004300DE006140600000417800C0B5200074
:10AC7000104078000080FB004400DE00614060006E
:10AC8000804078001E0078000342780085417800FB
:10AC9000B69F02000000000022003700C0DA20004A
:10ACA000104078000080FB004200DE006140600040
:10ACB00000417800C0DA2000104078006340600056
:10ACC00080417800C0DA2000104078000080FB004E
:10ACD0004300DE006140600080427800C0B5200083
:10ACE000104078000080FB004400DE0061406000FE
:10ACF00000437800A0B42000104078000080FB00E2
:10AD000080004000C0AD20000080400010007800AE
:10AD1000024278000541780086407800B69F020024
:10AD200000000000C0DA200010407800634060009E
:10AD3000E34F500003003A0091C0B300B0B42000CC
:10AD4000014878003AA0020000000000C111800014
:10AD500040118000808F500004003100010220006B
:10AD600010152100D29E0200000000000080FA00B1
:10AD7000000006000000FA0046A0020000000000EB
:10AD80000080FA00000006000400FA00000F7800BE
:10AD90001E007800100798001E009000E10F500080
:10ADA0000C0032001E009000E10F5000040039003A
:10ADB0001E009000E20F50003D00320059003700A5
:10ADC00031052000C0DD2000489E02000000000088
:10ADD00058003700B1002000F0E22000D29E0200AF
:10ADE00000000000D1002000A0E32000D29E02005D
:10ADF00000000000789F0200000000000000E0005A
:10AE00004C00320090118000D1FF2F000100600043
:10AE1000901188000000370032C2BF00614060001E
:10AE20000004E0000600320023C2BF006240600060
:10AE30000004E00002003A00B011800020118800F8
:10AE400022C2BF00614060000004E0000600320042
:10AE500033C2BF00624060000004E00002003A001C
:10AE600030118000A011880032C2BF006240600033
:10AE70000004E00004003A0022C2BF00624060000B
:10AE80000004E000E4FF320091118000D0FF2F00A9
:10AE9000008060009011880011118000D0FF2F0009
:10AEA0000080600010118800CA82A900DAFF370014
:10AEB000E100200070E42000D29E020000000000AB
:10AEC000F100200010172100D29E020000000000B7
:10AED00090118000D1FF2F000100600090118800C8
:10AEE00032C2BF00614060000004E0000600320092
:10AEF00023C2BF00624060000004E00002003A008C
:10AF0000B01180002011880022C2BF0061406000A3
:10AF10000004E000F2FF320030118000000F7800E2
:10AF20000400370041022000C0202000D29E020011
:10AF3000000000000080FA00000006000000FA0097
:10AF400091118000D0FF2F000080600090118800D8
:10AF5000C0DA2000104078000040A000C1DA2000D4
:10AF600080487800C0B52000104078000020A00084
:10AF7000C1B5200080487800C101200050E52000C4
:10AF8000D29E0200000000000080FA0000000600CF
:10AF90000000FA00C0DA2000104078000040A10054
:10AFA000C1DA200080487800C0B520001040780049
:10AFB0000020A100C1B52000804878004101200098
:10AFC00010E72000D29E0200000000000080FA007E
:10AFD000000006000200FA000000EB00000F7800FD
:10AFE00034003700C0DA2000104078007040600064
:10AFF0000004E0002B00320060A6280078740200F4
:10B00000000000006100200060692000489E0200EE
:10B010000000000032C2BF00684060000004E00091
:10B02000040032003100200010CF2000489E0200B2
:10B030000000000032C2BF00644060000004E00075
:10B04000040032003100200040CF2000489E020062
:10B050000000000076A0020000000000049B020037
:10B060000000000032C2BF00624060000004E00047
:10B0700008003200F100200070CF2000489E02003E
:10B080000000000090118000D1FF2F00010060003F
:10B090009011880060A6280078740200000000006B
:10B0A0000200370076A0020000000000100020001F
:10B0B000000F780086A00200000000000004E000FD
:10B0C000C8FF3A001E0078000080FA000000060069
:10B0D0000000FA00B100200010092100D29E0200F9
:10B0E000000000000080FA00000006000000FA00E6
:10B0F00070A628004C740200000000000080FA00D6
:10B10000000006000400FA00C0DA200010407800B9
:10B110000000A1000010A100C1DA200080487800E2
:10B12000C0DA2000104078000020A100C1DA200021
:10B1300080487800C0DA2000104078000030A1007C
:10B14000C1DA200080487800C0B5200010407800A7
:10B150000040A000C1B520008048780080578000E2
:10B16000306D8800C0DA2000104078000040A10057
:10B17000C1DA200080487800C0DA20001040780052
:10B180000080FB004200DE006140600080417800EA
:10B19000C0DA2000104078006340600080427800F0
:10B1A000C0DA2000104078000080FB004300DE0081
:10B1B0006140600000417800C0B520001040780078
:10B1C0000080FB004400DE006140600080407800A9
:10B1D000306D80000342780085417800B69F020000
:10B1E000000000003AA0020000000000BFFF0700BE
:10B1F0000000370086A00200000000000004E0000C
:10B200000C003200C0DA200010407800704060006E
:10B210000004E0000500320076A0020000000000FB
:10B22000A8780200000000000200370076A00200AB
:10B230000000000032C2BF00624060000004E00075
:10B240000400320090118000D1FF2F000100600047
:10B250009011880022C2BF00614060000004E0003D
:10B26000E4FF32003011800080407800A0DA200036
:10B2700001487800A0DA2000104078000080FB0030
:10B280004400DE008040780090DA20000148780019
:10B2900090DA2000104078000080FB001007980032
:10B2A0001E009000E40F5000D00032009E0090007D
:10B2B000E48F500007003C001E0090000000E000FA
:10B2C0000F0032009E009000E18F50009F0032007E
:10B2D0008A0137001E009000E60F5000CB003200BC
:10B2E0009E009000E68F5000840135009E00900083
:10B2F00068805000E10F500080013E00FB003700E5
:10B30000A0DA2000104078000080FB00000F7800D9
:10B310001E007800E20F5000190032009E007800F5
:10B32000E28F500007003C001E0078000000E000A3
:10B330000E0032009E007800E18F50000E003200B7
:10B340007E0037001E007800E70F50002600320014
:10B350009E007800EF8F50005B0032001E007800E6
:10B36000E30F5000170032007400370046A00200BF
:10B3700000000000650137005CFF07009DFF3700FB
:10B3800010C0B300A87802000000000032C2BF0065
:10B39000624060000004E000040032009011800070
:10B3A000D1FF2F000100600090118800C0DA20005A
:10B3B000104078000040A000C1DA200080487800EA
:10B3C0008CFF3700C0DA2000104078000040A10058
:10B3D000C1DA20008048780010C0B300A8780200CD
:10B3E0000000000083FF370010C0B300A8780200FF
:10B3F0000000000046A002000000000022C2BF00C2
:10B40000614060000004E000FCFF32003011800069
:10B410004800DD00306D880010C0B300A87802003D
:10B420000000000022C2BF00614060000004E00094
:10B43000FCFF3200316D8000301180000080700010
:10B44000306D8800C0DA2000104078000080FB00DA
:10B450004200DE006140600080417800C0DA2000D8
:10B46000104078006340600080427800C0DA20001D
:10B47000104078000080FB004300DE006140600067
:10B4800000417800C0B52000104078000080FB002B
:10B490004400DE006140600080407800306D800034
:10B4A0000342780085417800B69F0200000000004A
:10B4B0003AA002000000000010C0B300A87802000B
:10B4C000000000004BFF370010C0B300A878020056
:10B4D0000000000090118000D1FF2F0001006000EB
:10B4E000901188000000370032C2BF006140600048
:10B4F0000004E0000600320023C2BF00624060008A
:10B500000004E00002003A00B01180002011880021
:10B5100022C2BF00614060000004E000F2FF320080
:10B5200033C2BF00624060000004E000EEFF3A005A
:10B5300030118000A0118800EBFF37000040EB00C5
:10B54000A8780200000000002AFF3700A0DA2000DF
:10B5500090407800F0C0B30080C06000A0DA200006
:10B5600001487800A0DA2000104078008040E80010
:10B57000A0DA20000148780010C0B300A8780200CB
:10B58000000000008040EB0080DA200001487800D5
:10B590000F00370022C2BF00614060000004E000DD
:10B5A000FCFF32003011800062A0020000000000A9
:10B5B00010C0B300A87802000000000080DA20006C
:10B5C000104078008040E80080DA200001487800D0
:10B5D00080DA200090407800A0DA20001040780047
:10B5E00080CF5000EBFF390002FF3700A0DA2000C7
:10B5F0001040780028A102000000000010C0B30035
:10B60000A878020000000000FAFE3700A0DA20004F
:10B6100090407800F0C0B30080C06000A0DA200045
:10B6200001487800A0DA200010407800EA4F50006E
:10B6300003003600A1C0B300A0DA20000148780062
:10B64000A0DA2000104078000080FB00800040005D
:10B6500000AF20000080400010007800306D8800AE
:10B6600046A0020000000000C0DA20001040780070
:10B670000080FB004200DE006140600080417800F5
:10B68000C0DA2000104078006340600080427800FB
:10B69000C0DA2000104078000080FB004300DE008C
:10B6A0006140600000417800C0B520001040780083
:10B6B0000080FB004400DE006140600080407800B4
:10B6C000306D80000342780085417800B69F02000B
:10B6D000000000003AA002000000000010C0B3000B
:10B6E000A878020000000000C2FE3700C0DA200087
:10B6F000104078000000A1000010A100C1DA200075
:10B7000080487800C0DA2000104078000020A100B6
:10B71000C1DA200080487800C0DA200010407800AC
:10B720000030A100C1DA200080487800C0B52000B8
:10B73000104078000040A100C1B52000804878008A
:10B74000A0DA2000104078000080FB004300DE00FB
:10B75000610060000004E0000D003200C0DA20004B
:10B7600010407800634060000014A000E3406000D7
:10B77000C0DA20001040780063C16000C1CFB30080
:10B780000140600002407000C1DA2000804878006B
:10B79000A0DA2000104078000080FB004200DE00AC
:10B7A000610060000004E0000D003200C0DA2000FB
:10B7B00010407800634060000004A000E340600097
:10B7C000C0DA20001040780063C16000C1CFB30030
:10B7D0000140600002407000C1DA2000804878001B
:10B7E000A0DA2000104078000080FB000000D100AB
:10B7F000610060000004E00005003200C0DA2000B3
:10B80000104078000020A000C1DA200080487800B5
:10B81000A0DA2000104078000080FB00610060008A
:10B820000004E00005003200C0DA2000104078007B
:10B830000030A000C1DA200080487800A0DA2000A3
:10B84000104078000080FB004400DE000000A200F1
:10B85000610060000004E00005003200C0B5200077
:10B86000104078000040A000C1B52000804878005A
:10B8700046A0020000000000C0DA2000104078005E
:10B880000080FB004200DE006140600080417800E3
:10B89000C0DA2000104078006340600080427800E9
:10B8A000C0DA2000104078000080FB004300DE007A
:10B8B0006140600000417800C0B520001040780071
:10B8C0000080FB004400DE006140600080407800A2
:10B8D000306D80000342780085417800B69F0200F9
:10B8E000000000003AA002000000000010C0B300F9
:10B8F000A8780200000000003EFE37000040EB0088
:10B90000A8780200000000003AFE37000080FA002C
:10B91000000006000000FA00729D02000000000016
:10B920000080FB000080FA00000006000200FA0020
:10B93000000F78001E007800DA9C02000000000072
:10B94000001020000080FA00000006000000FA004D
:10B95000D89D0200000000000080FB000080FA007B
:10B96000000006000000FA0080B7200010407800B8
:10B97000389D0200000000000080FA000000060070
:10B980000000FA0080B72000104078000080FB0023
:10B990000080FA00000006000000FA008040EB0082
:10B9A00080B720000148780041022000B00020004C
:10B9B000D29E0200000000000080FA000000060095
:10B9C0000000FA0011C0B30080B7200001487800E1
:10B9D00041022000B0002000D29E020000000000C2
:10B9E0000080FA00000006000000FA00C0B5200048
:10B9F000104078000040A000C1B5200080487800C9
:10BA00008040EB00A0B8200001487800C922A800BF
:10BA1000CB22A900E1022000F0022000D29E020009
:10BA2000000000000080FA00000006000400FA0098
:10BA3000881F7800000F78001E00E00044003200EC
:10BA4000200320009E0F100041003E001E0FE90061
:10BA5000A0B82000104078000080FB009E0F50002E
:10BA600005003E0091022000D0052000D29E020079
:10BA70000000000063013700E100200060082000A2
:10BA8000489E0200000000001E0078000040E80010
:10BA9000E47602000000000020A428004C7402009C
:10BAA000000000008040EB0040B820000148780012
:10BAB0001F0037001E01780040B8200010407800B9
:10BAC0008080FB004310DD0081004000B0B8200002
:10BAD00000804000104078000080FB00049B0200C2
:10BAE0000000000000C2B300A878020000000000BF
:10BAF0001E01780040B82000104078008080FB00D4
:10BB00004310DD0081004000B0B8200000804000FC
:10BB100010407800DA9C02000000000040B82000CD
:10BB2000104078008040E80040B8200001487800CC
:10BB300040B8200010407800E74F5000DDFF36008D
:10BB400050A4280078740200000000002D01370086
:10BB50001E00780010079800500520009E009000FD
:10BB6000808F500011013200500520009E0090008F
:10BB7000808F500008003E001E0090000000E00092
:10BB800012003200300320009E009000808F500091
:10BB9000DD00320017013700C00E20009E0090002B
:10BBA000808F500063003200000F20009E00900044
:10BBB000808F50005F003200C00C20009E0090007B
:10BBC000808F5000020132000A013700D1002000AE
:10BBD00040092000D29E02000000000071012000F8
:10BBE000100A2000D29E020000000000A0B8200031
:10BBF000104078000004E00005003A0091022000A7
:10BC0000D0052000D29E0200000000004400370052
:10BC10008040EB0050B82000014878003A0037001F
:10BC200000C2B300A87802000000000050B8200055
:10BC3000104078000040E800E476020000000000B8
:10BC400060A428004C740200000000008040EB005B
:10BC500040B82000014878001600370050B8200096
:10BC6000104078000081FB0040B8200010407800B0
:10BC70008080FB004310DD0081004000B0B8200050
:10BC800000804000104078000080FB00049B020010
:10BC90000000000000C2B300A8780200000000000D
:10BCA00040B82000104078008040E80040B82000F4
:10BCB0000148780040B8200010407800E74F50005D
:10BCC000E6FF360061002000800B2000489E020045
:10BCD0000000000050B82000104078000080FB00F9
:10BCE000C300DD00B0B820000080400010407800A4
:10BCF000F700070050B82000104078008040E800AE
:10BD000050B8200001487800A0B82000904078008A
:10BD100050B820001040780080CF5000C0FF3E0097
:10BD2000310D2000E00B2000D29E02000000000038
:10BD3000B40037001E00780080407800C0832000E7
:10BD400001487800C00E20009E0F100005003A0048
:10BD50003101200010192000D29E020000000000D6
:10BD600004003700D1002000401A2000D29E0200BB
:10BD70000000000071012000100A2000D29E020085
:10BD8000000000008040EB0040B82000014878002F
:10BD90000A0107008040780050B820000148780070
:10BDA0008040EB00A0B82000014878004D0037002B
:10BDB00000C2B300A87802000000000040B82000D4
:10BDC000104078000040E800E47602000000000027
:10BDD00060A428004C740200000000000000EB008A
:10BDE000105C88000D003700115C8000B0BD2000A1
:10BDF00000804000104078000080FB00049B02009F
:10BE00000000000000C2B300A8780200000000009B
:10BE1000105C80000000E800105C8800105C80006E
:10BE2000E70F5000F0FF360061002000800B20007B
:10BE3000489E020000000000B0BD200010407800C5
:10BE4000A300070040B8200010407800E94F5000E0
:10BE50001B003E000000EB00105C88001000370063
:10BE6000A0B82000104078008081FB00145C8000A6
:10BE7000115C8000B0BD20000080400010417800BF
:10BE80004318DD0084004000B0B82000008040006E
:10BE900002487800105C80000000E800105C880018
:10BEA000105C8000E70F5000EDFF3600A0B82000C6
:10BEB000104078008040E800A0B8200001487800D9
:10BEC00040B82000104078008040E80040B82000D2
:10BED00001487800C70007008040780050B8200073
:10BEE0000148780050B82000104078000004E000BD
:10BEF000AFFF3A00B1022000101B2000D29E0200CA
:10BF0000000000003F00370048000700110120003A
:10BF1000C01D2000489E02000000000030C3B30096
:10BF2000DA9C0200000000000000EB00105C8800BA
:10BF300014003700185C8000729D020000000000B1
:10BF40008040780090B7200000004400014878004D
:10BF5000115C800090B72000008040001040780005
:10BF60000080FB00049B02000000000000C2B30040
:10BF7000A878020000000000105C80000000E800CB
:10BF8000105C8800105C8000E70F5000E9FF36006D
:10BF900050A42800787402000000000090B7200030
:10BFA000104078004A000700160037001F00070005
:10BFB00001012000D01E2000D29E020000000000DF
:10BFC00050C5B300DA9C0200000000000D003700ED
:10BFD00016000700F1002000D01F2000D29E0200B2
:10BFE00000000000C0CCB300DA9C0200000000009A
:10BFF0000400370041022000C0202000D29E020031
:10C00000000000004F0478000080FA0000000600E5
:10C010000000FA009100200080082100D29E02005A
:10C02000000000000080FA00000006000200FA0094
:10C03000549C020000000000004F7800A100200086
:10C0400000232000489E0200000000001E04E000C3
:10C0500005003A003100200050BB2000D29E0200B3
:10C06000000000001800370091002000A0232000ED
:10C07000489E0200000000001E80FB00610060007E
:10C080000004E000040032005101200030242000B0
:10C09000489E0200000000001E80FB000000D1004E
:10C0A000610060000004E000040032004101200053
:10C0B00080252000489E02000000000050A42800B7
:10C0C00078740200000000000080FA000000060002
:10C0D0000400FA00004F78001E80FB001007980053
:10C0E000200220009E009000808F50001E00320031
:10C0F000200220009E009000808F500007003C002E
:10C100001E009000E40F50001C0032009E009000C2
:10C11000F08F50000A003200220037008002200019
:10C120009E009000808F50000A003200D002200054
:10C130009E009000808F50001500320019003700DB
:10C14000B1012000C0262000D29E020000000000A5
:10C1500018003700A101200070282000D29E0200A4
:10C16000000000001300370051012000102A2000B9
:10C17000D29E0200000000000E0037008101200066
:10C18000602B2000D29E0200000000000900370052
:10C1900001012000E02C2000D29E020000000000DF
:10C1A00004003700E1002000E02D2000489E02003E
:10C1B000000000000080FA00000006000000FA0005
:10C1C0008040EB0030BE2000014878008040EB004A
:10C1D00050BE2000014878008040EB0040BE2000A7
:10C1E00001487800080007000080FB000080FA008A
:10C1F000000006000000FA00030007000080FB00BA
:10C200000080FA00000006000A00FA0010C0B30027
:10C21000704798000040EB00604798000040EB003A
:10C220005047980010C0B300104798000040EB0042
:10C23000404798008040EB0060BE20000148780035
:10C2400050BE2000104078000004E0009C003A003E
:10C25000549C0200000000000004E0000C003200CA
:10C260008040EB0030BE2000014878008040EB00A9
:10C2700050BE2000014878008040EB0040BE200006
:10C28000014878000000EB0040079800A10037004B
:10C29000C083200010407800DA9C020000000000FB
:10C2A000D89D02000000000030479800D89D020091
:10C2B00000000000204798003E409000E14F5000F1
:10C2C00003003A002E409000E14F50006800320019
:10C2D000BE4090002E40900080CF500003003200FE
:10C2E000BE409000014F78002600370030BE20008D
:10C2F000904078007E409000814F50000E00310049
:10C300005E4090008080FB00B0BD200000804000B7
:10C31000904078001E40900080C060000040EB001C
:10C32000004F78000104E0000C00320010C0B300A0
:10C33000004F78000900370030BE200090407800A0
:10C340000040EB00004F78007E409000814F50008D
:10C3500002003A0010C0B300004F78001E04E00055
:10C3600008003A007E409000604798006E409000C0
:10C37000E84F500003003E0040BE2000EE40900019
:10C380000148780010C0B3009E4F10000D003A0025
:10C390005E4090000081FB005E4090008080FB00CA
:10C3A000B0BD200000804000904078001E4090000A
:10C3B00080C07000B0BD200000004100014878003E
:10C3C000110037005E4090000082FB005E4090004C
:10C3D0008080FB00B0BD200000804000104078004D
:10C3E000804178001E419000024078000080EA0001
:10C3F0008180EA0000C0610080407800B0BD20006C
:10C4000000004200014878001E407800389D02007C
:10C41000000000007E4090000040E8007047980057
:10C420001E40900000404000104798001E409000C1
:10C430000004E0000B003A005E4090008080FB00AA
:10C44000B0BD20000080400010407800920007003E
:10C450005E4090000040E8005047980010C0B300D4
:10C46000104798005E409000E74F50008CFF360068
:10C47000FE40900000C4B30080CF50001000360092
:10C4800060BE2000104078000004E0000C003A007C
:10C4900030BE2000EE4090000148780030BE200001
:10C4A000104078000004E00003003A0011C0B3001F
:10C4B00050BE20000148780010C0B30040479800EB
:10C4C0004E4090000004E00004003200B0BD2000A7
:10C4D000104078000004E0000B003A008040EB00C0
:10C4E00030BE2000014878008040EB0050BE2000A4
:10C4F000014878008040EB0040BE200001487800F1
:10C500000040EB00404798004E4090000080FB0048
:10C51000400798004E0090000080FA0000000600DE
:10C520000E00FA000040EB00404798000C00370076
:10C530004E4090000081FB004E4090008080FB0048
:10C54000B0BD2000008040009040780065004700AA
:10C55000017178004E4090000040E800404798008C
:10C560004E409000E74F5000F1FF360030BE2000F3
:10C57000904078002147980050BE200090407800FD
:10C580001147980040BE2000104F780001C4B3004E
:10C5900030BE2000014878008040EB0050BE2000F3
:10C5A0000148780018FF07000004E0001A0032007C
:10C5B00010C0B300304798000040EB00404798009F
:10C5C000110037004E4090008080FB00650047005E
:10C5D000614178004E4090008080FB00B0BD20009B
:10C5E0000080400010407800804F5100030032006E
:10C5F0000040EB0030479800090037004E409000A3
:10C600000040E800404798004E409000E74F50003F
:10C61000ECFF3600020037000040EB003047980086
:10C620000040EB00404798000C0037004E4090005F
:10C630000081FB004E4090008080FB0065004700B9
:10C64000E1407800B0BD20000000410001487800C2
:10C650004E4090000040E800404798004E40900057
:10C66000E74F5000F1FF360030BE2000AE40900092
:10C670000148780050BE20009E409000014878009C
:10C6800040BE20001E4878003E4090000080FB0025
:10C690000080FA00000006000200FA00004F780057
:10C6A00060BE2000104078001E4068008080FB00C3
:10C6B000D0832000008040009040780060BE2000C1
:10C6C0000148780060BE2000104078000080FB0028
:10C6D0000080FA00000006000000FA0080A4280094
:10C6E0004C740200000000000080FA000000060008
:10C6F0000400FA00C922A800CB22A900C8C2A900E0
:10C70000C0B52000104078000040A000C1B5200056
:10C7100080487800C0B52000104078000030A100AB
:10C72000C1B5200080487800EBFF0700000037000B
:10C7300022C2BF00614060000004E000FCFF320044
:10C74000301180008040780090B8200001487800C7
:10C7500090B82000104078000080FB004400DE000C
:10C760008040780080B820000148780080B8200020
:10C77000104078000080FB00100798001E00900019
:10C78000E10F5000780032009E009000E48F5000CE
:10C790009D0032001E0090000000E0000100320009
:10C7A000A100370090B82000104078000080FB0006
:10C7B000000F78009E007800E28F500017003200D2
:10C7C0001E007800E20F500007003C009E00780039
:10C7D0000100E000980032001E007800E10F5000D8
:10C7E0000C0032005C0037009E007800E48F50009F
:10C7F000130032001E007800E40F50005600350090
:10C800009E00780068805000E10F500052003E000A
:10C8100010003700B0FF0700C5FF3700549C02002E
:10C82000000000008040780060B8200001487800D7
:10C8300010C0B300A878020000000000BCFF370061
:10C84000729D020000000000A878020000000000B5
:10C85000B7FF370010C0B300A87802000000000046
:10C8600090B8200010407800E94F500004003A00D2
:10C87000C1CEB300C0832000014878000300370018
:10C8800001CFB300C0832000014878004BFE0700B1
:10C890008040780060B82000014878001900370017
:10C8A0008040EB0070B82000014878000D00370090
:10C8B00070B82000104078008080FB00B0BD2000E0
:10C8C0000080400010407800A878020000000000BE
:10C8D00070B82000104078008040E80070B8200058
:10C8E0000148780070B8200010407800E74F5000F1
:10C8F000EFFF36003FFE07008040780060B8200060
:10C900000148780060B82000104078000004E00082
:10C91000E3FF3A008040EB0070B820000148780047
:10C920000800370000C0EB00A878020000000000FB
:10C9300070B82000104078008040E80070B82000F7
:10C940000148780070B8200010407800E74F500090
:10C95000F4FF360076FF37000040EB00A8780200B5
:10C960000000000072FF370090B82000904078006F
:10C97000F0C0B30080C0600090B82000014878008B
:10C9800090B82000104078008040E80090B8200067
:10C990000148780010C0B300A87802000000000031
:10C9A0008040EB0070B82000014878000F0037008D
:10C9B00022C2BF00614060000004E000FCFF3200C2
:10C9C00030118000DA9C02000000000010C0B300AB
:10C9D000A87802000000000070B820001040780025
:10C9E0008040E80070B820000148780070B820004E
:10C9F0009040780090B820001040780080CF500020
:10CA0000EBFF39004AFF370090B820001040780053
:10CA100028A102000000000010C0B300A8780200A6
:10CA20000000000042FF37000040EB00A878020041
:10CA3000000000003EFF37000080FA000000060002
:10CA40000000FA0020A728004C740200000000003B
:10CA50000080FA00000006000000FA000040EB0031
:10CA600096850200000000000040EB009685020061
:10CA7000000000000040EB0096850200000000006E
:10CA80000040EB0096850200000000000000EB0073
:10CA9000D2840200000000000000EB00D2840200FB
:10CAA000000000000000EB00D28402000000000043
:10CAB0000080FA00000006000C00FA00C0B520005B
:10CAC000104078000040A000C1B5200080487800E8
:10CAD000C0B52000104078000030A100C1B5200092
:10CAE0008048780011C0B300A0B42000014878004D
:10CAF00081C0B300B0B420000148780021C0B30069
:10CB0000F0DB20000148780080C0EB0020C0B300BB
:10CB10007283020000000000C922A900C902A90016
:10CB2000C8E2A80010C0B3000286020000000000A6
:10CB3000C3FF07000000370022C2BF006140600051
:10CB40000004E000FCFF32003011800080407800DB
:10CB500030DC20000148780030DC200010407800F4
:10CB60000080FB004400DE008040780020DC2000D4
:10CB70000148780020DC2000104078000080FB0095
:10CB8000300798003E009000E30F5000170132007C
:10CB9000BE009000E38F50000A003C003E01900070
:10CBA000E10F5100A5003200BE019000E18F51005D
:10CBB000FB003C003E0090000000E000120032004C
:10CBC000E8023700BE009000E68F5000910232006C
:10CBD0003E019000E60F510004003C00BE019000B1
:10CBE000E48F510083023200DE0237003E009000E5
:10CBF000E80F50009E023200BE009000EA8F500005
:10CC000034013200D702370030DC200010407800B9
:10CC10000080FB006101B9004207980053079800AB
:10CC2000D0002000010020004E019000DE019000A5
:10CC3000800F5100818F59007C003E004E00900013
:10CC4000DE00900000600100CA0237000C003700CF
:10CC50000D00370012003700170037001D003700A5
:10CC60002300370044003700480037004C003700ED
:10CC700052003700580037005E003700640037006C
:10CC80006FFF0700ACFF37000084020000000000C7
:10CC900010C0B300A878020000000000A6FF370013
:10CCA000408402000000000010C0B300A878020019
:10CCB00000000000A0FF37000040EB0002860200E9
:10CCC0000000000010C0B300A878020000000000BF
:10CCD00099FF370010C0B300028602000000000078
:10CCE00010C0B300A87802000000000092FF3700D7
:10CCF000F0DB200010407800E24F500006003A00C0
:10CD000026850200000000008040780010DC200032
:10CD10000148780006003700F00F20006084020010
:10CD2000000000008040780010DC200001487800FE
:10CD3000C0B5200010407800684060000004E000AA
:10CD40000800320010DC2000104078000080FB005A
:10CD50000C9C0200000000008040780010DC2000E5
:10CD60000148780010DC200010407800A87802000C
:10CD70000000000070FF3700748502000000000012
:10CD8000A8780200000000006BFF37001486020044
:10CD900000000000A87802000000000066FF3700D5
:10CDA00010C0B300B88502000000000010C0B3003E
:10CDB000A8780200000000005FFF37000040EB0091
:10CDC000F08502000000000010C0B300A878020047
:10CDD0000000000058FF370010C0B300F0850200CB
:10CDE0000000000010C0B300A8780200000000009E
:10CDF00051FF37000040EB00DE850200000000001C
:10CE000010C0B300A8780200000000004AFF3700FD
:10CE100010C0B300DE8502000000000010C0B300A7
:10CE2000A87802000000000043FF37000040EB003C
:10CE3000A8780200000000003FFF370030DC20002F
:10CE400090407800F0C0B30080C0600030DC20006B
:10CE50000148780030DC2000104078008040E80075
:10CE600030DC20000148780010C0B300A878020030
:10CE7000000000008040EB0010DC2000014878003A
:10CE80004000370022C2BF00614060000004E000A3
:10CE9000FCFF3200301180008040780000DC200070
:10CEA00001487800C0B5200010407800684060005C
:10CEB0000004E0000800320000DC20001040780090
:10CEC0000080FB000C9C0200000000008040780005
:10CED00000DC200001487800F0DB200010407800E2
:10CEE000E24F500009003A0000DC200010407800BA
:10CEF0000080FB00D28402000000000010C0B300DC
:10CF0000A8780200000000001900370000DC2000B3
:10CF1000104078000080FB006084020000000000E8
:10CF20008040780000DC200001487800C0B5200077
:10CF300010407800684060000004E0000800320003
:10CF400000DC2000104078000080FB000C9C0200F8
:10CF5000000000008040780000DC200001487800DC
:10CF600000DC200010407800A878020000000000DB
:10CF700010DC2000104078008040E80010DC200029
:10CF80000148780010DC20009040780030DC200060
:10CF90001040780080CF5000BAFF3900E6FE37001D
:10CFA00030DC200090407800F0C0B30080C060000A
:10CFB00030DC20000148780030DC20001040780090
:10CFC0008040E80030DC20000148780030DC2000A0
:10CFD00010407800B88502000000000010C0B300C7
:10CFE000A878020000000000D3FE370030DC2000EB
:10CFF00090407800F0C0B30080C0600030DC2000BA
:10D000000148780030DC2000104078008040E800C3
:10D0100030DC20000148780010C0B300A87802007E
:10D020000000000022C2BF00614060000004E00078
:10D03000FCFF3200301180008040780020DC2000AE
:10D04000014878008040EB0010DC200001487800A7
:10D050001600370020DC2000104078000004E000BB
:10D0600004003D0010C0B3009685020000000000DF
:10D07000030037000040EB0096850200000000002E
:10D0800020DC200010407800004040008040780004
:10D0900020DC20000148780010DC200010407800DF
:10D0A0008040E80010DC20000148780010DC2000FF
:10D0B0009040780030DC20001040780080CF500095
:10D0C000E4FF390010C0B300A8780200000000009F
:10D0D00099FE370030DC2000104078000080FB0013
:10D0E00020079800400A2000AE009000808F50007A
:10D0F00015003200500A20002E019000800F5100D0
:10D10000C5003200000A2000AE019000808F51005F
:10D11000010032003301370022C2BF0061406000CD
:10D120000004E000FCFF32003011800080407800F5
:10D13000E0DB20000148780010C0B300A8780200AE
:10D14000000000007CFE3700E0DB2000104078008B
:10D150000080FB00100798001E009000E10F5000B7
:10D16000040032009E009000E28F50003B0032002D
:10D17000A500370022C2BF00614060000004E0004B
:10D18000FCFF320030118000E06D8800E06D80000F
:10D190006300B900E06D88000000EB00D06D8800EE
:10D1A0000C00370022C2BF00614060000004E000B4
:10D1B000FCFF320071408000D06D80008080400014
:10D1C0003011800080487800D06D80000000E800B9
:10D1D000D06D8800D16D8000E06D8000808F5000A0
:10D1E000F0FF39000000EB00D06D8800130037001D
:10D1F00071408000D06D8000008040000080E80019
:10D200001041780071408000D06D800000804000A7
:10D210000000E8009041780071408000D06D8000EF
:10D2200000804000104078008340780053010700E0
:10D23000D06D800063004000D06D8800D16D80000B
:10D24000E06D8000808F5000E9FF390010C0B3000E
:10D25000A87802000000000037FE370022C2BF009D
:10D26000614060000004E000FCFF320030118000EB
:10D27000E06D8800E06D80004200DD00E06D880018
:10D280000000EB00D06D88000C00370022C2BF0008
:10D29000614060000004E000FCFF3200714080004B
:10D2A000D06D800080804000301180008048780080
:10D2B000D06D80000000E800D06D8800D16D800046
:10D2C000E06D8000808F5000F0FF39000000EB001F
:10D2D000D06D8800440037000040EB0096850200C6
:10D2E000000000000040EB009685020000000000F6
:10D2F0000040EB0096850200000000000040EB00BB
:10D30000968502000000000071408000D06D800012
:10D3100000804000104078000080FB00D2840200B2
:10D320000000000071408000D06D8000008040004F
:10D330000000E800104078000080FB00D28402006A
:10D340000000000071408000D06D8000008040002F
:10D350000080E800104078000080FB00D2840200CA
:10D360000000000071408000D06D8000008040000F
:10D370006301400071408000D06D8000008040005B
:10D3800063004000104078006F4060000049780062
:10D390008040EB0010DC20000148780006003700D8
:10D3A000ADFD070010DC2000104078008040E80050
:10D3B00010DC20000148780071408000D06D8000B2
:10D3C00000804000630040009040780010DC2000A6
:10D3D0001040780080CF5000F1FF3E00D06D8000FB
:10D3E00064004000D06D8800D16D8000E06D800049
:10D3F000808F5000B8FF390010C0B300A878020039
:10D4000000000000CCFD37000040EB00A8780200CF
:10D4100000000000C8FD3700E0DB2000104078006D
:10D420000080FB00000F78001E017800E10F510022
:10D43000040032009E017800E28F51004500320066
:10D44000BDFD370022C2BF00614060000004E00063
:10D45000FCFF320030118000E06D880022C2BF0066
:10D46000614060000004E000FCFF320030118000E9
:10D470008040780020DC2000014878000000EB00AC
:10D48000D06D88002E00370020DC2000904078000E
:10D4900000DC2000014878008040EB0010DC200018
:10D4A000014878001900370000DC200010407800A7
:10D4B0000080FB00610060000004E0000400320016
:10D4C00010C0B30096850200000000000300370082
:10D4D0000040EB00968502000000000000DC200008
:10D4E000104078000080FB000000D10080407800F0
:10D4F00000DC20000148780010DC2000104078009B
:10D500008040E80010DC20000148780010DC20009A
:10D5100010407800E34F5000E3FF360026850200FC
:10D52000000000002685020000000000A87802002C
:10D5300000000000D06D80000000E800D06D880081
:10D54000D16D8000E06D8000808F5000CEFF3900EB
:10D5500079FD370022C2BF00614060000004E00096
:10D56000FCFF320030118000E06D88000000EB000D
:10D57000D06D88001600370022C0B30060B92000CB
:10D58000A10B2000B7000700EA00070022C0B3008B
:10D5900060BB2D00A10B2000B200070022C0B30029
:10D5A000603D2D00A10B2000AE000700E100070048
:10D5B00022C0B30060BB2000A10B2000A90007001F
:10D5C000DC000700D06D80000000E800D06D88000E
:10D5D000D16D8000E06D8000808F5000E6FF390043
:10D5E00055FD37000040EB00A87802000000000065
:10D5F00051FD370030DC20001040780028A10200E7
:10D600000000000010C0B300A87802000000000075
:10D6100049FD370030DC20009040780030C0B30076
:10D6200080C0600030DC20000148780030DC200041
:10D6300090407800A0B4200001487800A0B42000F9
:10D6400090407800F0DB20001040780072830200E8
:10D650000000000010C0B3000286020000000000BD
:10D6600010C0B300A87802000000000032FD3700AF
:10D67000C0B52000104078000040A100C1B52000D6
:10D680008048780030DC2000104078000080FB00EB
:10D690004300DE000000A200610060000004E00022
:10D6A00005003200C0B52000104078000040A00006
:10D6B000C1B520008048780021C0B300F0DB200015
:10D6C0000148780030DC2000104078000080FB002A
:10D6D0004200DE00610060000004E0000300320050
:10D6E00031C0B300F0DB200001487800C0B5200055
:10D6F000104078000030A100C1B5200080487800BB
:10D7000030DC2000104078000080FB000000D100D9
:10D71000610060000004E00005003200C0B5200098
:10D72000104078000030A000C1B52000804878008B
:10D73000A0B4200090407800F0DB2000104078007A
:10D74000728302000000000010C0B30002860200D5
:10D750000000000010C0B300A87802000000000024
:10D76000F5FC37000040EB00A87802000000000044
:10D77000F1FC37000080FA00000006000600FA0005
:10D780002047980031479800424798002E4090006B
:10D790000080FB004600DE00004F78000040EB00F8
:10D7A00010479800220037001E409000E34F5000C1
:10D7B0000C003A001E04E0000A00320010C0B30062
:10D7C000F0850200000000001E80FB00AA9B020002
:10D7D000000000000040EB00F085020000000000A7
:10D7E000100037002E4090000080FB0061006000B8
:10D7F0000004E0000400320010C0B300968502006F
:10D8000000000000030037000040EB009685020096
:10D81000000000002E4090000080FB000000D100BE
:10D82000204798001E4090000040E80010479800F4
:10D830001E409000E34F5000DBFF36003E4090005A
:10D840000080FB00D2840200000000004E409000E7
:10D850000080FB00D2840200000000000080FA007B
:10D86000000006000800FA00100798002107980041
:10D87000624798000040EB0096850200000000001F
:10D880000040EB0096850200000000000040EB0025
:10D8900096850200000000000040EB009685020023
:10D8A000000000001E0090000C9C02000000000020
:10D8B000D2840200000000001E009000AE00900024
:10D8C0004809DD004800DE0000007100C808DE00E5
:10D8D0000C9C020000000000D28402000000000046
:10D8E0001E009000AE0090004008DE000100200005
:10D8F0000C9C020000000000D28402000000000026
:10D900006E4090006F406000604798000040EB0060
:10D91000004F7800020037004FFC07001E4FE80060
:10D920006E4090009E4F1000FBFF39000080FA000F
:10D93000000006000000FA0010C0B3009685020047
:10D94000000000000040EB0096850200000000008F
:10D950000040EB0096850200000000000040EB0054
:10D9600096850200000000000000EB00D284020057
:10D97000000000002685020000000000A8780200D8
:10D98000000000002685020000000000A8780200C8
:10D990000000000030FC07002FFC07000080FA00A8
:10D9A000000006000200FA000040EB00004F780083
:10D9B000905B80000000E0001200320000C2B30063
:10D9C000A878020000000000310020001044200070
:10D9D000489E02000000000000C2B300A8780200C8
:10D9E00000000000805B80000000E00003003A00BF
:10D9F0000040EB0096850200000000000000EB00F4
:10DA0000905B8800805B80000000E00003003A002B
:10DA10002685020000000000004F78001000200062
:10DA2000905B88001E80FB000080FA00000006006A
:10DA30000400FA00000F7800905B80000000E00016
:10DA40001200320000C2B300A878020000000000FB
:10DA50003100200010442000489E02000000000019
:10DA600000C2B300A878020000000000805B8000C4
:10DA70000000E00003003A000040EB009685020041
:10DA8000000000000000EB00905B8800805B8000DD
:10DA90000000E00007003A001E007800D284020077
:10DAA0000000000074850200000000000080FB0000
:10DAB000000F780000C2B300A87802000000000048
:10DAC0001E00E00007003A00310020001044200052
:10DAD000489E02000000000000302000100798005F
:10DAE000060037004100200040442000489E02000C
:10DAF0000000000000102000100798001E00900099
:10DB00000080FA00000006000000FA00905B800030
:10DB10000000E0000F0032004100200040442000DF
:10DB2000489E02000000000040A328007874020014
:10DB300000000000805B80000000E00003003A006D
:10DB400010C0B30096850200000000000000EB004A
:10DB5000905B8800805B80000000E0000F003A00CE
:10DB600000840200000000000000E0000B00320012
:10DB700091002000A0232000489E02000000000029
:10DB80005101200030242000489E020000000000C7
:10DB900040A328007874020000000000D10020009B
:10DBA00080442000D29E0200000000000080FA00A5
:10DBB000000006000000FA00905B80000000E0001A
:10DBC0000F0032004100200040442000489E020027
:10DBD0000000000040A3280078740200000000004C
:10DBE000805B80000000E00003003A0010C0B3003A
:10DBF00096850200000000000000EB00905B8800AA
:10DC0000805B80000000E00002003A0040840200D7
:10DC100000000000C100200050452000D29E0200FC
:10DC2000000000000080FA00000006000000FA007A
:10DC30000101200020522000489E02000000000048
:10DC40000040EB00E47602000000000000C2B300D8
:10DC5000A878020000000000A0B420001040780066
:10DC6000E47602000000000000C2B300A8780200C1
:10DC70000000000050A3280078740200000000009B
:10DC80000080FA00000006000400FA000000EB002B
:10DC9000100798000000EB00805B88002021020044
:10DCA00000000000521D020000000000000F78007C
:10DCB0001E00E00009003400400020009E0F10000C
:10DCC00006003C001E0078000040E900804078001B
:10DCD000A0B4200001487800020037000000EB00EB
:10DCE000000F78001E00E0002D003A000000EB005D
:10DCF000F06788000000EB00805B8800805B80009C
:10DD00000000E0000F003A00B1032000604820004E
:10DD1000D29E0200000000008001EB0042002000C3
:10DD200011002000100020004C2202000000000022
:10DD30000040E90080407800A0B42000014878004D
:10DD400022003700C140800030002300808F500047
:10DD500004003E0051032000104C2000489E0200A9
:10DD600000000000C1022000604F2000489E020019
:10DD7000000000008001EB003200200011002000B4
:10DD8000100020004C220200000000000040E900CA
:10DD900080407800A0B42000014878000B003700D4
:10DDA000C140800030002300808F500004003E00FE
:10DDB00051032000104C2000489E0200000000008B
:10DDC0009AFF07000000EB00905B8800C0B52000C0
:10DDD000104078000040A000C1B5200080487800C5
:10DDE000805B80000000E00009003A00C922A80022
:10DDF000C902A800CB02A900CB22A900A0B4200030
:10DE00009040780020C0B300728302000000000040
:10DE10000080FA00000006000000FA000000EB009D
:10DE2000905B8800805B8000E10F500001003A00A9
:10DE300007E2A9000080FA00000006000600FA00D0
:10DE4000100798001E009000200798002E009000F8
:10DE5000E10F50000C0032002E009000E10F500046
:10DE6000040039002E009000E20F500065003200DF
:10DE7000730037005103200020532000489E020009
:10DE800000000000720037008040EB0000302000EE
:10DE90002086020000000000E102200070562000F1
:10DEA000D29E020000000000CBC2BF0061406000B3
:10DEB0000004E00004003200CBC2BF0062406000FA
:10DEC0000004E0000C003A0091002000A023200094
:10DED000489E020000000000510120003024200074
:10DEE000489E02000000000040A328007874020051
:10DEF00000000000560037000000EB00000F780023
:10DF000039003700805B80000000E00009003A0023
:10DF100000840200000000001E007800D28402008D
:10DF20000000000074850200000000000080FB007B
:10DF3000100798001E0090000000E00024003A0046
:10DF40001E007800049B02000000000080C2B300A5
:10DF5000A8780200000000001E0078000080D100B8
:10DF6000049B0200000000001E0078000000A200D8
:10DF7000610060000004E0000400320070A328008B
:10DF80004C740200000000000B003700805B800032
:10DF90000000E00005003A002685020000000000B5
:10DFA00010C0B3009685020000000000A0A3280066
:10DFB0004C7402000000000050A328004C740200C2
:10DFC0000000000000C2B300A878020000000000BA
:10DFD000805B80000000E00002003A004084020004
:10DFE000000000001E0FE800F00F20009E0F100040
:10DFF000C4FF340040A32800787402000000000031
:10E0000013003700805B8000E10F500001003A00F0
:10E0100007E2A9007100200050592000D29E0200A2
:10E0200000000000F100200010172100D29E020025
:10E030000000000010C0B3000E000700040037000D
:10E0400041022000C0202000D29E020000000000FB
:10E050000080FA00000006000000FA00B100200075
:10E06000C0092100D29E0200000000000080FA00DA
:10E07000000006000A00FA00004F98000040EB0084
:10E08000204798000040EB00104798000040EB004C
:10E09000004F78005079020000000000C922A8005B
:10E0A000C902A800CB02A900CB22A90062A0A80047
:10E0B00062C0A8008660A900CBC2BF000080FB0040
:10E0C0000000D10061406000604798006E40900001
:10E0D00050479800CBC2BF00614060006047980085
:10E0E0006E409000304798000000370086C0BF00A7
:10E0F000684060000004E00012003A0023C2BF0044
:10E10000624060000004E0000E003A009A790200CC
:10E110000000000022C2BF00614060000004E00077
:10E12000F2FF320030118000004F780062A0A90099
:10E1300062C0A9000E4890000004E00061003A00AF
:10E14000630037008660A900CBC2BF000080FB00DF
:10E150000000D1006140600060479800CBC2BF0062
:10E1600061406000404798002E4090000004E000AD
:10E170002E0032003E4090000004E0002B003A00E8
:10E180004E4090000004E000280032001E40900045
:10E19000E74F50000B003E001E407800004040005A
:10E1A000004F78006E4090000004E0000100320053
:10E1B0001E04A0001E4090000040E8001047980098
:10E1C0003B0037000E4890000004E00004003200DD
:10E1D0001E80FB0070770200000000000600370080
:10E1E000C0C5B30064790200000000001E40780042
:10E1F00064790200000000006E4090000004E0001E
:10E2000004003200D0C2B3006479020000000000B4
:10E2100003003700B0C2B3006479020000000000C0
:10E220000040EB0010479800210037003E4090006E
:10E230000004E0001E0032004E4090000004E000A8
:10E240001B0032005E4090000004E0000B00320032
:10E250006E4090000004E00008003A0010C0B300D7
:10E26000204798000040EB0010479800B0C5B3006D
:10E2700064790200000000000D0037005E4090004D
:10E280000004E0000A003A006E4090000004E00044
:10E29000070032000040EB00204798000040EB00F0
:10E2A00010479800D0C5B300647902000000000058
:10E2B0006E409000504798004E40900030479800C4
:10E2C0008AFF370040A32800787402000000000095
:10E2D0000080FA00000006000000FA00D0A3280029
:10E2E0004C740200000000000080FA0000000600EC
:10E2F0000A00FA00881F7800C922A800C902A800F5
:10E30000CB02A900CB22A900C8C2A900C0B5200039
:10E31000104078000040A000C1B52000804878007F
:10E32000C0B52000104078000030A100C1B5200029
:10E330008048780080C0EB0020C0B30072830200E8
:10E3400000000000E4FF07000000370022C2BF0009
:10E35000614060000004E000FCFF320030118000EA
:10E3600080407800E0B6200001487800E0B6200048
:10E37000104078000080FB004400DE008040780000
:10E38000D0B6200001487800D0B6200010407800B8
:10E390000080FB00400798004E009000E10F500005
:10E3A000EB0032004E009000E10F500004003C00F2
:10E3B0004E0090000000E000080032002401370009
:10E3C0004E009000E40F5000190132004E00900002
:10E3D000E60F5000070132001D013700E0B62000B3
:10E3E000104078000080FB00300798003E0090004D
:10E3F000E40F5000330032003E009000E40F500064
:10E4000011003C003E009000E10F50001F00320060
:10E410003E009000E10F500004003C003E009000E0
:10E420000000E0000E013200C50037003E00900001
:10E43000E20F5000170032003E009000E30F500042
:10E440001A003200BE0037003E009000E70F500077
:10E45000280032003E009000E70F500004003C000E
:10E460003E009000E60F50001B003200B400370061
:10E470003E009000E80F5000250032003E00900062
:10E48000EF0F5000A8003200AD00370092FF0700E8
:10E49000AEFF3700008402000000000010C0B3008F
:10E4A000A878020000000000A8FF370040840200A6
:10E4B0000000000010C0B300A878020000000000B7
:10E4C000A2FF37002685020000000000A8780200A5
:10E4D000000000009DFF37000040EB009685020021
:10E4E0000000000010C0B300A87802000000000087
:10E4F00096FF370010C0B3009685020000000000B0
:10E5000010C0B300A8780200000000008FFF3700A1
:10E5100022C2BF00614060000004E000FCFF320046
:10E5200030118000100798001E0090004800DD00A8
:10E530001007980022C2BF00614060000004E000A4
:10E54000FCFF3200301180009E00900000807000BF
:10E550001007980022C2BF00614060000004E00084
:10E56000FCFF320030118000000F78001E007800A0
:10E570004800DD00000F780022C2BF00614060004B
:10E580000004E000FCFF3200301180001E0F70001C
:10E590009E00900000002100808F500003003E008C
:10E5A000000021009E0F1000040036000040EB0028
:10E5B000A87802000000000064FF37000000EB00B4
:10E5C000200798000C00370022C2BF0061406000A5
:10E5D0000004E000FCFF3200714080002E0090003B
:10E5E0008080400030118000804878002E0090002C
:10E5F0000000E80020079800AE0090001E00900088
:10E60000808F5000F0FF39000084020000000000FD
:10E610000000EB00200798000E00370071408000DA
:10E620002E00900000804000104078000080FB0029
:10E63000D284020000000000748502000000000087
:10E64000E14F5000D9FF32002E0090000000E8009A
:10E6500020079800AE0090001E009000808F5000B0
:10E66000EEFF39001E00E900100798000000EB00E3
:10E670002007980014003700714080002E009000A1
:10E68000008440002685020000000000004C780055
:10E69000AE0090001E009000808F500004003100FA
:10E6A0000040EB00968502000000000003003700E8
:10E6B00010C0B30096850200000000002E009000FC
:10E6C0000000E800200798002E0090009E0F5000E8
:10E6D000E9FF3900408402000000000010C0B300D0
:10E6E000A8780200000000000000EB00200798005E
:10E6F00009003700714080002E009000008040002B
:10E7000010407800A8780200000000002E00900061
:10E710000000E800200798002E0090009E0F500097
:10E72000F4FF390009FF37000040EB0051FE0700FD
:10E7300010C0B300A87802000000000003FF3700FB
:10E740000040EB00A878020000000000FFFE370048
:10E75000E0B6200090407800F0C0B30080C06000B8
:10E76000E0B6200001487800E0B6200010407800B4
:10E770008040E800E0B620000148780010C0B300F7
:10E78000A8780200000000008040EB00C0B6200026
:10E79000014878001000370022C2BF0061406000CD
:10E7A0000004E000FCFF320030118000D28402003F
:10E7B000000000007485020000000000A87802003C
:10E7C00000000000C0B62000104078008040E80043
:10E7D000C0B6200001487800C0B620009040780004
:10E7E000E0B620001040780080CF5000EAFF3900EA
:10E7F000D6FE3700E0B620009040780030C0B3006D
:10E8000080C06000E0B6200001487800E0B620003B
:10E810009040780020C0B300728302000000000026
:10E8200010C0B300A878020000000000C7FE370047
:10E83000E0B620001040780028A10200000000008F
:10E8400010C0B300A878020000000000BFFE37002F
:10E850000040EB00A878020000000000BBFE37007B
:10E860004F0478000080FA00000006000200FA0061
:10E87000000F78001E00E0000300320010C3B30058
:10E88000330207000200370000C3B3003002070064
:10E890000080FA00000006000600FA001007980049
:10E8A000020037001E407800290207001E00900079
:10E8B000104F78001E407800404798004E4090006E
:10E8C0000004E0000200320010C0B300404798008E
:10E8D0004E4090009E0090008100E80011079800D3
:10E8E0000004E000EFFF3A000080FA00000006009C
:10E8F0000600FA0010079800020037001E4078005A
:10E90000130207001E009000104F78001E40780090
:10E91000404798004E4090000004E00002003200A2
:10E9200010C0B300404798004E4090009E009000F9
:10E930008100E800110798000004E000EFFF3A00B2
:10E94000D0C0B30002020700A0C0B300000207005D
:10E950000080FA00000006000400FA00204798003A
:10E9600000C8B300004F7800E09F2800CAFF0700EE
:10E970000040EB00104798000F0037002E40900039
:10E980001E4060000004E0000300320010C3B3002A
:10E99000EF0107000200370000C3B300EC010700DD
:10E9A0001E80FB000000D100004F78001E40900048
:10E9B0000040E800104798001E409000E74F5000CC
:10E9C000EEFF36000080FA00000006000E00FA009C
:10E9D00050079800610798000040EB00004F780056
:10E9E00000102E00515F200030079800410798006A
:10E9F0000040EB0010479800320037003E019000C5
:10EA0000CE0190005E009000EE0090003006020003
:10EA10000000000010079800210798001E04E00085
:10EA200005003A001E009000AE009000E00F50007C
:10EA3000E08F5800180032001E0090000043B00024
:10EA4000C30107009E0090003E009000000AB8003D
:10EA50009E0090004E0090000088B90005017800EB
:10EA600000014100BE0090002E0090000088B90017
:10EA700000014100820278005E009000EE009000EC
:10EA800004005000858058005007980061079800E6
:10EA900010C0B300004F78003E009000CE00900000
:10EAA000A200200003002000300602000000000049
:10EAB00030079800410798001E4090000040E80091
:10EAC000104798001E409000E74F5000CBFF3600E3
:10EAD0005E0090000043B0009D0107000080FA0036
:10EAE000000006000C00FA0040079800510798004B
:10EAF0000000EB00100798000000EB00000F78000A
:10EB00006000B80020079800310798004E0190007F
:10EB1000DE019000F0232400F1002000800F51005E
:10EB2000818F5900210036004E009000DE009000D9
:10EB300002242400F3002000300602000000000040
:10EB400020079800310798002E0090006F00070002
:10EB5000C0C2B3007E0107004E009000DE009000AE
:10EB600002242400F30020005006020000000000F0
:10EB700040079800510798004E019000DE01900078
:10EB8000703E200001002000800F5100818F59004D
:10EB900002003E0010A028003FFF070010002000E8
:10EBA0001007980010002000000F78004E01900020
:10EBB000DE019000703E200001002000800F510017
:10EBC000818F5900320036004E009000DE00900028
:10EBD000823E2000030020003006020000000000FA
:10EBE00020079800310798002E019000BE01900088
:10EBF0004006200001002000800F5100818F590045
:10EC0000030036002E00900040000700140037007B
:10EC10001E0090000000E0000F0032002E01900066
:10EC2000BE019000A000200001002000800F5100D4
:10EC3000818F59000300360000C3B3004401070070
:10EC40000200370060A0280013FF07002E0090008C
:10EC50002E000700020037002E0090002B00070056
:10EC6000C0C2B3003A0107004E009000DE009000E1
:10EC7000823E200003002000500602000000000039
:10EC8000400798005107980010002000000F7800FE
:10EC90004E019000DE01900040062000010020009F
:10ECA000800F5100818F5900030036004E00900004
:10ECB00016000700130037001E00E0000F003200AE
:10ECC0004E019000DE019000A00020000100200015
:10ECD000800F5100818F59000300360000C3B3003C
:10ECE0001B0107000200370060A02800EAFE0700B1
:10ECF0004E00900005000700020037004E00900013
:10ED0000020007000080FA00000006000800FA0078
:10ED1000300798000040EB00004F7800007122009F
:10ED2000200798000040EB00104798001E003700B5
:10ED30003E0090002E019000110009000280D800D2
:10ED4000100798001E04E00003003A001E00900027
:10ED50000000E0000C0032001E0090000043B000F4
:10ED6000FB0007009E0090002E0090000088B90074
:10ED7000800078003E0090000100500030079800AD
:10ED800010C0B300004F78002E009000A2002000B9
:10ED9000110009000280D800200798001E40900052
:10EDA0000040E800104798001E409000E34F5000DC
:10EDB000DFFF36003E0090000043B000E400070093
:10EDC0000080FA00000006000600FA0040479800A4
:10EDD0000040EB00004F780040C6B3003047980079
:10EDE0000040EB0020479800200037004E40900084
:10EDF0008080FB003E4090000081FB001100090074
:10EE00008280D800104798001E04E00003003A00FA
:10EE10001E4090000004E0000B0032001E409000F5
:10EE20000043B000CA0007004E4190009E40900091
:10EE30003E4090000088B9000040510040479800D3
:10EE400010C0B300004F78003E4090000080FB00EF
:10EE5000A2002000110009000280D800304798006D
:10EE60002E4090000040E800204798002E4090007F
:10EE7000E14F5000DDFF36004E4090000043B000EF
:10EE8000B30007000080FA00000006000400FA004A
:10EE90001007980090A128007FFE07001E00900038
:10EEA0004400DE006F0F60009E00780090A02800F4
:10EEB0000080400010407800A50007001E00900070
:10EEC0006F0F60009E00780090A028000080400036
:10EED000104078009E0007000080FA000000060045
:10EEE0000400FA001007980000C3B300F600070002
:10EEF00080C7B300F40007001E0090004400DE004D
:10EF00006F0F60009E00780090A0280000804000F5
:10EF100010407800EC0007001E0090006F0F6000AA
:10EF20009E00780090A028000080400010407800EB
:10EF3000E50007000080FA00000006000400FA0067
:10EF40001007980090A1280053FE07001E009000B3
:10EF50004C00DE006F0F60009E00780090A028003B
:10EF60000080400010407800790007001E009000EB
:10EF70004800DE006F0F60009E00780090A028001F
:10EF80000080400010407800710007001E009000D3
:10EF90004400DE006F0F60009E00780090A0280003
:10EFA0000080400010407800690007001E009000BB
:10EFB0006F0F60009E00780090A028000080400045
:10EFC00010407800620007000080FA000000060090
:10EFD0000800FA00300798003E009000CF80DE0065
:10EFE000F403020000000000926C2200B331240000
:10EFF000520402000000000010079800210798004A
:10F000001E009000AE0090005606020000000000B6
:10F01000004F78001E4078006BFF0700E0C2B3008D
:10F020004B0007001E009000AE0090005606020044
:10F0300000000000CF80DE00F403020000000000AA
:10F040000001BE001E009000AE009000D604020039
:10F05000000000001007980021079800020020001F
:10F06000031224001E009000AE00900092050200E2
:10F070000000000010079800210798001E00900073
:10F08000AE0090005606020000000000004F78001D
:10F090001E4078004CFF07001E009000AE0090005C
:10F0A0005606020000000000CF80DE00F4030200DC
:10F0B000000000000001BE001E009000AE009000A5
:10F0C000D6040200000000001007980021079800F5
:10F0D00002002000031224001E009000AE009000E9
:10F0E0009205020000000000100798002107980018
:10F0F0001E009000AE0090005606020000000000C6
:10F10000004F78001E4078002FFF07000080FA00B3
:10F11000000006000000FA0022C2BF00614060004B
:10F120000080FB000080FA00000006000000FA00EA
:10F1300022C2BF00614060000004E000FCFF32001A
:10F14000301180000080FB000080FA000000060003
:10F150000200FA00004F7800D0408000011020002B
:10F16000010060000000E00006003A0023C2BF007A
:10F17000624060000004E000FCFF3A001E00FB005B
:10F18000201188000080FA00000006000200FA004A
:10F19000004F78001E80FB00401188000080FA00BC
:10F1A000000006000000FA0095C0BF00704060003B
:10F1B0000004E00010003A00514080004040800010
:10F1C000808F50000C00320023C2BF0062406000FC
:10F1D0000004E000FCFF3A008580A9009580A800AB
:10F1E00031408000404080000080400010407800A6
:10F1F0000080FB00201188000080FA00000006005B
:10F20000809FBE000000FA00014080002040800086
:10F2100080804000301180008048780020408000CD
:10F220000000E8002040880021408000104080005D
:10F23000808F500001003A009560A9008560A90008
:10F240000080FA004F00BE0000400600809FBE0014
:10F250000000FA00404080000000E80040408800C4
:10F260004140800050408000808F500002003A00F2
:10F270009580A900060037003140800040408000A2
:10F2800000804000104078000080FB0020118800C2
:10F290008580A9000080FA004F00BE0000400600F3
:10F2A0000000FA000000EB00206D88001000200034
:10F2B000106D8800D040800000A0A100D0408800E0
:10F2C0000080FA00000006000200FA00004F7800FB
:10F2D000116D8000206D8000808F500005003A0085
:10F2E000CA82A900D040800000A0A000D0408800C1
:10F2F0000E00370071408000106D8000808040005B
:10F300001E40780080487800106D80000000E80002
:10F31000106D8800116D800000002100808F50006A
:10F3200002003A000000EB00106D88000080FA0037
:10F33000000006000200FA00206D8000000FE800C7
:10F34000000021009E0F100002003A000000EB00B8
:10F35000000F7800106D80009E0F10000C0032002E
:10F3600023C2BF00624060000004E00008003A00D1
:10F370001E007800206D880071408000206D8000A4
:10F3800000804000104078000080FB0020118800C1
:10F390000080FA00000006000200FA0000003700BA
:10F3A000206D8000000FE800000021009E0F10007B
:10F3B00002003A000000EB00000F7800106D8000A2
:10F3C0009E0F10000D00320023C2BF00624060009B
:10F3D0000004E000F2FF3A001E007800206D880073
:10F3E00071408000206D8000008040001040780057
:10F3F0000080FB0020118800E9FF37000080FA0040
:10F40000000006000800FA00200798003107980065
:10F4100090018000100798002E0090009001880055
:10F420003E0090001080BA00C800DD003E00900051
:10F430001000BA00008F70001E009000900188003C
:10F440001E0078000080FA00000006000600FA00A6
:10F450000000EB00800888000000EB00F008880046
:10F460000000EB00E00C8800B05F80000000E000CE
:10F4700008003A00A16C20009140780000CEB30053
:10F4800000C06000CAE6B7000000EB00405F8800E3
:10F490003D003700B05F8000E30F500005003C00E6
:10F4A000E0032000000F780010A1A8001081A80040
:10F4B00015003700B05F8000FE0F500005003C00D3
:10F4C000A00F2000000F780010A1A8001081A90053
:10F4D0000D003700B15F8000400F2000808F50008A
:10F4E00005003C00007D2000000F780010A1A9005D
:10F4F0001081A8000400370000E82300000F780006
:10F5000010A1A9001081A900B05F8000000178005F
:10F510001E007800110009000280D8000000E900F8
:10F52000200798002E00900060088800C05F8000CF
:10F53000800078002E0090000088B900420620006C
:10F54000110009000280D80010079800A16C20006B
:10F550009140780000CEB30000C060006041B3006D
:10F56000CAE6B7001E009000D00C88001E00900074
:10F57000C00C880060002000E00C880011E1A800A9
:10F5800020002000405F88000080FA000000060094
:10F590001200FA000000EB00800888000000EB0079
:10F5A000F00888000000EB00E00C8800405F80005D
:10F5B000E20F500014003A00A16C20009140780046
:10F5C00000CEB30000C06000CAE6B700C100200052
:10F5D000C02E2000D29E0200000000000000EB00C0
:10F5E000405F8800E06780008000E800F00F2000A6
:10F5F00080806000A0BF20000080400010407800A4
:10F600000004E000AC0032000000EB00200798008E
:10F61000E06780008000E800F00F200000806000BC
:10F62000E06788002021020000000000521D020057
:10F6300000000000400798002021020000000000A8
:10F64000521D020000000000CF80DE00F403020023
:10F6500000000000008FBE004E0090000000E0009F
:10F6600007003200CE009000F0F92000808F50009B
:10F6700003003E002E0090000000E80020079800E4
:10F680006011B8001E00BE004A0402000000000025
:10F690000000E00001003C000B00370002002000E9
:10F6A000832C24001E00BE004E0402000000000057
:10F6B0000000E00001003500030037002E0090003C
:10F6C0000000E800200798002E009000E20F500094
:10F6D000110032000000EB00F067880011012000EB
:10F6E000802F2000D29E02000000000011012000A7
:10F6F00090302000489E0200000000008001EB00D6
:10F7000002FA200011002000200320004C220200F9
:10F7100000000000400798004E009000E30F5000EA
:10F7200005003E00E00320003007980010A1A8006B
:10F730001081A800150037004E009000FE0F500009
:10F7400005003E00A00F20003007980010A1A8007F
:10F750001081A9000D003700CE009000400F20005E
:10F76000808F500005003E00007D2000300798008B
:10F7700010A1A9001081A8000400370000E82300B0
:10F780003007980010A1A9001081A9003E00900048
:10F790004E019000110009000280D8000000E9002D
:10F7A000600798002E009000E20F50000E0032001B
:10F7B0000101200070322000489E0200000000007D
:10F7C0008001EB00320620008000EB0020032000C7
:10F7D0004C22020000000000CF80DE00F403020093
:10F7E00000000000008FBE0002002000832C2400D7
:10F7F0001E00BE005204020000000000008FBE0088
:10F800006E009000CF80DE00F403020000000000D4
:10F8100070079800010F98006E0090000000E00053
:10F8200008003D0002002000037824007E009000C4
:10F830008E089000D80402000000000070079800B5
:10F84000010F98001E01BE007E0090008E089000FF
:10F850009205020000000000FA050200000000000E
:10F8600050079800A16C20009140780000CEB300B2
:10F8700000C060006041B300CAE6B7005E009000BF
:10F88000D00C88005E009000C00C88006000200052
:10F89000E00C88006E0090006008880011E1A8006C
:10F8A000A100200070332000D29E02000000000062
:10F8B00020002000405F88000080FA000000060061
:10F8C0000000FA00405F8000E20F500005003A009F
:10F8D000F101200010342000D29E02000000000040
:10F8E0003E003700F100200000362000489E020054
:10F8F000000000000000EB00F00888000000EB00B2
:10F9000080088800C942A800616820009140780002
:10F9100000CEB30000C06000A040B30086E6B70090
:10F92000A0032000800888002E000700505F880098
:10F93000615F8800525F8000635F8000F00F2000ED
:10F9400001002000800F5100818F5900090036000E
:10F95000505F8000615F8000C808DD000080FD000E
:10F96000804078000040EB00505F8800615F8800B5
:10F9700009003700B100200000122100489E02005B
:10F9800000000000A000200080088800150007008B
:10F99000505F8800615F8800505F8000615F800079
:10F9A000727502000000000000A628004C740200DE
:10F9B0000000000040A6280078740200000000004B
:10F9C00086C6BF00F041B30086E6B7000000EB003A
:10F9D000F00888000000EB00800888000080FA0032
:10F9E000000006000000FA000080EB0070088800AC
:10F9F0000080EB00600888000000EB0040088800F1
:10FA00000000EB00300888000000EB00B008880020
:10FA10000000EB00A008880080002000F0088800AB
:10FA2000400F2000E008880000402200D008880035
:10FA30008780A9001FE1A80011E1A80087C0BF00CE
:10FA4000704060000004E000FCFF320011E1A900FA
:10FA50001FE1A90030088000A05F880040088000F6
:10FA6000905F8800905F800001002000705F880038
:10FA7000815F8800705F8000815F8000C000DD00D2
:10FA800000002000705F8800815F8800A05F800018
:10FA90006101B800705F8000815F8000020040005B
:10FAA00083804800705F8800815F8800705F8000FD
:10FAB000815F80000080FA00000006000000FA006C
:10FAC000C0B5200010407800634060000004E000F2
:10FAD00002003A00C942A80001003700C8C2A800CD
:10FAE000E1002000F0362000489E020000000000E7
:10FAF0000080FA00000006000000FA00C0B52000F7
:10FB000010407800634060000004E00003003A0009
:10FB1000C942A900CB42A80002003700C8C2A90010
:10FB2000CAC2A80081002000D0372000D29E020067
:10FB3000000000000080FA00000006000000FA004B
:10FB4000C0B5200010407800634060000004E00071
:10FB500003003A00C942A900CB42A90002003700C5
:10FB6000C8C2A900CAC2A9007100200050382000F4
:10FB7000D29E0200000000000080FA000000060093
:10FB80000200FA00C0B52000104078006340600019
:10FB90000004E00009003A00C942A800000000008B
:10FBA00000000000CBC2BF000080FB004200DE006E
:10FBB00061406000004F780008003700C8C2A8000C
:10FBC0000000000000000000CAC2BF000080FB006F
:10FBD0004600DE0061406000004F78001E80FB00A0
:10FBE0000080FA00000006000C00FA000000EB00A4
:10FBF000800888000000EB00F00888000000EB009F
:10FC0000E00C8800405F8000E20F500014003A00D2
:10FC1000A16C20009140780000CEB30000C06000CD
:10FC2000CAE6B700C1002000C02E2000D29E02000C
:10FC3000000000000000EB00405F8800E0678000EB
:10FC40008000E800F00F200080806000A0BF20004E
:10FC500000804000104078000004E00064003200A2
:10FC6000E06780008000E800F00F20000080600066
:10FC7000E06788002021020000000000521D020001
:10FC800000000000CF80DE00F4030200000000004E
:10FC9000008FBE00F06780000000E00008003A001E
:10FCA00002002000433324001E00BE004A0402006C
:10FCB000000000000000E00001003C0010003700E0
:10FCC0000000EB00F067880031012000901C21004B
:10FCD000D29E0200000000008001EB00420B2000D9
:10FCE0008000EB00A00520004C2202000000000074
:10FCF000CF80DE00F403020000000000008FBE0091
:10FD000010A1A8001081A800204E20003007980004
:10FD100002002C00A35524001E00BE005204020065
:10FD200000000000008FBE003E009000CF80DE008B
:10FD3000F4030200000000004007980051079800FB
:10FD40003E0090000000E00008003D00020020009E
:10FD5000037824004E009000DE009000D8040200DA
:10FD60000000000040079800510798001E01BE00E7
:10FD70004E009000DE00900092050200000000009E
:10FD80000200200083272400D804020000000000A5
:10FD9000FA0502000000000020079800A16C200076
:10FDA0009140780000CEB30000C060006041B30015
:10FDB000CAE6B7002E009000D00C88002E009000FC
:10FDC000C00C880060002000E00C88003E0090001D
:10FDD0006008880011E1A800C1002000C01D2100BA
:10FDE000D29E02000000000020002000405F88003A
:10FDF0000080FA00000006000000FA00C0A62800FB
:10FE00004C740200000000000080FA0000000600B0
:10FE10000200FA00CA82A800FA000700F6FF0700F5
:10FE200000003700EE0007008040780080DB2000F3
:10FE30000148780080DB2000104078000004E000DA
:10FE4000E100350080DB2000104078000004E00075
:10FE500002003A00E8FF0700F2FF370080DB2000D5
:10FE600010407800E14F500006003A00E50007001E
:10FE7000BC4F020000000000E2000700DEFF0700A8
:10FE8000E8FF370080DB200010407800E24F500090
:10FE900006003A00DB000700787102000000000055
:10FEA000D8000700D4FF0700DEFF370080DB20000A
:10FEB00010407800E34F500006003A00D1000700E0
:10FEC0008258020000000000CE000700CAFF0700B1
:10FED000D4FF370080DB200010407800E44F500052
:10FEE00006003A00C7000700786302000000000027
:10FEF000C4000700C0FF0700CAFF370080DB2000F6
:10FF000010407800E54F500006003A00BD000700A1
:10FF10005C65020000000000BA000700B6FF0700A1
:10FF2000C0FF370080DB200010407800E64F500013
:10FF300004003A00B3000700B2000700AEFF07005C
:10FF4000B8FF370080DB200010407800E74F5000FA
:10FF500004003A00AB000700AA000700A6FF070054
:10FF6000B0FF370080DB200010407800EF4F5000DA
:10FF70000A003A0010C0B300A87802000000000098
:10FF8000CA82A90023C2BF00614060000004E000F3
:10FF9000FCFF32000000FE00A2FF370080DB2000E3
:10FFA00010407800F24F500035003A000000EB009E
:10FFB000800888000000EB00F00888000000EB00DB
:10FFC000E00C8800A16C20009140780000CEB300C6
:10FFD00000C060006041B300CAE6B70080000700BF
:10FFE0000080FB00000F78001E0078000000D100A8
:10FFF000610060000004E0000100320010A1A800D0
:020000040001F9
:100000009E007800618060000004E0000100320082
:100010001081A800720007000080FB004800DD008E
:10002000000F78006E0007000080FB001E0F7000BC
:100030001E007800D00C88009E007800C10C88005B
:1000400060002000E00C8800650007000080FB00D5
:100050004800DD00000F7800610007000080FB0011
:100060001E0F70001E0078006008880011E1A800D3
:1000700010C0B300A87802000000000069FF37003C
:1000800080DB200010407800F34F50000D003A0054
:100090000000EB00800888000000EB00E00C880006
:1000A000A16C20009140780000CEB30000C0600039
:1000B000CAE6B70010C0B300A87802000000000034
:1000C00058FF370080DB200010407800F44F5000CC
:1000D0000E003A0021E3A800C0C0B3004C9A020011
:1000E00000000000000F780021E3A9001E00780046
:1000F0004800DE00A8780200000000001E00780022
:10010000A87802000000000046FF370080DB2000D6
:1001100010407800F54F500018003A0021E3A80085
:10012000C0C0B3004C9A020000000000000F78002D
:1001300023C2BF00614060000004E000FCFF320009
:100140001E0078004800DE00A878020000000000D1
:100150001E007800A87802000000000022C2BF0044
:10016000614060000004E000EDFF320031118000CA
:10017000010F780021E3A9002AFF370080DB20006F
:10018000104078000080FB004500DE000080FB008E
:100190000000D100610060000004E00006003200B1
:1001A00080DB2000104078001F000700A8780200C4
:1001B000000000001BFF37000040EB00A8780200A1
:1001C0000000000017FF370080DB2000104078009F
:1001D000A5000700A87802000000000011FF37000A
:1001E0000000FA0022C2BF00614060000004E0008D
:1001F000FCFF3200301180000080FB000080FA001C
:10020000000006000000FA0000C0EB000600070036
:100210000040EB0094000700C962A900CB62A9006E
:100220000080FA00000006000400FA002047980051
:100230000040EB00004F78002E4090000080FB0053
:100240004400DE00610060000004E00002003200B3
:1002500010C0B300004F78009E40780061C060007D
:10026000614060004201DD00912C20009140780047
:10027000B0CFB30000C0600002407000C9E2B70018
:100280000040EB00004F78002E4090000080FB0003
:100290004300DE00610060000004E0000200320064
:1002A00010C0B300004F78009E40780061C060002D
:1002B0006140600000414000912C20009140780096
:1002C000D0CFB30000C0600002407000C9E2B700A8
:1002D0000040EB00004F78002E4090000080FB00B3
:1002E0004200DE00610060000004E0000200320015
:1002F00010C0B300004F78009E40780061C06000DD
:1003000061416000912C200091407800E0CFB30063
:1003100000C0600002407000C9E2B7000040EB007E
:10032000004F78002E4090000080FB000000D100BC
:10033000610060000004E0000200320010C0B30061
:10034000004F78009E40780061C06000C700DD006B
:10035000C8C2BF000074A10001407000C8E2B7002D
:100360000040EB00004F78002E4090000080FB0022
:10037000610060000004E0000200320010C0B30021
:10038000004F78009E40780061C0600061406000CE
:100390004601DD00812C200091407800F0CBB300B5
:1003A00000C0600002407000C8E2B70050002000AA
:1003B000D69B020000000000AE40900000CEB300CB
:1003C00000C0600020479800CBC2BF0064406000BE
:1003D0000004E000030032002E4090000044A00022
:1003E00020479800CBC2BF00624060000004E000DC
:1003F000030032002E4090000034A00020479800F7
:10040000CBC2BF00614060000004E0000300320086
:100410002E4090000024A00020479800CAC2BF00D0
:1004200001C8B300014060000004E0000300320096
:100430002E4090000014A00020479800CAC2BF00C0
:100440000044B2000004E000030032002E4090009F
:100450000004A000204798002E4090000080FB0080
:100460000080FA00000006000400FA00204798000F
:100470002E4090000080FB004600DE00610060001E
:100480000004E00005003200C082A900C282A8007A
:10049000C8A2A900CAA2A80004003700C082A9000F
:1004A000C282A900C8A2A900CAA2A9000040EB000C
:1004B000004F78002E4090000080FB004400DE00DA
:1004C000610060000004E0000200320010C0B300D0
:1004D000004F78009E40780061C06000614060007D
:1004E0004201DD00B12C200091407800B0CFB30074
:1004F00000C0600002407000CBE2B7000040EB009B
:10050000004F78002E4090000080FB004300DE008A
:10051000610060000004E0000200320010C0B3007F
:10052000004F78009E40780061C06000614060002C
:1005300000414000B12C200091407800D0CFB300A2
:1005400000C0600002407000CBE2B7000040EB004A
:10055000004F78002E4090000080FB004200DE003B
:10056000610060000004E0000200320010C0B3002F
:10057000004F78009E40780061C0600061416000DB
:10058000B12C200091407800E0CFB30000C06000A3
:1005900002407000CBE2B7000040EB00004F780053
:1005A0002E4090000080FB000000D1006100600040
:1005B0000004E0000200320010C0B300004F7800D9
:1005C0009E40780061C06000C700DD00CAC2BF0065
:1005D0000074A10001407000CAE2B7000040EB00C7
:1005E000004F78002E4090000080FB00610060000A
:1005F0000004E0000200320010C0B300004F780099
:100600009E40780061C06000614060004601DD00EE
:10061000A12C200091407800F0CBB30000C0600016
:1006200002407000CAE2B70050002000D69B0200D2
:1006300000000000AE40900000CEB30000C060009B
:1006400020479800CBC2BF00644060000004E00077
:10065000030032002E4090000044A0002047980084
:10066000CBC2BF00624060000004E0000300320023
:100670002E4090000034A00020479800CBC2BF005D
:10068000614060000004E000030032002E40900052
:100690000024A00020479800CAC2BF0001C8B300D0
:1006A000014060000004E000030032002E40900092
:1006B0000014A00020479800CAC2BF000044B20046
:1006C0000004E000030032002E4090000004A0006F
:1006D000204798002E4090000080FB000080FA0028
:1006E000000006000400FA00004F7800114798004F
:1006F000E0DA20001E48780030C0B3009E4F1000A2
:1007000005003A0000202000806D880000082000CD
:10071000906D88000400370000202000806D880064
:1007200000202000906D88001E4090000080FB009B
:10073000100798001E009000E10F500011003200D9
:100740001E009000E20F5000180032001E009000C2
:100750000000E000010032001E00370041C1B3007C
:1007600040DB20000148780041C6B30050DB200088
:100770000148780021C3B30060DB20000148780005
:100780001D00370021C0B30040DB20000148780085
:10079000A1C0B30050DB20000148780051C0B30075
:1007A00060DB2000014878001300370011C0B3005F
:1007B00040DB20000148780051C0B30050DB20002E
:1007C0000148780021C0B30060DB200001487800B8
:1007D000090037008040EB0040DB20000148780032
:1007E0008040EB0050DB2000014878008040EB00A7
:1007F00060DB2000014878000080FA00000006005D
:100800000200FA000000EB00000F780050DB20002F
:10081000904078000030200009010700CBC2BF00E3
:10082000614060000004E00004003200CBC2BF0061
:10083000624060000004E00002003A001000200066
:10084000000F780050DB200090407800002020004E
:100850001701070050DB20009040780000102000B6
:100860001301070050DB200090407800002020009A
:10087000F30007001E0078000080FA000000060068
:100880000000FA0050DB200090407800003020008B
:100890000701070050DB2000904078000010200086
:1008A000E700070050DB2000904078000020200087
:1008B000E30007000000EB000080FA0000000600E3
:1008C0000C00FA00500798000000EB00000F7800C1
:1008D000B0B42000104078000080FB008000E900E8
:1008E000100020000100DD00300798005E0090003D
:1008F000200798000000EB00400798002000370018
:1009000040DB200010417800AE0090003E009000D7
:100910000080600001202000FC00070050DB200068
:100920009040780000102000C5000700000820005B
:10093000260107000080FB001007980050DB200014
:100940009040780000102000D90007002E00900091
:1009500000004000200798001E00780000004000C2
:10096000000F78001E0090000000E000010032003F
:100970001E0FE8004E0090000000E80040079800BD
:10098000B0B42000104078008080FB004E00900042
:10099000808F5000DAFF3E001E0078000080FA00D1
:1009A000000006000800FA0030079800B0B42000EC
:1009B000104078000080FB008000E900100020005B
:1009C0000100DD00100798003E009000000F780045
:1009D0000000EB00200798001400370040DB2000E7
:1009E000104178001E0090001E00600001202000D1
:1009F000C600070050DB2000904078000010200067
:100A00008F00070050DB200090407800001020008D
:100A1000A70007001E00780000004000000F7800CB
:100A20002E0090000000E80020079800B0B42000DD
:100A3000104078008080FB002E009000808F5000D6
:100A4000E6FF3E000080FA00000006000600FA0003
:100A50000000EB00000F780000202000DB00070002
:100A60000000EB00200798001600370050DB200044
:100A70009040780000102000710007000020200046
:100A8000D20007000080FB001007980050DB200018
:100A90009040780000102000850007001E007800BC
:100AA00000004000000F78001E0090000000E000F1
:100AB000010032001E0FE8002E0090000000E80048
:100AC00020079800B0B42000104078008080FB0020
:100AD0002E009000808F5000E4FF3E001E00780042
:100AE0000080FA00000006000200FA00906D80000D
:100AF000B600070050DB2000904078000010200076
:100B00004F000700906D8000B0000700004F780094
:100B100050DB2000904078000010200064000700A7
:100B20001E80FB000080FA00000006000200FA00B0
:100B3000004F780040DB200010417800816D80007C
:100B40001E80FB007100070050DB20009040780001
:100B5000001020003A00070050DB20009040780091
:100B600000102000520007000080FA00000006007C
:100B70000400FA00204798000040EB00004F780086
:100B80000900370050DB2000904078000010200062
:100B90002B00070050DB2000904078000010200060
:100BA000430007001E4FE8002E4090009E4F1000AB
:100BB000F4FF39000080FA00000006000200FA008D
:100BC000004F780040DB200010417800816D8000EC
:100BD0001E80FB004D0007000080FA0000000600A8
:100BE0000200FA00004F780040DB2000104178003E
:100BF0001E80FB0001102000440007000080FA0066
:100C0000000006000200FA00004F780040DB2000E0
:100C1000104178001E80FB00010420003B0007000B
:100C20000080FA00000006000000FA00906D8000CD
:100C3000660007000080FB000080FA00000006004C
:100C40000400FA00000F780021479800C0B520008A
:100C500010407800704060000004E0000B003A0093
:100C6000601680001E007000601688001E0078006C
:100C70000080EA008180EA00800078004016800051
:100C80000080600040168800030037004016800096
:100C90001E007000401688002E4090000080FB006F
:100CA000D69B0200000000000080FA000000060051
:100CB0000400FA00000F7800214798001E00780019
:100CC0000080EA008180EA008000780060168000E1
:100CD00000806000601688001E0078000080EA0036
:100CE0008180EA008000780040168000008060006B
:100CF000401688002E4090000080FB00D69B02002A
:100D0000000000000080FA00000006000600FA0063
:100D1000000F780011079800424798001E00E0007D
:100D20000F003A001E0090000080EA008180EA0077
:100D300080007800601680000080600060168800E7
:100D40001E0090000080EA008180EA0080007800A8
:100D500040168000008060004016880015003700B3
:100D6000C0B5200010407800704060000004E00032
:100D70000C003A00611680001E0090000080700098
:100D8000601688001E0090000080EA008180EA0062
:100D900080007800401680000080600040168800C7
:100DA00004003700401680009E0090000100700093
:100DB000401688004E4090000080FB00D69B020049
:100DC000000000000080FA00000006000400FA00A5
:100DD000000F7800401680001E007000401688004A
:100DE000000000000000000000000000501680001D
:100DF0001E0060000000E000030032001000200030
:100E000010079800020037000000EB001007980060
:100E10001E0090000080FA00000006000000FA00AA
:100E200026850200000000000080FA000000060095
:100E30000200FA00000F78001E007800D284020041
:100E400000000000001020000080FA0000000600F2
:100E50000000FA0000840200000000008100200071
:100E6000D0922000489E020000000000D100200027
:100E700080442000D29E0200000000000080FA00A2
:100E8000000006000000FA0040840200000000009C
:100E90006100200050932000489E020000000000E6
:100EA000C100200050452000D29E0200000000003A
:100EB0000080FA00000006000000FA0074850200BD
:100EC000000000000080FB000080FA000000060027
:100ED0000000FA0014860200000000000080FB0001
:100EE0000080FA00000006000000FA000040EB005D
:100EF000F0850200000000000080FA0000000600FB
:100F00000000FA0010C0B300F085020000000000ED
:100F10000080FA00000006000000FA0010C0B300D4
:100F2000B8850200000000000080FA000000060002
:100F30000000FA000040EB00DE8502000000000027
:100F40000080FA00000006000000FA0010C0B300A4
:100F5000DE850200000000000080FA0000000600AC
:100F60000000FA0001012000A0982000489E020025
:100F700000000000A0B4200010407800E4760200D9
:100F80000000000000C2B300A878020000000000CA
:100F9000C0B52000104078000080FB004400DE0057
:100FA00061406000E47602000000000000C2B3006F
:100FB000A87802000000000031002000F0AD200001
:100FC000489E0200000000000080FA0000000600B9
:100FD0000400FA002021020000000000521D02005F
:100FE000000000001007980020210200000000000F
:100FF000521D020000000000000F78001E0090004B
:101000000000E000090034001E009000E40F5000D2
:1010100006003C001E0090000040E900804078007F
:10102000A0B4200001487800020037000000EB0067
:10103000100798001E00E00010003400200020007F
:101040009E0F10000D003C001E0078000040EA00DA
:1010500061416000C0B520009040780061406100AF
:101060004401DD00F0CEB30080C0600082C070009B
:10107000C0B5200001487800020037000000EB00F6
:10108000100798001E0090000000E00026003A00C3
:101090000000EB00F0678800B103200060482000EA
:1010A000D29E0200000000008001EB004200200000
:1010B00011002000100020004C220200000000005F
:1010C0000040E90080407800A0B42000014878008A
:1010D000F1042000B0932000D29E02000000000026
:1010E0008001EB00220020001100200010002000F1
:1010F0004C220200000000000040EA006141600054
:10110000C0B5200090407800614061004401DD00DE
:10111000F0CEB30080C0600082C07000C0B5200077
:1011200001487800010037008DFF0700CB02A900BD
:10113000CB22A900C922A800C902A900A0B420009E
:101140009040780020C0B3007283020000000000CD
:101150000080FA00000006000400FA00000F78008A
:101160001E007800100798001E009000E10F50004C
:101170000C0032001E009000E10F50000400390006
:101180001E009000E20F50000700320008003700F8
:1011900081032000A0992000489E0200000000006A
:1011A0000700370010000700250007000400370083
:1011B00041022000C0202000D29E0200000000005A
:1011C0000080FA00000006000200FA00000F78001C
:1011D000B1002000C0092100D29E020000000000E2
:1011E0000080FA00000006000000FA00F103200071
:1011F000209D2000D29E0200000000000040EB0075
:101200000286020000000000F00F2000D69B0200C2
:101210000000000010C0B3000286020000000000C1
:1012200010C0B300B8850200000000000040EB00D1
:1012300002860200000000000080FA0000000600A4
:101240000A00FA00881F7800D102200010A12000B7
:10125000489E0200000000000000EB00000F780034
:10126000100037001E0478002685020000000000F0
:101270008040780063004700017478009E00780089
:1012800063004700614078000080FB004677020061
:101290000000000000C2B300A878020000000000B7
:1012A0001E0FE800300020009E0F1000EDFF3600FA
:1012B00000A828007874020000000000A1002000AF
:1012C000E0A32000489E02000000000063004700E9
:1012D000104078000080FB004400DE000080FB002E
:1012E000400798004E009000E90F500013003200B4
:1012F0004E009000E90F500004003C004E009000AA
:10130000E80F5000080032001B0037004E0090002C
:10131000EA0F50000E0032004E009000EF0F500018
:1013200010003200140037006100200080A420006B
:10133000489E0200000000001300370061002000FA
:10134000E0A42000489E0200000000000E003700CC
:101350006100200040A52000489E0200000000001F
:101360000900370031002000A0A52000489E02009F
:10137000000000000400370071002000D0A520000C
:10138000489E02000000000000A8280078740200B7
:1013900000000000B100200040A62000489E02008E
:1013A0000000000063004700104090000080FB0038
:1013B0004700DE000004E00005003A006100200064
:1013C000F0A62000489E0200000000000400370044
:1013D000F100200050A72000489E020000000000FD
:1013E00000A828007874020000000000C10020005E
:1013F00040A82000489E0200000000006300470053
:10140000104090008080FB0080F72F00008060007B
:101410004380DE00204798002E4090000004E0004A
:1014200005003A00D100200000A92000489E0200DB
:10143000000000001E0037002E409000EF4F5000CB
:1014400005003A0031002000A0A52000489E0200BF
:10145000000000001600370000042000000F780094
:10146000E30047000040EB008048780008003700A8
:101470001E00780000004000000F78006300470065
:10148000104078008040E800630047000148780081
:1014900063004700904078002E40900080CF5000BD
:1014A000F3FF39001E00780086760200000000007D
:1014B00000A82800787402000000000091012000BC
:1014C000D0A92000489E02000000000063004700F1
:1014D0009040900070C0B30000C0600020479800AA
:1014E00010002000000F7800E30047000040EB00F0
:1014F00080487800080037001E0078000000400097
:10150000000F780063004700104078008040E8003A
:10151000630047000148780063004700904078006E
:101520002E40900080CF5000F3FF39001E0078005D
:10153000E47602000000000000A828007874020091
:10154000000000004F0478000080FA000000060050
:101550000000FA0040168000017C200001007000AD
:10156000401688001100070020C0B3002D000700BE
:101570008A780200000000000004E000050032004C
:101580009678020000000000260007000004E0003A
:1015900004003A00700107000004E00001003A0076
:1015A000F3FF37000080FA00000006000000FA0098
:1015B000CA82A9000000EB00400388000000EB0095
:1015C000500388000000EB00000388000000EB00DF
:1015D000100388000000EB00F0088800D10A20000A
:1015E00091407800F0C8B30000C06000ADE0B700E3
:1015F0000000EB00E008880000642000D0088800AC
:1016000000002100C06E88008040EB0060DD2000FB
:10161000014878000000EB00206E88000080FA008E
:10162000000006000A00FA00004F7800706E80008B
:1016300040079800CE009000E18F50007E003200FD
:101640004E019000E10F5100040039004E0090005F
:10165000E20F5000890032003A0137009E80FB0003
:10166000310798003E019000E20F5100180032004F
:101670003E009000E20F500007003C00BE009000CA
:101680000100E0000E0032003E019000E10F510029
:10169000130032005D0037003E009000F10F500053
:1016A00028013200BE009000F38F50002501320067
:1016B0003E019000E40F51001D003200530037003E
:1016C000BAFF070010002000200798001F01370014
:1016D000E0A428004C74020000000000190137004B
:1016E000CA82A8000000EB00F00888000000EB00B0
:1016F000B00888000000EB00A008880080002000EF
:10170000F00888008660A9009660A900D10A200030
:1017100091407800F0C8B30000C060000044A00011
:10172000ADE0B70010002000206E880005013700F2
:1017300010C0B300A87802000000000030A5280007
:101740004C740200000000000040EB00A87802008A
:101750000000000010C2B300A878020000000000E2
:101760000040EB00A8780200000000000040EB0001
:10177000A87802000000000000C1B300A8780200B1
:10178000000000000040EB00A8780200000000000C
:1017900030C2B300A8780200000000000040EB0057
:1017A000A878020000000000F0C0B300A878020092
:1017B0000000000020C4B300A87802000000000070
:1017C00000C4B300A87802000000000000C4B30009
:1017D000A87802000000000050C0B300A878020002
:1017E0000000000010C4B300A87802000000000050
:1017F00020C0B300A8780200000000000040EB0009
:10180000A878020000000000CE00370060DC200055
:101810001E48780041C0B300B0DC200001487800C9
:101820008040EB00C0DC2000014878001000200060
:10183000706E8800C3003700C0DC200010407800C4
:101840008040E800C0DC200001487800C0DC2000B7
:10185000104078008080FB0060DC200000804000A9
:101860001E487800C0DC200090407800B0DC2000EA
:101870001040780080CF5000B200390060DC2000BA
:10188000104078000080FB0010079800100820002E
:101890009E009000808F50003E003200000C20001F
:1018A0001E019000800F510005003200000820004A
:1018B0009E009000808F50004E0032009F00370045
:1018C00070DC2000104078000080FB004400DE0047
:1018D000610060000004E00003003200100380009B
:1018E0000000A0001003880070DC20001040780089
:1018F0000080FB004300DE00610060000004E000A7
:10190000040032001003800001022000010070007A
:101910001003880070DC2000104078000080FB007D
:101920004200DE00610060000004E00004003200BC
:1019300010038000010420000100700010038800E3
:1019400070DC2000104078000080FB000000D10017
:10195000610060000004E000040032001003800019
:1019600001082000010070001003880070DC2000D6
:10197000104078000080FB00610060000004E0007F
:1019800004003200100380000110200001007000EC
:101990001003880080DC2000104078000080FB00ED
:1019A000C06E8800C06E80004800DD00C06E8800F8
:1019B00070DC2000104078008080FB00C06E80004A
:1019C00000807000C06E8800C06E80004200DD00A4
:1019D00064004000C06E8800C16E800000002100DD
:1019E000808F50005500360000002100C06E880036
:1019F0005200370090DC2000104078000080FB008F
:101A000001002000806E8800916E8800806E80004A
:101A1000916E8000C808DD000080FD0080407800E5
:101A20000040EB00806E8800916E880080DC200012
:101A3000104078000081FB0003002000806E8000D1
:101A4000916E80000000710081807100806E8800BE
:101A5000916E8800806E8000916E8000C808DD0065
:101A60000080FD00804078000040EB00806E880020
:101A7000916E880070DC2000104078000081FB002F
:101A800003002000806E8000916E800000007100D5
:101A900081807100806E8800916E8800806E800069
:101AA000916E80004209DD00CE00DE0081007100F1
:101AB0004200DD0064004000E08048009201200008
:101AC000030020003006020000000000806E880045
:101AD000916E8800826E8000936E8000000120006D
:101AE00001002000800F5100818F5900070036004F
:101AF000806E8000916E800070005000E080580081
:101B0000806E8800916E880004003700100020006D
:101B100001002000806E8800916E8800806E800039
:101B2000916E80004008DE0001002000E00888007F
:101B3000806E8000916E8000D00888000000EB006D
:101B4000706E88000000EB00200798002E009000C7
:101B50000080FA00000006000200FA00206E8000FB
:101B6000E10F5000010032003600370086C0BF0090
:101B7000684060000004E00003003A0010038000A9
:101B80000000E0002F003A001FE1A8008780A900B4
:101B90000000EB00A06E88000E003700714080004E
:101BA000A06E800080804000501680004600DE005D
:101BB0008048780087C0BF00704060000004E000EB
:101BC000FCFF32008780A900A06E80000000E800C2
:101BD000A06E8800A16E8000C06E8000808F5000D3
:101BE000EEFF39000000EB00100388000000EB005E
:101BF000F0088800C06E8000A06E88000A003700E0
:101C000071408000A06E8000008040000000E9006C
:101C100010407800A878020000000000A06E80004C
:101C20000000E900A06E8800A06E80000000E000C7
:101C3000F3FF3A005DFE070010002000000F78005F
:101C4000020037000000EB00000F78001E00780053
:101C50000080FA00000006000200FA00000F780081
:101C60001E00780080407800202421001040780079
:101C70000080FB000000D1006140600044010700CB
:101C8000001020000080FA00000006000000FA00AA
:101C900020242100104078000010A1002124210000
:101CA0008048780041012000B0EC2000D29E020064
:101CB000000000000080FA00000006000000FA00AA
:101CC00020242100104078000010A00021242100D1
:101CD0008048780021012000F0ED2000D29E020013
:101CE000000000000080FA00000006000000FA007A
:101CF000C0B52000104078000040A000C1B5200011
:101D00008048780020242100104078000010A000B6
:101D10002124210080487800816A200091407800C9
:101D200000CEB30000C060007040B300A8E6B7006A
:101D3000916C20009140780000CEB30000C060009C
:101D40007040B300C9E6B700816C20009140780074
:101D500000CEB30000C060000034A000C8E6B700A9
:101D6000CAC2A900C8C2A900C902A900C8E2A80045
:101D7000C922A900D0132000101288000000EB0037
:101D8000201288000000EB000012880041E2A80049
:101D9000D101200040F02000D29E0200000000008F
:101DA0000080FA00000006000800FA0020079800F2
:101DB000E06780008000E800F00F200000806000F5
:101DC000E06788002021020000000000521D020090
:101DD00000000000100798000000EB00F06788008A
:101DE0002E009000300798003E009000E30F500056
:101DF0003C0032003E009000E30F500004003E0023
:101E00003E0090000000E0000B0032000F003700A1
:101E10003E009000E60F5000480032003E00900067
:101E2000E70F50006A0032003E009000E40F5000BF
:101E3000370032008B0037008109200060F6200057
:101E4000D29E0200000000008A00370051002000EE
:101E500030632000D29E020000000000AC000700AA
:101E60002E009000E10F5000820032001E00900012
:101E70000000E000030034001E009000E20F50005C
